:1080940020002A2A2000202A2A20002020204164AF
:1080A40064726573733A20202530345800202020F0
:1080B4002020536C617665206D6F6465200020205C
:1080C4002020205265766973696F6E3A002573002B
:1080D40057726F6E672043504C44206669726D7707
:1080E40061726500536C61766520616464723A2044
:1080F400256264005265713A202530326264202181
:108104003D204163743A202530326264004F766525
:108114007263757272656E74203E312E3541206F24
:108124006E00202020323456206F757470757420D0
:1081340021212120202000202020536C61766520FD
:10814400616464723A2025626400524553455400C8
:108154004F76657263757272656E74203E302E358B
:1081640041206F6E00202020203556206F757470DA
:108174007574202121210020202020536C61766514
:1081840020616464723A2025626400202020205516
:10819400203D2025312E32662056004E6577206D15
:1081A4006F64756C6520696E20706F72742025622F
:1081B4006400506C6573652073656C6563743A0084
:1081C4003E25303262582025732020202020202094
:1081D40020202020200053454C2020202020202037
:1081E4002020202020204E4558540053454C202068
:1081F40020202020202050524556202020202000DE
:1082040053454C2020202020202020505245562029
:108214004E455854004D4F4420205641525320207F
:1082240053595320202020202000502562643A25F1
:108234003032625820257320202020202020202046
:10824400200020202020202020202020202020204A
:1082540020202020202000455343202020202020BF
:1082640000202025632000202020200045534320A7
:10827400455241534520202020202020202020202A
:108284000045534320455241534520205052455602
:10829400204E4558540020202020457261736520EB
:1082A4006D6F64756C6520202020002020202069DB
:1082B4006E20706F727420256264203F202020009D
:1082C400534C415645204D4F44450041646472650A
:1082D4007373202532626400323031352D30362DEF
:1082E4003132202D2032613231336138005343530F
:0682F4002D323030310094
:10B66A00017D01C116C110C117C118C111C112C192
:10B67A0013C1154400A9000000004400AD000000F9
:09B68A000041114100411146008C
:02700C008F44AF
:10700E0090114874FFF07D017F0012B86C7D007FF7
:10701E000112B86CE4901A26F0901A26E0FFC39481
:10702E0002500B12A32A901A26E004F080EB12BA3B
:10703E006DEF24FF9209D20E200903027247E54438
:10704E007003027181E4901A29F0901A26F0901ABA
:10705E0026E0FFC39410400302718174882FF582DD
:10706E00E43400F583E0901A28F0F470030271788E
:10707E00E075F00BA42459F582E5F0343FF583E476
:10708E0093FB740193FA740293F9EA494B7003026D
:10709E007178E4901A27F0901A26E02498F582E48D
:1070AE003400F583E0FF901A27E0C39F400302717E
:1070BE0078AB1DAA1EA91F901A29E0FF75F01DA41A
:1070CE00F58285F08312072DFD7C00C004C0057D7E
:1070DE0000EF75F01DA429F9EA35F0FA90000D12B3
:1070EE000A6DD007D006120B22901A29E075F01DFA
:1070FE00A4AB1D251FF9E51E35F0FA90000D120AFE
:10710E006D157015701570A870A60308A60208A656
:10711E0001901A27E01570A870F6901A26E0FF5419
:10712E00071570A870F6EF131313541FFB7D04E0C0
:10713E0024B1F582E43400F583E0FF901A28E0755F
:10714E00F00BA42459F582E5F0343FF583740193D6
:10715E00FA740293F5828A83120B20901A29E004A6
:10716E00F0901A27E004F00270A5901A26E004F0C1
:10717E0002705CE4901A26F0901A26E0FFC3941079
:10718E00400302722C74882FF582E43400F583E0FC
:10719E00FFF4700302722375F00BEFA42459F582ED
:1071AE00E5F0343FF583E493FB740193FA74029394
:1071BE00F9EA494B605F157015701570A87076006E
:1071CE000876000876001570A870E4F6901A26E08E
:1071DE00FF54071570A870F6EF131313541FFB7DA1
:1071EE0001E0FE24B1F582E43400F583E0FF7488FB
:1071FE002EF582E43400F583E075F00BA42459F5E6
:10720E0082E5F0343FF583740193FA740293F582AC
:10721E008A83120B20901A26E004F0027186E49005
:10722E001A26F0901A26E0FFC3788296500B12B8F9
:10723E003D901A26E004F080EAE4FDFF12BADAE48B
:10724E00901A26F07B007A00799312BAB1EEC3132E
:10725E00FEEF13FFC374079FFFE49EFE901A26E015
:10726E00C39FE49E50117BFF7A80799412B8F09000
:10727E001A26E004F080CD7BFF7A80799612B8F062
:10728E007B007A00799312B8F07BFF7A80799A129C
:10729E00B8F07D01E4FF12BADA7BFF30090F7A8075
:1072AE00799F788DE6F54908E6F54A80047A80796B
:1072BE00B11256E97D02E4FF12BADA7BFF7A8079C9
:1072CE00C21256E97D03E4FF12BADA7549FF754A18
:0D72DE0082754BDC7BFF7A8079D10256E986
:07B18B00EF24FF920A7F018F
:10B19200E4F58420160FD216F58475D103F5BA753D
:0DB1A200BC9875E880C374079F5407F5BB87
:0DB1AF0075460275471300D547FCD546F6DE
:10B1BC00C2AFC2EDD2EC30EDFDD2AFAFBFEFFFAD01
:10B1CC00BEED901A44CFF0A3EFF0C3E094E8901AD0
:0CB1DC0044E0940350047F0180027F00D7
:01B1E8002244
:107889002009037F0122E4901A3DF012BB01C8ECE4
:10789900C8C9EDC9CAEECACBEFCB900000E0FCA382
:1078A900E0FDA3E0FEA3E0240AFFE43EFEE43DFD83
:1078B900E43CFCD31208D1501A12BB01900000E03D
:1078C900F8A3E0F9A3E0FAA3E0FBD31208D150032F
:1078D900027B3112BB019000001209DCE4901A3ED0
:1078E900F09000A8E0FE901A3EE0FFC39E4003021C
:1078F9007B407B017A1A793C12A9B4901A3CE0C406
:10790900540F640260617A007B647D017F0112AAD1
:10791900D820184B12BB5EE4FDFF12BADA7BFF7A5E
:107929008079D412B8F07D01E4FF12BADA901A3ED8
:10793900E0FFD39400400B7BFF7A8079E88F4912EE
:1079490056E97D02E4FF12BADA7BFF7A8079F8758D
:107959004902901A3CE0FFC4540FF54A1256E9D285
:1079690018901A3D7401F0901A3EE0FF75420175B6
:10797900431A75443F754503E4FB7D0112965D90FA
:107989001A3FE020E303027A137A007B647D017FCA
:107999000112AAD820174E12BB5EE4FDFF12BADA13
:1079A9007BFF7A8179111256E97D01E4FF12BADA77
:1079B9007BFF7A8179261256E97D02E4FF12BADA51
:1079C900901A3EE0FFD39400400B7BFF7A81793B0C
:1079D9008F491256E97D037F0F12BADA7BFF7A814C
:1079E900794E1256E9D2177F0312B192EF601590C2
:1079F9001A3EE0FF12B9C9C2177F0312B192EF70A4
:107A0900F812BB5E901A3D7401F012BB01E47B646D
:107A1900FAF9F8C31208D14003027B28901A3EE014
:107A2900FF75420175431A7544427545027B037D12
:107A39000212965D901A42E0C4F854F0C868FCA39B
:107A4900E0C4540F48FDE41203C2E4FBFA79C87894
:107A59004012019EE4FBFA798078451202A7E4FB03
:107A6900FA7990784012034460025003027B142093
:107A7900104912BB5E7A007B647D017F0112AAD88E
:107A8900E4FDFF12BADA7BFF7A8179541256E97D57
:107A990001E4FF12BADA7BFF7A8179691256E97D2E
:107AA90002E4FF12BADA901A3EE0FFD39400400BC9
:107AB9007BFF7A81797B8F491256E97D03E4FF12B6
:107AC900BADA901A42E0C4F854F0C868FCA3E0C4DA
:107AD900540F48FDE41203C2E4FBFA79C878401256
:107AE900019EE4FBFA798078451202A78F4C8E4BF0
:107AF9008D4A8C497BFF7A81798F1256E9D2109091
:107B090011477401F0901A3DF08014301011901A49
:107B19003EE0FF901147E06F7005C21012BB5E9006
:107B29001A3EE004F00278EA201706201003301804
:0C7B390006901A3D7401F0901A3DE0FF28
:017B4500221D
:1041020075840F75A4F575A5FF75A6FF75A70FE455
:10411200F584F5BA75BC9875E880F5D1F58475D14A
:1041220003F58475D48075840175D48012BB84E450
:10413200901A2EF0901A2CF0901A2BF075440F75ED
:104142004541901A28F0901A28E0FFC39402500EBD
:1041520012BA20EF6008901A28E004F080E8901A62
:1041620028E09000A8F0C214751D01751E00751F8D
:10417200C1E4901A26F0901A26E0FFC3941040037F
:104182000246D474B12FF582E43400F583E4F0746E
:10419200982FF582E43400F583E4F074882FF582D9
:1041A200E43400F58374FFF0EF131313541FFF90F0
:1041B2001A26E05407FD7B017A1A792712951C9082
:1041C2001A27E0D3940050030246CBE4A3F0901ADE
:1041D20028E075F00BA42451F582E5F0343FF58315
:1041E200E493FF6011901A27E0FEEF6E6008901AC8
:1041F20028E004F080D8901A27E06F60030245336C
:10420200901A26E02498F582E43400F583E4F090D5
:104212001A2AF0901A28E0FF75F00BA42458F582B0
:10422200E5F0343FF583E493FE901A2AE0FDC39E45
:10423200400302450475F00BEFA42455F582E5F026
:10424200343FF583E493FB740193FA740293F9ED1E
:1042520075F01DA4FFE92FF9EA35F0FA90000D126E
:104262000A6DCFE9CF901A2DEFF070030243EDE40F
:10427200901A29F0901A2DE0FF901A29E0C39F406E
:10428200030244FB901A28E075F00BA42455F58232
:10429200E5F0343FF583E493FB740193FA740293DF
:1042A200F9901A2AE075F01DA4FFE92FF9EA35F01A
:1042B200FAEAC0E0E9C0E0A3E075F01DA4251FF909
:1042C200E51E35F0C8E9C8FCAD1DD0E0F9D0E0FA32
:1042D2007E007F1D1206EE901A2BE075F01DA4AB36
:1042E2001D251FF9E51E35F0FAE92405F9E43AFA2D
:1042F2007D2512BA04EA494B603C901A26E0FFD3AE
:1043020094094005EF24378006901A26E02430FFF6
:10431200EFC0E0901A2BE075F01DA4AB1D251FF92C
:10432200E51E35F0FAE92405F9E43AFA7D2512BAD8
:1043320004D0E012075A901A2BE075F01DA4AB1DB1
:10434200251FF9E51E35F0FAE92405F9E43AFA7D6C
:104352002312BA04EA494B602D901A29E02430FF57
:10436200EFC0E0901A2BE075F01DA4AB1D251FF9DC
:10437200E51E35F0FAE92405F9E43AFA7D2312BA8A
:1043820004D0E012075AAA44A9457B01EBC0E0EA37
:10439200C0E0E9C0E0901A2BE075F01DA4AB1D252A
:1043A2001FF9E51E35F0FA90000D120A9DAB1DAA09
:1043B2001EA91F901A2BE075F01DA4F58285F083CB
:1043C20012072D2545F545E43544F544901A2BE0B6
:1043D20004F0901A26E02498F582E43400F583E094
:1043E20004F0901A29E004F0024276901A28E0754F
:1043F200F00BA42455F582E5F0343FF583E493FBFA
:10440200740193FA740293F9901A2AE075F01DA4CC
:10441200FFE92FF9EA35F0FAEAC0E0E9C0E0A3E0EB
:1044220075F01DA4251FF9E51E35F0C8E9C8FCADDD
:104432001DD0E0F9D0E0FA7E007F1D1206EE901A40
:104442002BE075F01DA4AB1D251FF9E51E35F0FA12
:10445200E92405F9E43AFA7D2512BA04EA494B60E7
:104462003C901A26E0FFD394094005EF24378006DA
:10447200901A26E02430FFEFC0E0901A2BE075F08E
:104482001DA4AB1D251FF9E51E35F0FAE92405F937
:10449200E43AFA7D2512BA04D0E012075AAA44A9D6
:1044A200457B01EBC0E0EAC0E0E9C0E0901A2BE0F6
:1044B20075F01DA4AB1D251FF9E51E35F0FA90001D
:1044C2000D120A9DAB1DAA1EA91F901A2BE075F0B2
:1044D2001DA4F58285F08312072D2545F545E435A7
:1044E20044F544901A2BE004F0901A26E02498F543
:1044F20082E43400F583E004F0901A2AE004F0022A
:104502004215901A27E0FF901A26E0FE24B1F582A8
:10451200E43400F583EFF0901A28E0FF74882EF55A
:1045220082E43400F583EFF0901A2CE004F00246A6
:10453200CBE4901A28F09000A8E0FE901A28E0FF41
:10454200C39E500DE4FD12B91A901A28E004F080BF
:10455200E512BB5EE4FDFF12BADA7BFF7A81799F36
:10456200901A26E0F5491256E97D01E4FF12BADA03
:104572007BFF7A8179B61256E9E4901A28F07D021F
:10458200E4FF12BADA901A28E0FF75F00BA4245166
:10459200F582E5F0343FF583E493F54975F00BEFCE
:1045A200A42452F582E5F0343FF583E493FB7401D1
:1045B20093FA7402938B4A8A4BF54C7BFF7A81798A
:1045C200C41256E97D03E4FF12BADA901A28E070A9
:1045D200087BFF7A8179DA8022901A28E075F00B45
:1045E200A4245CF582E5F0343FF583E4937BFF700D
:1045F200067A8179EF80047A8279041256E97F0083
:1046020012B899E4FF12B19212B18BEF24FF920B10
:104612007F0212B192EF24FF920C7F0312B192EF4C
:1046220024FF920D200A09200B06200C03300DCE28
:10463200300A44901A28E075F00BA42451F582E563
:10464200F0343FF583E493FB901A26E0FE13131334
:10465200541FFFEE5407FD1282FA901A26E014F05E
:10466200300A0CE4FF12B192EF24FF920A80F1901B
:104672001A2E7401F08052300C1B901A28E0D39449
:10468200004003E014F0300C0C7F0212B192EF24D0
:10469200FF920C80F1200D03024580901A28E075EC
:1046A200F00BA4245CF582E5F0343FF583E49360DB
:1046B20006901A28E004F0200D030245807F0312C1
:1046C200B192EF24FF920D80EE901A26E004F002E0
:1046D2004178AB1DAA1EA91F901A2BE075F01DA4EC
:1046E200F58285F083E412076C901A2EE06006E4EE
:0546F200F58475EF10D6
:0146F70022A0
:10B83D001570A870EFF6A870E6FF131313541F24AC
:10B84D0008F582E43400F583E0FEEF5407FF740140
:0FB85D00C8EFC8088002C333D8FC4EF005702234
:05BB8B008F397F00224C
:10BAC600120714901148F0AB3CAA3DA93E7401122E
:04BAD600075AFF22EA
:105AF60030190C12BB5EE4900004F0A374FFF02092
:105B060009037F0022300F03025B9DE4FDFF12BAFA
:105B1600DAE4901A3CF07B007A00799312BAB1EE7F
:105B2600C313FEEF13FFC374079FFFE49EFE901A94
:105B36003CE0C39FE49E50117BFF7A80799412B8B3
:105B4600F0901A3CE004F080CD7BFF7A80799612C3
:105B5600B8F07B007A00799312B8F07BFF7A8079EF
:105B66009A12B8F07D01E4FF12BADA7BFF7A8079E7
:105B76009F788DE6F54908E6F54A1256E97D027FDB
:105B86000112BADA12B4E97D03E4FF12BADA7BFF36
:105B96007A82791912B8F0200F03025EBB900005D5
:105BA600E0FF900004E06F7003025CF9C208E49025
:105BB6001A3DF0901A3CF0901A3FF0901A3CE0FF24
:105BC600C394104003025C9F74B12FF582E4340045
:105BD600F583E07003025C96901A3DE004F09000B5
:105BE60004E0FF901A3DE0D39F5003025C96901AA2
:105BF6003FE0FDE4FF12BADAE4901A3EF0901A3E56
:105C0600E075F00BA42451F582E5F0343FF583E40A
:105C160093FF601B901A3CE024B1F582E43400F552
:105C260083E0FEEF6E6008901A3EE004F080CE90AE
:105C36001A3EE0FF75F00BA42451F582E5F0343FDF
:105C4600F583E493FE603A901A3FE0B40304D20869
:105C56008047901A3CE0F5498E4A75F00BEFA42474
:105C660052F582E5F0343FF583E493FB740193FA31
:105C76007402938B4B8A4CF54D7BFF7A82792E808A
:105C8600067BFF7A8279461256E9901A3FE004F0C5
:105C9600901A3CE004F0025BC17D03E4FF12BADA1D
:105CA6007BFF7A82795B12B8F07D037F1012BADA35
:105CB6007BFF30080C7A8279657549131256E980A4
:105CC600077A82796B12B8F07D037F0A12BADA90EE
:105CD6000004E0D394007BFF400C7A827965754915
:105CE600121256E980077A82796B12B8F090000496
:105CF600E0A3F030080C300D09201506900004E0F2
:105D060004F0900004E0D394004009300C06201300
:105D160003E014F0300A0C201109C20FA20A9211F6
:105D260012BB5E300B03025EBB201203025EBBE4B5
:105D3600900006F0901A3CF0900006E0FE13131354
:105D4600541FFFEE5407FD12BA3BEF6006901A3C53
:105D5600E004F0900006E004F0E0C3941040D9E4BB
:105D6600900006F0900006E0FE131313541FFFEE9A
:105D76005407FD12BA3BEF700C900006E004F0E009
:105D8600C3941040DF901A3CE07002FF2212BB5E03
:105D96007D03E4FF12BADA901A3CE07BFF70067AC4
:105DA60082797080047A8279851256E9E4FDFF12C1
:105DB600BADA7BFF7A82799A1256E97D01E4FF12FC
:105DC600BADA7BFF7A8279AF900006E0F54912567F
:105DD600E97F0012B899E4FF12B19212B18BEF2459
:105DE600FF920B7F0212B192EF24FF920C7F0312F7
:105DF600B192EF24FF920D200A09200B06200C0316
:105E0600300DCE300A1F300A0CE4FF12B192EF2497
:105E1600FF920A80F112BB5E90000574FFF0C21279
:105E2600C2117F0022300B23900006E0FD7BFFE4C9
:105E3600FF1282FA300B0C7F0112B192EF24FF920F
:105E46000B80F1E4F58475EF10806A300C2E801219
:105E5600900006E0131313541FFF7D1012BA3BEF98
:105E6600700B900006E0240F540FF080E3300C0C0A
:105E76007F0212B192EF24FF920C80F1200D0302F3
:105E86005DB28015900006E0FE131313541FFFEE5B
:105E96005407FD12BA3BEF700A900006E004540F57
:105EA600F080E1200D03025DB27F0312B192EF2470
:105EB600FF920D80EE200F0D200B0A301207A20B69
:105EC60092127F0122200F0D200C0A301307A20C1C
:105ED60092137F0222300A0F20110CD20F12BB5EE2
:105EE600900004E004A3F0A20A9211A20B9212A25F
:095EF6000C9213A20D92157F001D
:015EFF002280
:105F00002009030261FEE4901A26F0901A26E0FFB1
:105F1000131313541F2408F582E43400F583E0FDC5
:105F20007C00EF5407FF74017E00C8EFC8088005AD
:105F3000C333CE33CED8F9FFEE5CFEEF5D4E700377
:105F400002608CE4901A27F0901A2AF0901A2AE046
:105F5000FFC39410400302605C74982FF582E43410
:105F600000F583E0FF901A27E0FD2FFFE433FE9059
:105F70001A26E0FCFBD3EF9B7480F86E9850030266
:105F8000603EEC9DA3F0901A2AE02488F582E43468
:105F900000F583E0901A28F0F4700302605CE0756D
:105FA000F00BA42459F582E5F0343FF583E493FB2C
:105FB000740193FA740293F9EA494B700302605C2E
:105FC000901A26E075F01DA4AB1D251FF9E51E35BE
:105FD000F0FA90000D120A6D157015701570A8700A
:105FE000C6EBC608C6EAC608C6E9C6901A27E01579
:105FF00070A870F6901A2AE0FF54071570A870F682
:10600000EF131313541FFB7D02901A28E0FE75F066
:106010000BA42451F582E5F0343FF583E493FF753A
:10602000F00BEEA42459F582E5F0343FF5837401BA
:1060300093FA740293F5828A83120B20801E901AC1
:106040002AE02498F582E43400F583E0FF901A27D3
:10605000E02FF0901A2AE004F0025F4C901A26E03C
:10606000FF131313541F2408F582E43400F583C092
:1060700083C082E0FEEF5407FF7401C8EFC80880B8
:1060800002C333D8FCF45ED082D083F0901A26E0AD
:1060900004F0E0C394805003025F0B901141E024B0
:1060A00088F582E43400F583E0FFF470030261BBFD
:1060B000901A27EFF0E4A3F0901141E02498F582C4
:1060C000E43400F583E0FF901A28E0FEC39F40030C
:1060D0000261BB901A27E075F00BA42459F582E504
:1060E000F0343FF583E493FB740193FA740293F95F
:1060F000EA494B6065157015701570A87076010837
:10610000761A08762B1570A870EEF6901141E0FF14
:1061100054071570A870F6EF131313541FFB7D037B
:10612000901A27E0FE75F00BA42451F582E5F034B7
:106130003FF583E493FF75F00BEEA42459F582E557
:10614000F0343FF583740193FA740293F5828A83E5
:10615000120B20901A29EFF08005E4901A29F09094
:106160001A29E0FFD394004049C2AF7E00EEC0E0A0
:10617000EFC0E0901A28E0FF901146E02FFFE433D3
:10618000FE7C007D1D12078EAB1DE51F2FF9E51E5D
:106190003EFA90000D120A6DC8E9C8CCEACCCDEBEE
:1061A000CD7B017A1A792BD0E0FFD0E0FE1206EE0B
:1061B000D2AF901A28E004F00260B8901141E024B8
:1061C00098F582E43400F583E0FF901146E02FF06B
:1061D000901141E004F0E0B41006E4F0901146F0B4
:1061E000901148E0F46017E0FE131313541FFFEE04
:1061F0005407FD7BFF1282FA90114874FFF012BB26
:1062000001C8ECC8C9EDC9CAEECACBEFCB901142A8
:10621000E0FCA3E0FDA3E0FEA3E0240AFFE43EFED1
:10622000E43DFDE43CFCD31208D1501712BB0190B1
:106230001142E0F8A3E0F9A3E0FAA3E0FBD31208CF
:10624000D1406F12BB019011421209DCE4FF12B180
:106250009212B18BEF24FF920B7F0212B192EF24C6
:10626000FF920C7F0312B192EF24FF920D300905CB
:10627000120BF4803D12BB01E47B2C7A01F9F8C3C8
:106280001208D1502D300E05C20E12BB5E7D017F6B
:106290000512BADA7BFF7A8279C41256E97D027F51
:1062A0000512BADA12BA548F497BFF7A8279CF127B
:1062B00056E930143112BB01E47B0AFAF9F8C31233
:1062C00008D15022C214E4901A27F09000A8E0FEF2
:1062D000901A27E0FFC39E500DE4FD12B91A901AE0
:0662E00027E004F080E558
:0162E6002295
:103A5B004C45442D4465627567004C45442D5075AB
:103A6B006C7365720044696E203556004F70744953
:103A7B006E0043504C4400446F75742035562F3202
:103A8B0034560052656C616973004F70744F7574D6
:103A9B000055696E20302D322E35560055696E203B
:103AAB002B2D3130560049696E20302D322E356D5D
:103ABB00410049696E20302D32356D410055696EDC
:103ACB0020302D322E3556204673740055696E20EA
:103ADB002B2D31305620466173740049696E2030AE
:103AEB002D322E356D41204673740049696E20309E
:103AFB002D32356D41204673740055696E202B2D88
:103B0B0031305620446966660055696E202B2D3185
:103B1B00305620466C740043696E20302D31306E68
:103B2B00460043696E20302D3175460050543130BC
:103B3B00302D38005054313030302D380041443561
:103B4B0039300050543130302D3200505431303038
:103B5B00302D32004345524E4F582D3200554F7584
:103B6B007420302D322E355600554F7574202B2D69
:103B7B0031305600494F757420302D322E356D4142
:103B8B0000494F757420302D32356D41004C6971F1
:103B9B002E4865206C6576656C00554F7574203228
:103BAB0030305600554F7574203330305600554F1A
:103BBB007574203130562F3235306D4100245265EB
:103BCB00762400013400000050254F75740000006E
:103BDB000100010000000000437F00003F80000057
:103BEB000418000001502555696E230000010008E0
:103BFB00040000000000000000000000000418009A
:103C0B000001502555696E230000010004040000DB
:103C1B00000000000000000000000418000001502C
:103C2B002555696E2300000100020400000000000E
:103C3B000000000000000004180000015025556929
:103C4B006E230000010008040000000000000000CB
:103C5B00000000000134000008502552616E6765BA
:103C6B000001000000000000000000000000000048
:103C7B000004180000015025556F757423000100D6
:103C8B00080200000000402000003DCCCCCD041801
:103C9B000000015025556F7574230001000802C107
:103CAB00200000412000003F0000000406FD000141
:103CBB00502549696E230000010008040000000034
:103CCB000000000000000000041DF7000150254318
:103CDB00696E2300000100040400000000000000D6
:103CEB0000000000000408000001502554230000D0
:103CFB0000000100080200000000000000000000AE
:103D0B0000000406FD000950254578636974000125
:103D1B000000010000000000000000000000000493
:103D2B000800000150255423000000000100080288
:103D3B00000000000000000000000000040800006C
:103D4B000150255423000000000100020200000076
:103D5B0000000000000000000004070000015025D7
:103D6B0054230000000001000202000000000000CC
:103D7B000000000000000406FD00015025496F758E
:103D8B00742300010008020000000041A000003D68
:103D9B00CCCCCD04180000015025556F7574230051
:103DAB0001000102C1200000412000003DCCCCCD20
:103DBB000406FD0009502545786369740001000075
:103DCB00010000000042C800003F800000045A00C0
:103DDB00000950254C4F66730000010000020000E3
:103DEB0000000000000000000000045D000009500E
:103DFB00254C4761696E00010000020000000000C5
:103E0B000000000000000002030000085025546F62
:103E1B0066660000010000000000000000000000CA
:103E2B000000000002030000085025546F6E0000D4
:103E3B000001000000000000000000000000000076
:103E4B0000045A00000150254C696E00000001006F
:103E5B000001000000000000000000000000013223
:103E6B00000000502544696E23000001000801008A
:103E7B000000000000000000000000013200000004
:103E8B00502544696E23000001000401000000006E
:103E9B00000000000000000001320000005025442B
:103EAB006F7574230001000801000000003F8000C3
:103EBB00003F8000000132000000502552656C234A
:103ECB00000001000401000000003F8000003F8063
:103EDB000000013200000050254F757423000001D3
:103EEB00000401000000003F8000003F8000000440
:103EFB001800000150255544230000000100080361
:103F0B0000000000434800003F8000000418000040
:103F1B00015025552300000000010008030000009C
:103F2B000000000000000000000406FA000150250C
:103F3B0049230000000001000803000000000000FE
:103F4B0000000000000001FF3A5BFF3BCE01FFB118
:103F5B00E902FF3A650000000100000020FF3A7003
:103F6B00FF3E6901FF9AFC21FF3A77FF3E8601FF76
:103F7B009AFC22FF3A7DFF3E6901FF9AFC40FF3A13
:103F8B0082FF3EA301FF8E4241FF3A8EFF3EC001EE
:103F9B00FF8E4242FF3A95FF3EDD01FF8E4260FFEE
:103FAB003A9CFF3BEB01FF62E761FF3AA7FF3BEB5C
:103FBB0001FF62E762FF3AB1FF3CB601FF62E763C4
:103FCB00FF3ABDFF3CB601FF62E764FF3AC8FF3B17
:103FDB00EB01FF669265FF3AD7FF3BEB01FF669261
:103FEB0066FF3AE6FF3CB601FF669267FF3AF6FFC3
:103FFB003CB601FF669268FF3B05FF3C0801FF6280
:10400B00E769FF3B14FF3C2501FF7DF270FF3B226C
:10401B00FF3CD301FF7B4671FF3B2DFF3CD301FFE0
:10402B007B4672FF3B37FF3CF002FF51CA73FF3BED
:10403B003FFF3CF002FF51CA74FF3B48FF3D2A0192
:10404B00FF6D1E75FF3B4EFF3D4701FF46F876FFA8
:10405B003B56FF3D4701FF46F877FF3B5FFF3D6453
:10406B0001FF46F880FF3B68FF3C7C01FF878081A6
:10407B00FF3B74FF3C9901FF4C6982FF3B7FFF3D87
:10408B008101FF878083FF3B8CFF3D8101FF878090
:10409B0084FF3B98FF3DBB06FF16BF85FF3BA5FF8B
:1040AB003EFA03FF296586FF3BAFFF3EFA03FF296C
:1040BB006587FF3BB9FF3D9E01FF87800000000035
:1040CB00000000000000003CA3D70A3D23D70A3DA7
:1040DB00A3D70A3E23D70A3EA3D70A3F23D70A3FCB
:1040EB00A3D70A4023D70A050403020100060706DB
:0740FB0002070300040501A8
:06B6930004150000000098
:108CC500E5702412F8E6FFE5702413F8E6FD755308
:038CD500017B061A
:108CD800D2B1C2B0C2B2E4901A46F0901A46E0FE91
:108CE800C39404504CEFC8EEC8088002C333D8FCC4
:108CF8005408D394004003D38001C392B30000000A
:108D0800000000000000000000000000000000005B
:108D180000D2B000000000000000000000000000C9
:108D280000000000000000C2B0901A46E004F08085
:108D3800AAE4901A46F0901A46E0FFC39403504CF8
:108D4800EDC8EFC8088002C333D8FC5404D394009C
:108D58004003D38001C392B300000000000000006C
:108D6800000000000000000000000000D2B0000079
:108D780000000000000000000000000000000000EB
:108D88000000C2B0901A46E004F080AAE4901A46A7
:108D9800F0901A46E0FFC39404504CEBC8EFC808A3
:108DA8008002C333D8FC5408D394004003D3800115
:108DB800C392B300000000000000000000000000A3
:108DC80000000000000000D2B00000000000000019
:108DD80000000000000000000000000000C2B09089
:108DE8001A46E004F080AAD2B20000000000000099
:108DF80000000000000000000000000000D2B000E9
:108E0800000000000000000000000000000000005A
:108E1800000000C2B0C2B2C2B3E55324FF92B0D280
:108E2800B2C2B10000000000000000000000000015
:098E380000000000000000C2B2BD
:018E4100220E
:10BA8500E5702409F8E6FFE570240AF8E6FD7B0673
:06BA9500E4F553028CD819
:05ABF900F8E6FD7BFF02
:03ABFE00CCEBCCD1
:10AC01007B0312BA95E4901A40F0EC5480D394007F
:10AC11004003D38001C392B3000000000000000094
:10AC2100000000000000000000000000D2B00000A1
:10AC31000000000000000000000000000000000013
:10AC41000000C2B0EC25E0FC901A40E004F0E0B452
:10AC510008B8C2B3D2B2000000000000000000003A
:10AC610000000000000000000000D2B00000000061
:10AC710000000000000000000000000000000000D3
:04AC8100C2B0C2B2E9
:01AC850022AC
:10A5FE00E5702405F8EFF6E5702412F8E6FFE57035
:0CA60E002413F8E6FDE5702405F8E6FBD7
:03A61A00CCEBCCBA
:10A61D007B0212BA95E4901A40F0EC5480D394006A
:10A62D004003D38001C392B300000000000000007E
:10A63D00000000000000000000000000D2B000008B
:10A64D0000000000000000000000000000000000FD
:10A65D000000C2B0EC25E0FC901A40E004F0E0B43C
:10A66D0008B8C2B3D2B20000000000000000000024
:10A67D0000000000000000000000D2B0000000004B
:10A68D0000000000000000000000000000000000BD
:04A69D00C2B0C2B2D3
:01A6A1002296
:0CA74500F8E6FD7B00E5702408F97A00BE
:06A751008B468A4789488F
:10A75700E4FB12BA95D2B20000000000000000002E
:10A767000000000000000000000000D2B000000060
:10A7770000000000000000000000000000000000D2
:10A7870000C2B0C2B2E4901A40F00000000000001E
:10A797000000000000000000000000000000D2B030
:10A7A70000000000000000000000000000000000A2
:10A7B70000000000C2B0901A41E025E0FFA2B4E417
:10A7C700334FF0901A40E004F0E0B408BD901A410E
:0AA7D700E0AB46AA47A94802075A62
:06AB69008B468A47894873
:10AB6F007B0112BA95D2B200000000000000000075
:10AB7F000000000000000000000000D2B000000044
:10AB8F0000000000000000000000000000000000B6
:10AB9F0000C2B0C2B2E4901A40F000000000000002
:10ABAF000000000000000000000000000000D2B014
:10ABBF000000000000000000000000000000000086
:10ABCF0000000000C2B0901A41E025E0FFA2B4E4FB
:10ABDF00334FF0901A40E004F0E0B408BD901A41F2
:0AABEF00E0AB46AA47A94802075A46
:03AD9E00CCEDCC2D
:10ADA1007B05E4FD12BA95E4901A30F0EC5480D39F
:10ADB10094004003D38001C392B30000000000005F
:10ADC1000000000000000000000000000000D2B000
:10ADD1000000000000000000000000000000000072
:10ADE10000000000C2B0EC25E0FC901A30E004F055
:10ADF100E0B408B8C2B3D2B2000000000000000005
:10AE0100000000000000000000000000D2B00000BF
:10AE11000000000000000000000000000000000031
:06AE21000000C2B0C2B245
:01AE27002208
:06A9B4008B488A49894A24
:10A9BA007B04E4FD12BA95D2B20000000000000048
:10A9CA0000000000000000000000000000D2B000FB
:10A9DA00000000000000000000000000000000006D
:10A9EA00000000C2B0C2B2E4901A44F000000000B5
:10A9FA00000000000000000000000000000000004D
:10AA0A00D2B00000000000000000000000000000BA
:10AA1A00000000000000C2B0901A45E025E0FFA245
:10AA2A00B4E4334FF0901A44E004F0E0B408BD9067
:0CAA3A001A45E0AB48AA49A94A02075A95
:10BA3B007B017A1A794012951C901A40E0D394003E
:08BA4B0040047F0180027F002E
:01BA530022D0
:06951C008B468A478948D6
:109522007B0712BA95D2B3000000000000000000D1
:109532000000000000000000000000D2B0000000A7
:109542000000000000000000000000000000000019
:1095520000C2B0D2B3000000000000000000000012
:10956200000000000000000000D2B0000000000077
:10957200000000000000000000000000000000C227
:10958200B0C2B300000000000000000000000000B4
:1095920000000000000000D2B00000000000000047
:1095A20000000000000000000000000000C2B0E463
:1095B200901A41F0C2B30000000000000000000059
:1095C20000000000000000000000D2B00000000017
:1095D2000000000000000000000000000000000089
:1095E200C2B0901A41E004F0E0B406C830B409AB4E
:1095F20046AA47A948E4805FE4901A41F0000000BF
:109602000000000000000000000000000000000058
:1096120000D2B000000000000000000000000000C6
:1096220000000000000000C2B0901A43E025E0FFF5
:10963200901A42E033FEA2B4E433FDEF4DFFEEF0A8
:10964200A3EFF0901A41E004F0E0B410B0901A4297
:0A965200E0AB46AA47A94812075AE8
:01965C0022EB
:10B73400901A51EFF0A3EDF0A3EBF012BA3BEF70C7
:10B7440002FF22901A51E0FFA3E0FD7B017A1A79EF
:10B754005012951C901A53E0FF901A50E06F700439
:06B764007F0180027F005E
:01B76A0022BC
:0382FA00CCEBCCFE
:1082FD007B0712BA95D2B300000000000000000009
:10830D000000000000000000000000D2B0000000DE
:10831D000000000000000000000000000000000050
:10832D0000C2B0C2B3000000000000000000000059
:10833D00000000000000000000D2B00000000000AE
:10834D00000000000000000000000000000000C25E
:10835D00B0C2B300000000000000000000000000EB
:10836D0000000000000000D2B0000000000000007E
:10837D0000000000000000000000000000C2B0E49A
:10838D00901A40F0D2B30000000000000000000081
:10839D0000000000000000000000D2B0000000004E
:1083AD0000000000000000000000000000000000C0
:1083BD00C2B0901A40E004F0E0B406C8D2B200009A
:1083CD0000000000000000000000000000000000A0
:1083DD000000C2B2D2B30000000000000000000097
:1083ED0000000000000000000000D2B000000000FE
:1083FD000000000000000000000000000000000070
:10840D00C2B0C2B300000000000000000000000078
:10841D000000000000000000D2B0000000000000CD
:10842D000000000000000000000000000000C2B0CD
:10843D00D2B30000000000000000000000000000AA
:10844D00000000000000D2B000000000000000009D
:10845D00000000000000000000000000C2B0E49029
:10846D001A40F0C2B3000000000000000000000040
:10847D00000000000000000000D2B000000000006D
:10848D00000000000000000000000000000000C21D
:10849D00B0901A40E004F0E0B406C8E4901A40F041
:1084AD00EC5480D394004003D38001C392B30000F9
:1084BD0000000000000000000000000000000000AF
:1084CD000000D2B00000000000000000000000001D
:1084DD000000000000000000C2B0EC25E0FC901A86
:1084ED0040E004F0E0B410B8D2B20000000000008B
:1084FD000000000000000000000000000000C2B2FB
:0A850D00E4901A41F0A3F020B42717
:0D85170075460175470300D547FCD546F6B3
:10852400901A42E004F07006901A41E004F0901AA8
:0A85340041E0B427DBA3E0B410D649
:01853E00221A
:108E42001570A870EBF61570A870EDF61570A87085
:048E5200EFF61570B2
:108E5600A8700808E664016003028EE4E570240445
:108E6600F8E6FEE5702403F8E6FF75F008A42EF593
:108E760082E435F0F583E5822449F582E5833411F1
:108E8600F583E4F0F584E5EF20E119E5702404F8B4
:108E9600E6FDEF75F008A42D2449F9E43411FA7BB8
:108EA6000112AB69E5702403F8E6FFE5702404F8C7
:108EB600E6FD75F008EFA42DF582E435F0F583E5BF
:108EC600822449F582E5833411F583E0FB12A61A64
:108ED600E5702403F8E6FFE570240412ABF9A870E8
:108EE6000808E664026003028FADE5702406F8CB3D
:108EF600E6CB08E6FA08E6F9120714A870F6603E13
:108F0600E5702404F8E6FFE5702403F8E675F0083A
:108F1600A42FF582E435F0F583E5822449F582E550
:108F2600833411F583E0FFE5702405F8E6FE74014D
:108F3600C8EEC8088002C333D8FC4FF0803DE57008
:108F46002404F8E6FFE5702403F8E675F008A42F7C
:108F5600F582E435F0F583E5822449F582E583342C
:108F660011F583E0FFE5702405F8E6FE7401C8EE0E
:108F7600C8088002C333D8FCF45FF0E5702403F818
:108F8600E6FFE5702404F8E6FD75F008EFA42DF57C
:108F960082E435F0F583E5822449F582E5833411D0
:098FA600F583E0FB12A61A7F001E
:078FAF00E5702409F57022B2
:109AFC001570A870EBF61570A870EDF61570A870BF
:049B0C00EFF61570EB
:109B1000A8700808E664036003029C03E57024064D
:109B2000F8CBE6CB08E6FA08E6F9120714603EE542
:109B3000702404F8E6FFE5702403F8E675F008A445
:109B40002FF582E435F0F583E5822449F582E5833B
:109B50003411F583E0FFE5702405F8E6FE7401C8D2
:109B6000EEC8088002C333D8FC4FF0803DE5702476
:109B700004F8E6FFE5702403F8E675F008A42FF575
:109B800082E435F0F583E5822449F582E5833411DA
:109B9000F583E0FFE5702405F8E6FE7401C8EEC821
:109BA000088002C333D8FCF45FF0E5702403F8E6C4
:109BB000FFE5702404F8E6FD7B00A9707A0012A787
:109BC00051E5702405F974017E00C8E7C8088005D6
:109BD000C333CE33CED8F9FFA870E6FDEF5DD39442
:109BE000007480948040047F0180027F00E570242F
:109BF00006F8CBE6CB08E6FA08E6F9EF12075A7F3B
:059C00000180027F005D
:079C0500E5702409F570224F
:10B1E9001570A870EBF61570A870EDF61570A870BB
:10B1F900EFF6A87008E6B4010DA8700808E6FFE5A7
:10B2090070240312ABF9A87008E6B40222A87008EA
:10B2190008E6FFE5702403F8E6FDE5702405F8CBA0
:10B22900E6CB08E6FA08E6F9120714FB12A61A7F1C
:08B2390000E5702408F5702205
:108780001570A870EBF61570A870EDF61570A8704E
:08879000EFF6E57024F9F57025
:108798002408F8E664026003028987E570240CF86F
:1087A800CBE6CB08E6FA08E6F91208F5A870120934
:1087B800D0E5702407F8E6B40209E4FBFA79C87832
:1087C800428022E5702407F8E6B48209E4FBFA79CE
:1087D8002078408010E5702407F8E6B4832FE4FB86
:1087E800FA79C87841E8C0E0A87012095FD0E0F8CB
:1087F8001202A77B007AFF797F784712019E120345
:10880800FBE5702404F8EEF608EFF68046E57024E0
:1088180007F8E6B4873DE4FBFA79A07841E8C0E0C0
:10882800A87012095FD0E0F81202A7E4FBFAF97801
:108838003F1200AD7B007AFF797F784712019E12C4
:1088480003FBE5702404F8EEF608EFF6E570240B58
:10885800F8760112BA85E5702406F8E4F6E5702486
:1088680006F8E6FFC39404503FEF94014003D38019
:1088780001C392B3000000000000000000000000E7
:108888000000000000000000D2B00000000000005E
:108898000000000000000000000000000000C2B05E
:1088A800E5702406F80680B5E5702406F8E4F6E5D8
:1088B800702406F8E6C394045051E570240BF8E6DA
:1088C800FF5408D394004003D38001C392B300003F
:1088D8000000000000000000000000000000000090
:1088E8000000D2B0000000000000000000000000FE
:1088F8000000000000000000C2B0E570240BF8EF93
:1089080025E0F6E5702406F80680A4E5702406F84C
:10891800E4F6E5702406F8E6C394105060E5702488
:1089280004F8E6FE08E6FFEE5480FCD3E49400EC7D
:1089380094004003D38001C392B3000000000000FC
:108948000000000000000000000000000000D2B09D
:10895800000000000000000000000000000000000F
:1089680000000000C2B0E5702404F8EF25E0FFEE37
:1089780033F608EFF6E5702406F8068095D2B17F45
:0189880000EE
:07898900E570240FF57022D8
:104C69001570A870EBF61570A870EDF61570A870A0
:084C7900EFF6E57024F9F57077
:104C8100E5702408F8E6640260030251C1E570246E
:104C91000CF8CBE6CB08E6FA08E6F91208F5A8709D
:104CA1001209D0E4FFFE7D207C41A8701209771221
:104CB1000344600B4009A8701209E841200000E498
:104CC100FFFE7D207CC1A8701209771203445009B0
:104CD100A8701209E8C1200000E4FFFE7D207C419C
:104CE100A8701209771200ADE4FBFA79A07841129D
:104CF10002A77B007AFF797F784712019EE4FBFAD5
:104D0100F9783F1200AD1203FBE5702404F8EEF6CA
:104D110008EFF612BA85C2B30000000000000000DF
:104D2100000000000000000000000000D2B0000000
:104D31000000000000000000000000000000000072
:104D41000000C2B0C2B3000000000000000000007B
:104D510000000000000000000000D2B000000000D0
:104D61000000000000000000000000000000000042
:104D7100C2B0E570240BF8E6FFC394045049E57016
:104D81002406F8E4F6E5702406F8E6C39416400319
:104D9100024F6B0000000000000000000000000056
:104DA10000000000000000D2B00000000000000080
:104DB10000000000000000000000000000C2B0E59B
:104DC100702406F80680BEC2B30000000000000097
:104DD10000000000000000000000000000D2B00050
:104DE10000000000000000000000000000000000C2
:104DF100000000C2B0D2B3000000000000000000BB
:104E01000000000000000000000000D2B00000001F
:104E11000000000000000000000000000000000091
:104E210000C2B0C2B300000000000000000000009A
:104E3100000000000000000000D2B00000000000EF
:104E4100000000000000000000000000000000C29F
:104E5100B0C2B3000000000000000000000000002C
:104E610000000000000000D2B000000000000000BF
:104E710000000000000000000000000000C2B0EFD0
:104E81005402D394004003D38001C392B3000000C5
:104E91000000000000000000000000000000000011
:104EA10000D2B0000000000000000000000000007F
:104EB10000000000000000C2B0E570240BF8E654C9
:104EC10001D394004003D38001C392B300000000DA
:104ED10000000000000000000000000000000000D1
:104EE100D2B000000000000000000000000000003F
:104EF100000000000000C2B0E5702406F8E4F6E509
:104F0100702406F8E6C394105060E5702404F8E6B6
:104F1100FE08E6FFEE5480FCD3E49400EC940040DC
:104F210003D38001C392B300000000000000000021
:104F31000000000000000000000000D2B0000000EE
:104F41000000000000000000000000000000000060
:104F510000C2B0E5702404F8EF25E0FFEE33F60857
:104F6100EFF6E5702406F8068095C2B30000000054
:104F71000000000000000000000000000000000030
:104F8100D2B000000000000000000000000000009E
:104F9100000000000000C2B0C2B300000000000029
:104FA1000000000000000000000000000000D2B07E
:104FB10000000000000000000000000000000000F0
:104FC10000000000C2B0E570240BF8E6FFD39403A3
:104FD1004049E5702406F8E4F6E5702406F8E6C3D6
:104FE100941640030251BF000000000000000000C1
:104FF1000000000000000000000000D2B00000002E
:10500100000000000000000000000000000000009F
:1050110000C2B0E5702406F80680BEC2B3000000ED
:10502100000000000000000000000000000000007F
:1050310000D2B000000000000000000000000000ED
:1050410000000000000000C2B0D2B3000000000068
:10505100000000000000000000000000000000D27D
:10506100B00000000000000000000000000000008F
:105071000000000000C2B0C2B30000000000000048
:1050810000000000000000000000000000D2B0009D
:10509100000000000000000000000000000000000F
:1050A100000000C2B0C2B300000000000000000018
:1050B1000000000000000000000000D2B00000006D
:1050C10000000000000000000000000000000000DF
:1050D10000C2B0EF5402D394004003D38001C392C5
:1050E100B30000000000000000000000000000000C
:1050F1000000000000D2B00000000000000000002D
:105101000000000000000000000000C2B0E57024B3
:105111000BF8E65401D394004003D38001C392B34A
:10512100000000000000000000000000000000007E
:1051310000000000D2B000000000000000000000EC
:1051410000000000000000000000C2B0E57024066D
:10515100F8E4F6E5702406F8E6C394105060E570B3
:105161002404F8E6FE08E6FFEE5480FCD3E4940044
:10517100EC94004003D38001C392B300000000000F
:10518100000000000000000000000000000000D24C
:10519100B00000000000000000000000000000005E
:1051A1000000000000C2B0E5702404F8EF25E0FF24
:1051B100EE33F608EFF6E5702406F8068095D2B1D5
:0251C1007F006D
:0751C300E570240FF57022D6
:0B911C007D527F031291277D037F012D
:109127001570A870EDF61570A870EFF6157015702C
:10913700C2B3C2B100000000000000000000000040
:109147000000000000000000A870E4F6A870E6C365
:1091570094045031C2B0C2B3000000000000000008
:10916700000000000000000000000000D2B0000076
:1091770000000000000000000000000000000000E8
:1091870000000680C7A870E4F6A870087608A870E3
:10919700E6C39404504AC2B008E6FFA87008085610
:1091A70094004003D38001C392B300000000000085
:1091B7000000000000000000000000000000D2B026
:1091C7000000000000000000000000000000000098
:1091D70000000000A87008EFC313F6A8700680AE61
:1091E700D2B20000000000000000000000000000F4
:1091F700000000000000C2B2A870E4F6A87008766C
:1092070080A870E6C39408504DC2B008E6FFE57029
:109217002403F8E65FD394004003D38001C392B3DD
:109227000000000000000000000000000000000037
:1092370000000000D2B000000000000000000000A5
:1092470000000000000000000000A87008EFC31332
:10925700F6A8700680ABD2B1C2B3000000000000D0
:0E9267000000000000000000000000000000F9
:07927500E5702404F57022EE
:0AA7E1001570A870EFF615701570E2
:10A7EB00C2B3C2B100000000000000000000000076
:10A7FB000000000000000000A870E4F6A8700876C6
:10A80B0080A870E6C39408504AC2B008E6FFA8704F
:10A81B0008085694004003D38001C392B300000094
:10A82B00000000000000000000000000000000001D
:10A83B0000D2B0000000000000000000000000008B
:10A84B0000000000000000A87008EFC313F6A8700A
:10A85B000680AED2B1C2B3000000000000000000C1
:0BA86B000000000000000000000000E2
:07A87600057005700570225A
:0B8990007B00E5702409F97A007F04E9
:10899B00157015701570A870C6EBC608C6EAC60828
:0D89AB00C6E9C61570A870EFF615701570BE
:1089B800C2B100000000000000000000000000003C
:1089C800000000000000A870E4F6A870E6FFC39459
:1089D80004503BC2B0EFB40103D38001C392B3008B
:1089E800000000000000000000000000000000007F
:1089F800000000D2B00000000000000000000000ED
:108A0800000000000000000000A8700680BCA870EC
:108A1800E4F6A870087608A870E6C39404504AC221
:108A2800B008E6FFA87008085694004003D38001F8
:108A3800C392B30000000000000000000000000026
:108A480000000000000000D2B0000000000000009C
:108A580000000000000000000000000000A87008EE
:108A6800EFC313F6A8700680AED2B2000000000073
:108A7800000000000000000000000000000000C22C
:108A8800B2A870E4F6E5702403F8CBE6CB08E6FA62
:108A980008E6F9120A3200000000A870E6C394182C
:108AA8005070C2B00000000000000000000000008C
:108AB8000000000000000000E5702403F8CBE6CBBE
:108AC80008E6FA08E6F91208F578011208E2C8EC97
:108AD800C8C9EDC9CAEECACBEFCBA2B4E4334BFF89
:108AE800EAFEE9FDE8FCE5702403F8CBE6CB08E6EE
:108AF800FA08E6F9120945D2B000000000000000AB
:108B080000000000000000000000000000A870063F
:108B18008088D2B1000000000000000000000000C2
:088B2800000000000000000045
:078B3000E5702406F5702238
:10A55000E570240BF8E6FFE570240CF8E6FD7B07B8
:10A560008F468D47CAEBCA7B8012ABFEE4FBAD473A
:10A57000AF4612A61A7B80AD47AF4612A61A755396
:0DA58000017B06AD47AF46128CD812911C2E
:0DA58D0075486475490300D549FCD548F6B2
:10A59A00EA5407FF75F008E546A42547F582E43535
:10A5AA00F0F583E5822489F582E5833413F583EF98
:10A5BA00F0CFEACFCDEFCD7F0212912775F008E5F3
:10A5CA0046A42547F582E435F0F583E58224A9F50A
:10A5DA0082E5833415F583E4F012BB01E54675F094
:10A5EA0008A4254725E025E024D9F582E43413F5AB
:04A5FA00830209DCF3
:1062E7001570A870EBF61570A870EDF61570A8700C
:0862F700EFF6E57024F7F570E5
:1062FF00240AF8E6B4010312A550E570240AF8E663
:10630F00FF64027042E570240DF8E6B40839E570B9
:10631F00240EF8CBE6CB08E6FA08E6F9120714FECE
:10632F00E570240CF8E6FDE570240BF8E675F0082F
:10633F00A42DF582E435F0F583E5822489F582E515
:10634F00833413F583EEF0EF64036003026689E58F
:10635F0070240DF8E6D3940740057F0002668BE5A5
:10636F0070240BF8E6FFE570240C12A745E57024A6
:10637F0008F8E65401D39400405F12BB01ECC0E073
:10638F00EDC0E0EEC0E0EFC0E0E570240BF8E6757D
:10639F00F008A4FFE570240CF8EF2625E025E02493
:1063AF00D9F582E43413F583E0FCA3E0FDA3E0FE0E
:1063BF00A3E0242CFBEE3401FAE43DF9E43CF8D0E1
:1063CF00E0FFD0E0FED0E0FDD0E0FCC31208D150DA
:1063DF000312A5507F0002668BE570240CF8E6FFD0
:1063EF00E570240BF8E675F008A42FF582E435F07C
:1063FF00F583E58224A9F582E5833415F583E0FF63
:10640F00E570240DF8E66F60057F0002668B12BB06
:10641F0001EFC0E0E570240BF8E6F975F008A4FF72
:10642F00E570240CF8E6FB2F25E025E024D9F58252
:10643F00E43413F583D0E0FF1209DCCFE9CFCDEBC5
:10644F00CD128CD37B00E5702404128996E570245D
:10645F0009F8E66468702CE570240CF8E6FFE57027
:10646F00240BF8E6FE75F008A42FF582E435F0F55D
:10647F0083E58224A9F582E5833415F583E004547E
:10648F0003802AE570240CF8E6FFE570240BF8E68C
:10649F00FE75F008A42FF582E435F0F583E582242C
:1064AF00A9F582E5833415F583E0045407FD75F0F3
:1064BF0008EEA42FF582E435F0F583E58224A9F5E3
:1064CF0082E5833415F583EDF0E570240CF8E6FFD3
:1064DF00E570240BF8E6FE75F008A42FF582E4357D
:1064EF00F0F583E58224A9F582E5833415F583E081
:1064FF00C454F04408FD75F008EEA42FF582E4357E
:10650F00F0F583E5822489F582E5833413F583E082
:10651F004DFD7F02129127E5702404F812095FE404
:10652F001203BDE4FBFA7980784B1202A7E57024C1
:10653F000CF8E6FBE570240BF8E675F008A42BF5D4
:10654F0082E435F0F583E5822489F582E5833413FF
:10655F00F583E025E025E024D2F582E43440F5838D
:10656F0012099012019EA8701209D0E5702409F843
:10657F00E6B460028014E5702409F8E6B461028085
:10658F0043E5702409F8E6B46211A870E8C0E01280
:10659F00095FE4FBFA7980783F8018E5702409F8E9
:1065AF00E6B46317A870E8C0E012095FE4FBFA795C
:1065BF0020784112019ED0E0F88034E5702409F86C
:1065CF00E6B4682EE4FBFA79207840E8C0E0A870C2
:1065DF0012095FD0E0F81202A7E4FBFA79A0784124
:1065EF0012019EE4FBFA792078C11200ADA8701257
:1065FF0009D0E5702409F8E6FF64616009EF646370
:10660F006004EFB4682A7F007E507DC37C47A8707A
:10661F0012097712019EE4FBFAF9783F1200AD12CE
:10662F0003FBEC1203BD7B007A5079C378478028B7
:10663F007F007E247D747C49A87012097712019E19
:10664F00E4FBFAF9783F1200AD1203FBEC1203BD25
:10665F007B007A24797478491202A7A8701209D0A6
:10666F00A87012095FE570240EF8CBE6CB08E6FAA6
:0C667F0008E6F91209457F0480027F0044
:07668B00E5702411F57022F7
:1051CA001570A870EBF61570A870EDF61570A8703A
:0851DA00EFF6E57024F3F57017
:1051E200240EF8E6B4012DE570240FF8E6FFE57011
:1051F2002410F8E6FD7B0F12A560E5702410F8E696
:1052020025E025E02499F582E43413F583120A019E
:105212003F800000E570240EF8E66402600302524B
:10522200D9E5702411F8E6640860030252D9E570EA
:105232002412F8CBE6CB08E6FA08E6F91208F5E5FF
:10524200702410F8E6FB25E025E02499F582E43489
:1052520013F5831209DCEB25E025E02499F582E4BD
:105262003413F583E0FCA3E0FDA3E0FEA3E0FF7BA3
:105272000A7AD77923783C1203446002502AE570F7
:105282002410F8E625E025E02499F582E43413F5AC
:1052920083E0FCA3E0FDA3E0FEA3E0FFE4FBFA79D8
:1052A200207841120344502FE5702410F8E625E0DF
:1052B20025E02499F582E43413F583120A013F8034
:1052C2000000E5702412F8CBE6CB08E6FA08E6F90E
:1052D200120A323F800000E570240EF8E664036093
:1052E2000302567EE5702411F8E6D3940740057F49
:1052F20000025680E570240FF8E6FFE570241012D4
:10530200A745E5702408F8E65401D39400406F12D3
:10531200BB01ECC0E0EDC0E0EEC0E0EFC0E0E57044
:10532200240FF8E675F008A4FFE5702410F8EF26C4
:1053320025E025E024D9F582E43413F583E0FCA3CB
:10534200E0FDA3E0FEA3E0242CFBEE3401FAE43DF1
:10535200F9E43CF8D0E0FFD0E0FED0E0FDD0E0FC84
:10536200C31208D15013E570240FF8E6FFE570244C
:1053720010F8E6FD7B0F12A5607F00025680E570F3
:105382002410F8E6FDE570240FF8E6FE75F008A497
:105392002DF582E435F0F583E58224A9F582E583D3
:1053A2003415F583E0FFE5702411F8E66F60057FA0
:1053B20000025680CFEECF128CD3128990E5702472
:1053C20010F8E6FFE570240FF8E6FE75F008A42F4A
:1053D200F582E435F0F583E58224A9F582E583348C
:1053E20015F583E0045407FD75F008EEA42FF5824D
:1053F200E435F0F583E58224A9F582E5833415F5D9
:1054020083EDF0E5702410F8E6FFE570240FF8E66E
:1054120075F008A42FF582E435F0F583E58224A91E
:10542200F582E5833415F583E0C454F0440FFD7F23
:1054320002129127E5702409F812095FE41203BDF4
:10544200E4FBFA7980784B1202A77B0A7AD7792398
:10545200784012019EA8701209D0A87012095FE567
:10546200702404F81209D0E5702411F8E6D39400F0
:10547200403BA870E8C0E012095FE570240FF8E62F
:1054820075F008A4FBE5702410F8EB2625E025E072
:105492002419F582E43414F583E0F8A3E0F9A3E0DB
:1054A200FAA3E0FB1200A9D0E0F81209D0E57024BB
:1054B20004F812095FE570240FF8E675F008A4FB02
:1054C200E5702410F8EB2625E025E02419F582E4A6
:1054D2003414F5831209DCA870E8C0E012095FEC0D
:1054E200C0E0EDC0E0EEC0E0EFC0E0E5702410F8EF
:1054F200E625E025E02499F582E43413F583E0FC07
:10550200A3E0FDA3E0FEA3E0FF7B6F7A127983782C
:105512003A12019EC8ECC8C9EDC9CAEECACBEFCB9C
:10552200D0E0FFD0E0FED0E0FDD0E0FC1202A7D038
:10553200E0F81209D0E570240DF8E6B47318A870EB
:10554200E8C0E012095FE4FBFA792078411202A771
:10555200D0E0F81209D07F757E787D0C7C35A8707A
:1055620012097712019EA87012097712019EA87083
:1055720012097712019EECC0E0EDC0E0EEC0E0EF50
:10558200C0E07FFA7EED7D6B7C3AA870120977123B
:10559200019EA87012097712019ED0E0FBD0E0FABA
:1055A200D0E0F9D0E0F81200ADECC0E0EDC0E0EEE2
:1055B200C0E0EFC0E07F177ED97D167C40A8701254
:1055C200097712019ED0E0FBD0E0FAD0E0F9D0E0FA
:1055D200F81200AD7BD37A4D79E278411200ADA882
:1055E200701209D0A870E8C0E012095F7B337A9389
:1055F200798878431200A9D0E0F81209D0E4FFFEBE
:105602007D207C41A87012097712019EE4FBFAF911
:10561200783F1200AD1203FBEC1203BDE4FBFA79F2
:105622002078411202A7A8701209D07F007EC07DA7
:10563200797C44A870120977120344600B4009A8D0
:10564200701209E84479F99AE4FFFE7D487CC3A808
:10565200701209771203445009A8701209E8C4793C
:10566200F99AA87012095FE5702412F8CBE6CB080C
:0E567200E6FA08E6F91209457F0480027F017E
:07568000E5702415F570220E
:1046F8001570A870EBF61570A870EDF61570A87017
:08470800EFF6E57024F6F570F0
:10471000240BF8E664017055E570240AF8E6B477D6
:1047200012E570240CF8E6FFE570240DF8E6FD7B39
:10473000888010E570240CF8E6FFE570240DF8E69B
:10474000FD7B8C12A560E570240DF8E6FFE5702472
:104750000CF8E675F008A42FF582E435F0F583E552
:104760008224A9F582E5833415F583E4F0E570240D
:104770000BF8E664036003024C60E570240EF8E673
:10478000D3940240057F00024C62E570240CF8E6E9
:10479000FFE570240DF8E6FD7B00E5702404F97A4E
:1047A0000012A751E5702404F8E65401D394005098
:1047B0000302483E12BB01ECC0E0EDC0E0EEC0E0F9
:1047C000EFC0E0E570240CF8E675F008A4FFE57092
:1047D000240DF8EF2625E025E024D9F582E43413F2
:1047E000F583E0FCA3E0FDA3E0FEA3E0242CFBEEB8
:1047F0003401FAE43DF9E43CF8D0E0FFD0E0FED02B
:10480000E0FDD0E0FCC31208D1502EE570240AF878
:10481000E6B47712E570240CF8E6FFE570240DF895
:10482000E6FD7B888010E570240CF8E6FFE5702437
:104830000DF8E6FD7B8C12A5607F00024C62E570EE
:10484000240DF8E6FDE570240CF8E6FE75F008A4EA
:104850002DF582E435F0F583E58224A9F582E58320
:104860003415F583E0FFE5702405F8EFF65401FFF9
:10487000E570240EF8EF6660057F00024C62CFEE13
:10488000CF128CD37B00E5702406128996E5702444
:104890000AF8E66477600302492FE570240DF8E614
:1048A000FFE570240CF8E6FE75F008A42FF582E40D
:1048B00035F0F583E58224A9F582E5833415F58387
:1048C000E0045401FD75F008EEA42FF582E435F004
:1048D000F583E58224A9F582E5833415F583EDF0AF
:1048E000E570240DF8E6FF75F008EEA42FF582E4DC
:1048F00035F0F583E58224A9F582E5833415F58347
:10490000E070047D8880027D987F02129127E57017
:104910002406F812095FE41203BDE4FBFA798078FB
:104920004B1202A77B0A7AD779A3783C0249BFE5EC
:1049300070240DF8E6FFE570240CF8E6FE75F0082B
:10494000A42FF582E435F0F583E58224A9F582E50C
:10495000833415F583E0045401FD75F008EEA42FAF
:10496000F582E435F0F583E58224A9F582E5833408
:1049700015F583EDF0E570240DF8E6FF75F008EE0F
:10498000A42FF582E435F0F583E58224A9F582E5CC
:10499000833415F583E0C454F0448CFD7F021291FA
:1049A00027E5702406F812095FE41203BDE4FBFA60
:1049B0007980784B1202A77B0A7AD779A3783E12C6
:1049C000019EA8701209D0E570240AF8E6FF64750C
:1049D0006008EF64766003024ABBA870E8C0E0128A
:1049E000095F7B6F7A127983783A1202A7D0E0F8D8
:1049F0001209D0E570240AF8E6B47618A870E8C069
:104A0000E012095FE4FBFA792078411202A7D0E0B6
:104A1000F81209D07F757E787D0C7C35A87012095C
:104A20007712019EA87012097712019EA8701209D0
:104A30007712019EECC0E0EDC0E0EEC0E0EFC0E018
:104A40007FFA7EED7D6B7C3AA87012097712019E89
:104A5000A87012097712019ED0E0FBD0E0FAD0E0F6
:104A6000F9D0E0F81200ADECC0E0EDC0E0EEC0E03F
:104A7000EFC0E07F177ED97D167C40A870120977C1
:104A800012019ED0E0FBD0E0FAD0E0F9D0E0F812BD
:104A900000AD7BD37A4D79E278411200ADA8701257
:104AA00009D0A870E8C0E012095F7B337A93798857
:104AB00078431200A9D0E0F8024BDEE570240AF832
:104AC000E664776003024BE1A870E8C0E012095F7A
:104AD0007B007A247974784912019ED0E0F812099B
:104AE000D07F5D7E0B7D237C2CA87012097712018C
:104AF0009EA87012097712019EA870120977120100
:104B00009EA87012097712019EECC0E0EDC0E0EEA5
:104B1000C0E0EFC0E07F177EEE7D8B7C32A8701284
:104B2000097712019EA87012097712019EA87012CF
:104B3000097712019EC8ECC8C9EDC9CAEECACBEF0D
:104B4000CBD0E0FFD0E0FED0E0FDD0E0FC1200A929
:104B5000ECC0E0EDC0E0EEC0E0EFC0E07F4B7E5F78
:104B60007D047C38A87012097712019EA870120982
:104B70007712019ED0E0FBD0E0FAD0E0F9D0E0F867
:104B80001200ADECC0E0EDC0E0EEC0E0EFC0E07FB1
:104B90004B7E767D6C7C3DA87012097712019ED009
:104BA000E0FBD0E0FAD0E0F9D0E0F81200AD7B1FD6
:104BB0007A85796B78BE1200ADA8701209D0E4FF37
:104BC000FEFDFCA8701209771203446014A870124D
:104BD0000977E4FFFE7D7A7C441202A7A8701209CF
:104BE000D0E4FFFE7DC87C42A87012097712019EB6
:104BF000E4FBFAF9783F1200AD1203FBEC1203BD9F
:104C0000E4FBFA79C878421202A7A8701209D07F93
:104C10005C7EFF7D797C44A87012097712034460A2
:104C20000B4009A8701209E84479FF5CE4FFFE7D9F
:104C3000487CC3A8701209771203445009A8701267
:104C400009E8C479FF5CA87012095FE570240FF8C9
:104C5000CBE6CB08E6FA08E6F91209457F048002A4
:024C60007F01D2
:074C6200E5702412F5702239
:106D1E001570A870EBF61570A870EDF61570A870CA
:086D2E00EFF6E57024F7F570A3
:106D3600E570240AF8E66401704FE570240BF8E666
:106D4600FFE570240CF8E6FD7B0512A560E57024CE
:106D56000CF8E6FFE570240BF8E675F008A42FF5AD
:106D660082E435F0F583E58224A9F582E5833415BE
:106D7600F583E4F0EF25E025E02499F582E4341369
:106D8600F583120A013F800000E570240AF8E664E4
:106D9600036003027003E570240DF8E6D394074000
:106DA600057F00027005E570240BF8E6FFE5702408
:106DB6000CF8E6FD7B00E5702404F97A0012A75171
:106DC600E5702404F8E65401D39400406F12BB0129
:106DD600ECC0E0EDC0E0EEC0E0EFC0E0E570240BF3
:106DE600F8E675F008A4FFE570240CF8EF2625E018
:106DF60025E024D9F582E43413F583E0FCA3E0FD15
:106E0600A3E0FEA3E0242CFBEE3401FAE43DF9E412
:106E16003CF8D0E0FFD0E0FED0E0FDD0E0FCC312AD
:106E260008D15013E570240BF8E6FFE570240CF842
:106E3600E6FD7B0512A5607F00027005E570240C57
:106E4600F8E6FDE570240BF8E6FE75F008A42DF5CE
:106E560082E435F0F583E58224A9F582E5833415CD
:106E6600F583E0FFE570240DF8E66F60057F00020C
:106E76007005CFEECF128CD37B00E5702405128906
:106E860096E570240CF8E6FFE570240BF8E6FE752F
:106E9600F008A42FF582E435F0F583E58224A9F500
:106EA60082E5833415F583E0045407FD75F008EE9A
:106EB600A42FF582E435F0F583E58224A9F582E571
:106EC600833415F583EDF0E570240CF8E6FFE570E4
:106ED600240BF8E675F008A42FF582E435F0F58367
:106EE600E58224A9F582E5833415F583E0C454F0E0
:106EF6004405FD7F02129127E5702405F812095F0B
:106F0600E41203BDE4FBFA7980784B1202A77B0AF0
:106F16007AD779A3783F12019EC8ECC8C9EDC9CAD1
:106F2600EECACBEFCB7F0A7ED77D237C3F1200A92A
:106F3600A8701209D0A870E8C0E012095FE4FBFA55
:106F4600797A78441202A7D0E0F81209D0A870E83E
:106F5600C0E012095F7B007A247974784912019E99
:106F6600D0E0F81209D0A870E8C0E012095F7B9A59
:106F76007A99798878431200A9D0E0F81209D0E40A
:106F8600FFFE7DC87C42A87012097712019EE4FBC1
:106F9600FAF9783F1200AD1203FBEC1203BDE4FBD5
:106FA600FA79C878421202A7A8701209D0E4FFFE47
:106FB6007D167C43A870120977120344600B4009C2
:106FC600A8701209E84479FF5CE4FFFE7D5C7CC290
:106FD600A8701209771203445009A8701209E8C470
:106FE60079FF5CA87012095FE570240EF8CBE6CB3A
:0F6FF60008E6FA08E6F91209457F0480027F01D8
:07700500E5702411F5702273
:0CA87D007F0112927C7FFC12A8897F00F2
:08A889001570A870EFF61570C0
:10A89100C2B3C2B1000000000000000000000000CF
:10A8A1000000000000000000A870E4F6A870E6C3F4
:10A8B10094085047D2B008E6FF548094004003D377
:10A8C1008001C392B30000000000000000000000FE
:10A8D100000000000000000000C2B0000000000005
:10A8E100000000000000000000000000000000A8BF
:10A8F1007008EF25E0F6A8700680B1D2B1C2B300AE
:10A901000000000000000000000000000000000046
:03A9110000000043
:05A91400057005702232
:10927C001570A870EDF61570A870EFF615701570D6
:10928C00C2B3C2B1000000000000000000000000EA
:10929C000000000000000000A8700808E62450A898
:1092AC007008F6A870E4F6A870E6C394085047D28C
:1092BC00B008E6FF548094004003D38001C392B3FE
:1092CC000000000000000000000000000000000092
:1092DC0000000000C2B00000000000000000000010
:1092EC0000000000000000000000A87008EF25E05E
:1092FC00F6A8700680B1A8700808E62450A870087B
:10930C00F6A870E4F6A870E6C394085040D2B0C238
:10931C00B30000000000000000000000000000008E
:10932C000000000000C2B0000000000000000000BF
:10933C00000000000000000000000008E8C0E0E6AB
:10934C0025E0FFD0E0F8EFF6A8700680B8A870E42E
:10935C00F6A870E6C39408504ED2B0E5702403F81A
:10936C00E6FF5480D394004003D38001C392B30032
:10937C0000000000000000000000000000000000E1
:10938C00000000C2B000000000000000000000005F
:10939C00000000000000000000E5702403F8EF2539
:1093AC00E0F6A8700680AAD2B1C2B300000000009B
:0F93BC00000000000000000000000000000000A2
:0793CB00E5702404F5702297
:108FB600157015701570A870C6EBC608C6EAC60807
:098FC600C6E9C6E57024FCF57053
:108FCF00C2B100000000000000000000000000001F
:108FDF00000000000000F8087601A870E4F6A87001
:108FEF00E6C394085047D2B008E6FF54809400407F
:108FFF0003D38001C392B300000000000000000003
:10900F000000000000000000000000C2B0000000DF
:10901F000000000000000000000000000000000041
:0D902F0000A87008EF25E0F6A8700680B1DB
:10903C00A87008087605A8700808E6D394004022AA
:10904C00E5702403F87613E5702403F8E6D3940056
:10905C00400900E5702403F81680ECA87008081687
:02906C0080D4AE
:10906E00A870E4F6E5702404F8CBE6CB08E6FA081F
:10907E00E6F9120A3200000000A870E6C3941850F8
:10908E0070D2B000000000000000000000000000E0
:10909E0000000000000000E5702404F8CBE6CB08C9
:1090AE00E6FA08E6F91208F578011208E2C8ECC8EB
:1090BE00C9EDC9CAEECACBEFCBA2B4E4334BFFEA7B
:1090CE00FEE9FDE8FCE5702404F8CBE6CB08E6FAF1
:1090DE0008E6F9120945C2B00000000000000000C9
:1090EE00000000000000000000000000A8700680D4
:1090FE0088D2B10000000000000000000000000057
:07910E00000000000000005A
:07911500E5702407F570224C
:106692001570A870EBF61570A870EDF61570A8705D
:0866A200EFF6E57024F6F57037
:1066AA00240BF8E664016003026781E570240CF8A4
:1066BA00E6FFE570240D12BA907D027F0012927CEB
:1066CA001D7F0212927C7DD07F0312927C7FF01292
:1066DA00A889E5702404F81209E8000000007FA0E8
:1066EA007E867D017C00E5702404F8120977C312C6
:0766FA0008D1505730B554E0
:10670100E5702408F87601E5702408F8E6D39400D2
:106711004023E5702409F87603E5702409F8E6D3EF
:106721009400400900E5702409F81680ECE5702416
:0567310008F81680D2FB
:10673600E5702404F812095FEF2401FFE43EFEE44D
:106746003DFDE43CFCE5702404F81209D080937DFD
:106756000F12A87DE570240DF8E6FFE570240CF80D
:10676600E675F008A42FF582E435F0F583E582247A
:10677600F9F582E5833414F583E4F0E570240BF82B
:10678600E664036003026A0EE570240EF8E6D3940D
:106796000740057F00026A10E570240CF8E6FFE565
:1067A60070240D12BA90E5702404F81209E800006E
:1067B6000000E47F107E27FDFCE5702404F8120932
:0A67C60077C31208D1505730B554C4
:1067D000E5702408F87601E5702408F8E6D3940003
:1067E0004023E5702409F87603E5702409F8E6D320
:1067F0009400400900E5702409F81680ECE5702447
:0568000008F81680D22B
:10680500E5702404F812095FEF2401FFE43EFEE47D
:106815003DFDE43CFCE5702404F81209D08094E4C5
:106825007F107E27FDFCE5702404F8120977C3125A
:1068350008D17004FF026A10E570240DF8E6FEE544
:1068450070240CF8E675F008A42EF582E435F0F511
:1068550083E58224F9F582E5833414F583E0FDE5CB
:1068650070240EF8E66D60057F00026A10E570245D
:106875000DF8E6FFE570240CF8E6FCED045407FD81
:1068850075F008ECA42FF582E435F0F583E5822454
:10689500F9F582E5833414F583EDF075F008ECA481
:1068A5002EF582E435F0F583E58224F9F582E5835A
:1068B5003414F583E0C454F0440FFD12A87D7B0029
:1068C500E5702404F97A00128FB6E5702404F812F5
:1068D500095F78081208E2EC1203BDA8701209D00E
:1068E500E4FBFA7980784FE8C0E0A87012095FD020
:1068F500E0F81202A7E4FBFA79A0784012019EA8FD
:10690500701209D0E570240AF8E6B46402803FE508
:1069150070240AF8E6B4652DE4FBFA79207840E89E
:10692500C0E0A87012095FD0E0F81202A7E4FBFAF4
:1069350079A0784112019EE4FBFA792078C1120012
:10694500ADA870803EE570240AF8E6B46617A87015
:10695500E8C0E012095FE4FBFA7980783F12019EF6
:10696500D0E0F8801EE570240AF8E6B46718A87030
:10697500E8C0E012095FE4FBFA7920784112019E34
:10698500D0E0F81209D0E570240AF8E6FF646560E6
:1069950004EFB4672A7F007E407D1C7C46A87012F8
:1069A500097712019EE4FBFAF9783F1200AD120354
:1069B500FBEC1203BD7B007A40791C784680287F6A
:1069C500007E507DC37C47A87012097712019EE4B2
:1069D500FBFAF9783F1200AD1203FBEC1203BD7B05
:1069E500007A5079C378471202A7A8701209D0A877
:1069F5007012095FE570240FF8CBE6CB08E6FA08BC
:0B6A0500E6F91209457F0480027F01C2
:076A1000E5702412F570226D
:107B46001570A870EBF61570A870EDF61570A87094
:087B5600EFF6E57024F5F5706F
:107B5E00240CF8E664036003027DE9E570240FF857
:107B6E00E6FED3940340057F00027DEB7401C8EE60
:107B7E00C8088002C333D8FCA8700808F6758401C3
:107B8E00E5702403F81209E800000000A870E4F67E
:107B9E00A870E6C3940A4003027C56E4F5CCF5CDFA
:107BAE00F5C975C804E570240DF8E6FFE570240EDE
:107BBE0012BA90E570240DF8E6FFE570240EF8E693
:107BCE00FDE4FB12BA957F0012B899E570240DF80A
:107BDE00E6FFE570240EF8E6FD7B00A970097A0039
:107BEE0012A751A8700808C9E8C9A87008E657601E
:107BFE0005E5C830E7D0E4F5C8E5702403F8E8C021
:107C0E00E012095FECC0E0EDC0E0EEC0E0EFC0E0D6
:107C1E00AFCDEFFEADCC7C00E42DFFEC3ECBEFCB39
:107C2E00FAE4F9F8D0E0FFD0E0FED0E0FDD0E0FCC1
:107C3E00EF2BFFEE3AFEE93DFDE83CFCD0E0F812FA
:107C4E0009D0A87006027B9EE5C85480FFBF0127AD
:107C5E00E570240BF8E6B4700FE5702407F81209EE
:107C6E00E8411FFFFF027DCCE5702407F81209E8FA
:107C7E004479FFFE027DCCE5702403F812095FE41F
:107C8E001203BDECC0E0EDC0E0EEC0E0EFC0E0A836
:107C9E0070E6FCE41203C7C8ECC8C9EDC9CAEECA47
:107CAE00CBEFCBD0E0FFD0E0FED0E0FDD0E0FC1279
:107CBE0002A7E4FBFA79C478421202A7E4FBFA7930
:107CCE0040784112019EE5702407F81209D0E57044
:107CDE002407F8E8C0E012095F7B007A24797478F3
:107CEE00491202A7D0E0F81209D0E570240BF8E68D
:107CFE0064707BCD7ACC798C783F7044E8C0E0E537
:107D0E00702407F812095FD0E0F81202A77B007A00
:107D1E00B8790878491202A77B287A6B796E784E6B
:107D2E0012019EE5702407F81209D0E5702407F8B9
:107D3E00E8C0E012095F7B777ABE799F783D80417B
:107D4E00E8C0E0E5702407F812095FD0E0F81202EF
:107D5E00A7E4FBFA79AF78451202A77B287A6B79F4
:107D6E006E784E12019EE5702407F81209D0E57068
:107D7E002407F8E8C0E012095F7B9A7A9979F978BE
:107D8E00401200A9D0E0F81209D0E4FFFE7D7A7C03
:107D9E0044E5702407F812097712019EE4FBFAF904
:107DAE00783F1200AD1203FBEC1203BDE4FBFA792F
:107DBE007A78441202A7E5702407F81209D0E5700C
:107DCE002407F812095FE5702410F8CBE6CB08E61D
:0D7DDE00FA08E6F91209457F0480027F01D2
:077DEB00E5702413F570227E
:1016BF001570A870EBF61570A870EDF61570A87080
:0816CF00EFF6E57024F0F57060
:1016D700E5702412F8E675F008A4FFE5702413F806
:1016E700EF26FFE570240DF8EFF6E5702411F8E614
:1016F70064046003021817E5702414F8E67032E5F5
:1017070070240DF8E625E025E02459F582E4341429
:10171700F583120A0142960000E5702415F8CBE61E
:10172700CB08E6FA08E6F9120A32429600000218D8
:1017370012E5702414F8E6B40132E570240DF8E6DA
:1017470025E025E02469F582E43415F583120A01C2
:1017570000000000E5702415F8CBE6CB08E6FA0890
:10176700E6F9120A3200000000021812E57024148C
:10177700F8E6B40231E570240DF8E625E025E0240B
:1017870099F582E43414F583120A013F800000E5DD
:10179700702415F8CBE6CB08E6FA08E6F9120A3208
:1017A7003F8000008065E5702414F8E6FFB4032B42
:1017B700E570240DF8E625E024D9F582E43414F524
:1017C70083E4F0A3743CF0E5702415F8CBE6CB086E
:1017D700E6FA08E6F9E475F03C802DEFB4042CE551
:1017E70070240DF8E625E024F9F582E43417F58333
:1017F700E4F0A37405F0E5702415F8CBE6CB08E612
:10180700FA08E6F9E475F00512088E7F0002202831
:10181700E570240DF8E62419F582E43418F583E021
:1018270060030218EE12BB01E570240DF8E625E00F
:1018370025E02409F582E43415F583E0F8A3E0F9FF
:10184700A3E0FAA3E0FBC3EF9BFFEE9AFEED99FD41
:10185700EC98FCECC0E0EDC0E0EEC0E0EFC0E0E5E6
:1018670070240DF8E625E024D9F582E43414F583D5
:10187700E0FEA3E0FF7C007D6412078ECBEFCBCAAE
:10188700EECAE4F9F8D0E0FFD0E0FED0E0FDD0E00A
:10189700FCC31208D140030219CAE570240DF8E60B
:1018A7002419F582E43418F5837401F012BB01E5BD
:1018B70070240DF8E6FB25E025E02409F582E434E1
:1018C70015F5831209DCEB25E025E02459F582E4C0
:1018D7003414F583E0FCA3E0FDA3E0FEA3E0FFA83A
:1018E700701209D002199312BB01E570240DF8E6B6
:1018F70025E025E02409F582E43415F583E0F8A313
:10190700E0F9A3E0FAA3E0FBC3EF9BFFEE9AFEED3D
:1019170099FDEC98FCECC0E0EDC0E0EEC0E0EFC054
:10192700E0E570240DF8E625E024F9F582E43417A4
:10193700F583E0FEA3E0FF7C007D6412078ECBEF0A
:10194700CBCAEECAE4F9F8D0E0FFD0E0FED0E0FD64
:10195700D0E0FCC31208D1506AE570240DF8E624E4
:1019670019F582E43418F583E4F012BB01E570241D
:101977000DF8E625E025E02409F582E43415F58322
:101987001209DCA8701209E800000000A9701570A0
:1019970015701570A870760008760008C6E9C61598
:1019A70070A870E4F6E5702417F8E61570A870F6CD
:1019B700E5702417F8E6FB7D02E5702415F8E6FFCD
:1019C7001216BFE5702411F8E664016003021A6A73
:1019D700E5702412F8E6FFE5702413F8E6FD7B0EA8
:1019E70012ABFEE5702412F8E6FFE5702413F8E663
:0C19F700FD7B0E12A61A128CC512911C6A
:101A0300E570240EF87664E570240EF8E6D39400AE
:101A13004023E570240FF87603E570240FF8E6D32E
:101A23009400400900E570240FF81680ECE570245B
:051A33000EF81680D240
:101A38007D077F02129127E570240DF8E62419F539
:101A480082E43418F5837401F012BB01E570240DAB
:101A5800F8E625E025E02409F582E43415F583123B
:101A680009DCE5702411F8E664026003021D40E514
:101A7800702414F8E6703FE5702415F8CBE6CB081F
:101A8800E6FA08E6F91208F5E4FBFAF9F812034455
:101A98005024E5702415F8CBE6CB08E6FA08E6F9F9
:101AA8001208F5E570240DF8E625E025E02459F53F
:101AB80082E434148058E5702414F8E6B40124E56F
:101AC800702415F8CBE6CB08E6FA08E6F91208F513
:101AD800E570240DF8E625E025E02469F582E43474
:101AE80015802BE5702414F8E6B40229E570241556
:101AF800F8CBE6CB08E6FA08E6F91208F5E5702413
:101B08000DF8E625E025E02499F582E43414F58300
:101B18001209DC8062E5702414F8E6FFB4032BE5B3
:101B2800702415F8CBE6CB08E6FA08E6F912082B7C
:101B3800FDE570240DF8E625E024D9F582E4341497
:101B4800F583E5F0F0A3EDF0802DEFB40429E570FE
:101B58002415F8CBE6CB08E6FA08E6F912082BFFBD
:101B6800E570240DF8E625E024F9F582E43417F54C
:101B780083E5F0F0A3EFF0E5702414F8E6D39400C1
:101B880040057F00022028E5702415F8CBE6CB0835
:101B9800E6FA08E6F91208F5A8701209D0E4FFFE83
:101BA800FDFCA8701209771203445009A8701209A5
:101BB800E800000000E4FFFE7DC87C42A87012091E
:101BC80077120344600B4009A8701209E842C80064
:101BD80000E4FBFA79C87842E8C0E0A87012095F0F
:101BE800D0E0F81202A77B007AFF797F78471201CC
:101BF8009E1203FBE570240AF8EEF608EFF6E5708E
:101C08002412F8E6FFE5702413F8E6FDE4FB12A6BB
:101C18001AE570240CF8E4F6E570240CF8E6FFC326
:101C280094045033EF940140047F0480027F001233
:101C3800A5FEE5702412F8E6FFE5702413F8E6FD2A
:101C4800E5702405F8E64408FB12A61A12A605E575
:101C580070240CF80680C1E570240CF8E4F6E570F1
:101C6800240CF8E6C39404504DE5702414F8E654A7
:101C780008D3940040047F0480027F0012A5FEE58B
:101C8800702412F8E6FFE5702413F8E6FDE57024E9
:101C980005F8E64408FB12A61A12A605E5702414F6
:101CA800F8E8C0E0E625E0FFD0E0F8EFF6E57024BC
:101CB8000CF806021C66E570240CF8E4F6E57024BE
:101CC8000CF8E6C39410505DE570240AF8E65480D9
:101CD800FED3E49400EE940040047F0480027F0069
:101CE80012A5FEE5702412F8E6FFE5702413F8E665
:101CF800FDE5702405F8E64408FB12A61A12A605AD
:101D0800E570240AF8E8C0E0C9E8C909E725E0FF5A
:101D180019E733FED0E0F8EEF608EFF6E570240C8C
:101D2800F806021CC5E5702412F8E6FFE5702413D6
:101D3800F8E6FD7B0E12A61AE5702411F8E6640396
:101D48006003022026E5702414F8E67013E5702479
:101D58000DF8E625E025E02459F582E434148036B0
:101D6800E5702414F8E6B40113E570240DF8E625AF
:101D7800E025E02469F582E43415801AE57024141E
:101D8800F8E6B40221E570240DF8E625E025E02404
:101D980099F582E43414F583E0FCA3E0FDA3E0FEAA
:101DA800A3E0FF02200DE5702414F8E6FEB4032832
:101DB800E570240DF8E625E024D9F582E43414F51D
:101DC80083E0F9A3E0FDE5702415F8CBE6CB08E63F
:101DD800FA08E6C98DF0802AEEB4042EE570240DC9
:101DE800F8E625E024F9F582E43417F583E0F9A351
:101DF800E0FFE5702415F8CBE6CB08E6FA08E6C95B
:101E08008FF012088E7F02022028E5702414F8E66D
:101E1800640560057F00022028E5702412F8E6FFBB
:101E2800E5702413F8E6FD7B00E5702404F97A00D8
:101E380012A751E5702404F8E65401D39400400534
:101E48007F00022028128CC57B00E57024061289C9
:101E5800967D077F02129127E5702406F812095F24
:101E6800E41203BDE4FBFA7980784B1202A77B0ADF
:101E78007AD779A3784012019E7B0A7AD77923789A
:101E8800C01200ADA8701209D0A870E8C0E012090D
:101E98005F7B387A1F7943784112019ED0E0F812AF
:101EA80009D0A870E8C0E012095FECC0E0EDC0E01E
:101EB800EEC0E0EFC0E0E570240DF8E625E025E08F
:101EC8002459F582E43414F583E0FCA3E0FDA3E093
:101ED800FEA3E0FFE4FBFA797A78441202A7C8EC83
:101EE800C8C9EDC9CAEECACBEFCBD0E0FFD0E0FE3F
:101EF800D0E0FDD0E0FC1202A7D0E0F81209D07BB8
:101F0800CD7ACC792C7840E8C0E0A87012095FD06F
:101F1800E0F81202A7C8ECC8C9EDC9CAEECACBEFEF
:101F2800CBE4FFFE7DC87C421200A9A8701209D03C
:101F3800E570240DF8E625E025E02469F582E4340F
:101F480015F583E0F8A3E0F9A3E0FAA3E0FBE8C005
:101F5800E0A87012095FD0E0F81200A9E570240D1E
:101F6800F8E625E025E02499F582E43414F583E0C9
:101F7800F8A3E0F9A3E0FAA3E0FB12019EA870120F
:101F880009D07F007E507DC37C47A8701209771264
:101F9800019EE4FBFAF9783F1200AD1203FBEC1244
:101FA80003BD7B007A5079C378471202A7A8701244
:101FB80009D0E570240DF8E62419F582E43418F503
:101FC80083E06401705412BB01E570240DF8E62526
:101FD800E025E02409F582E43415F583E0F8A3E070
:101FE800F9A3E0FAA3E0FBC3EF9BFFEE9AFEED999D
:101FF800FDEC98FCE47B64FAF9F8C31208D1501A96
:10200800A87012095FE5702415F8CBE6CB08E6FA4C
:1020180008E6F91209457F0480067F0080027F01E7
:07202800E5702418F5702299
:107DF2001570A870EBF61570A870EDF61570A870E6
:087E0200EFF6E57024F5F570C0
:107E0A00E570240CF8E664017021E570240DF8E6AB
:107E1A00FFE570240EF8E6FD7BFF12A61AE5702432
:107E2A000DF8E6FFE570240E12ABF9E570240CF8A4
:107E3A00E66403600302808BE570240FF8E6701293
:107E4A00E570240DF8E6FFE570240EF8E6FD7BFEEA
:107E5A008010E570240DF8E6FFE570240EF8E6FDC3
:107E6A007BFD12A61AE570240DF8E6FFE570240ED4
:037E7A0012BA90A9
:107E7D00E5702409F8760AE5702409F8E6D3940034
:107E8D004023E570240AF87603E570240AF8E6D35A
:107E9D009400400900E570240AF81680ECE5702482
:057EAD0009F81680D267
:107EB20030B418E570240DF8E6FFE570240EF8E6FC
:107EC200FD7BFF12A61A7F0002808DE5702404F864
:107ED2001209E800000000E5702408F8E4F6E570F5
:107EE2002408F8E6C3941B5075000000000000004F
:107EF20000000000000000000000000000D2B000FE
:107F0200000000000000000000000000000000006F
:107F1200000000C2B00000000000000000000000ED
:107F2200000000000000000000E5702404F81209BF
:107F32005F78011208E2C8ECC8C9EDC9CAEECACB23
:107F4200EFCBA2B4E4334BFFEAFEE9FDE8FCE570B7
:107F52002404F81209D0E5702408F8068080E57040
:107F6200240DF8E6FFE570240EF8E6FD7BFF12A66D
:107F72001AE5702404F812095FE4FFFEFDEC5402D6
:107F8200FC601EE5702404F812095FE4FFFEFDECBC
:107F92005401FC600CA8701209E840200000028025
:107FA20028E5702404F812095FE4FFFEFDEC540298
:107FB200FCE4FBFAF9F8C31208D1701DE570240441
:107FC200F812095FE4FFFEFDEC5401FC600BA8709F
:107FD2001209E800000000804DE5702404F812093F
:107FE2005FE4FFFEFDEC5402FCE4FBFAF9F8C31275
:107FF20008D1700CE5702404F812095F74FF80093F
:10800200E5702404F812095FE4FC1203BDE4FBFAF4
:108012007980784B1202A7E4FBFA792078401201AA
:108022009EA8701209D0E4FFFEFD7C41A8701209DF
:108032007712019EE4FBFA792078C11200ADA87094
:108042001209D07F007E247D747C49A870120977C2
:1080520012019EE4FBFAF9783F1200AD12A4A07B54
:10806200007A24797478491202A7A8701209D0A85C
:108072007012095FE5702410F8CBE6CB08E6FA0827
:0B808200E6F91209457F0480027F0030
:07808D00E5702413F57022D9
:10853F00E5702412F8E675F003A42459F582E434AB
:10854F0013F583E0FBA3E0FAA3E0F9E570240DF83F
:10855F00E675F004A4F58285F0831209158F4D8E10
:10856F004C8D4B8C4AE570240FF8E6FFE570241113
:10857F00F8E6FDE5702412F8E6FBE570240DF8E649
:02858F00F549AC
:068591008F468D478B4868
:10859700E4FFFEFDFCAB4DAA4CA94BA84A120344CD
:1085A7005009E4F54DF54CF54BF54AE546B4852001
:1085B700E4FFFE7D347C43AB4DAA4CA94BA84A127D
:1085C700034460324030E4F54DF54C754B3480235D
:1085D700E546B48621E4FFFE7D8C7C43AB4DAA4C77
:1085E700A94BA84A120344600D400BE4F54DF54C26
:1085F700754B8C754A43AF4DAE4CAD4BAC4AECC096
:10860700E0EDC0E0EEC0E0EFC0E0E54875F008A49B
:108617007C002549FFEC35F0FEEF7802C333CE33FB
:10862700CED8F924F9F58274153EF583D0E0FFD052
:10863700E0FED0E0FDD0E0FC1209DCE546B4851988
:10864700E4FBFA79937842AF4DAE4CAD4BAC4A128E
:1086570002A7E4FBFA79208018E4FBFA79937842C1
:10866700AF4DAE4CAD4BAC4A1202A77B6F7A127975
:108677008378401202A77B007AFF797F784712013F
:108687009E1203FB8E4E8F4F7B48AD48AF4712A615
:108697001A7B06AD48AF4712BA95E4FDEDD39401B6
:1086A7004003D38001C392B3000000000000000024
:1086B700000000000000000000000000D2B0000031
:1086C70000000000000000000000000000000000A3
:1086D7000000C2B00DBD04C4E4FDE5495408D394BD
:1086E700004003D38001C392B300000000000000E4
:1086F70000000000000000000000000000D2B000F1
:108707000000000000000000000000000000000062
:10871700000000C2B0E54925E0F5490DBD04BBE402
:10872700FDE54E5480FED3E49400EE94004003D35D
:108737008001C392B30000000000000000000000A9
:10874700000000000000000000D2B00000000000A0
:10875700000000000000000000000000000000C250
:10876700B0E54F25E0F54FE54E33F54E0DBD10B1A1
:098777007B40AD48AF4702A61A91
:0E9FD200E5702411F8E6FFE5702412F8E6FDB4
:109FE0008F468D477B7812ABFEE4FBAD47AF461240
:029FF000A61AAF
:0D9FF20075486475490300D549FCD548F653
:109FFF007B40AD47AF4612A61A7B70AD47AF4612F6
:10A00F00A61A7B06AD47AF4612BA9512911C7D1169
:05A01F007F07129127EC
:0DA0240075486475490300D549FCD548F620
:10A031007D577F0212912775F008E546A42547F563
:10A0410082E435F0F583E5822449F582E583341510
:10A05100F583E4F075F008E546A42547F582E4357B
:10A06100F0F583E5822459F582E5833415F583E41F
:10A07100F07B40AD47AF4612A61A12BB01E546750B
:10A08100F008A4254725E025E024D9F582E434131E
:10A09100F5831209DC12BB01E54675F008A42547DA
:10A0A10025E025E024B9F582E43415F5830209DCC5
:102965001570A870EBF61570A870EDF61570A870C7
:08297500EFF6E57024F1F570A6
:10297D00E5702411F8E6FF75F008A4FEE570241249
:10298D00F8E6FD2EFEE570240EF8EEF6E570241047
:10299D00F8E6B40112129FE07E027F007D007B01FC
:1029AD007A117959120B22E5702410F8E664026051
:1029BD0003022A62E5702413F8E6FED3940740055E
:1029CD007F00023242EE7029E5702414F8CBE6CB7D
:1029DD0008E6FA08E6F9E5702412F8E675F003A4A6
:1029ED002459F582E43413F583EBF0A3EAF0A3E95F
:1029FD00F0E5702414F8CBE6CB08E6FA08E6F912F8
:102A0D0008F5E4FBFA798078BF1200ADA8701209C1
:102A1D00D0E570240FF8E6FFEFC0E0E5702411F863
:102A2D00E6FDEDC0E0E5702412F8E6FBE570241339
:102A3D00F8E6F549A87012095F8F4D8E4C8D4B8CC1
:102A4D004AD0E0FDD0E0FF12859112BB018F188EA8
:102A5D00178D168C15E5702410F8E66403600302DB
:102A6D003240E5702413F8E6FFC394084006EFD317
:102A7D00941740057F00023242E5702411F8E6FFFD
:102A8D00E570241212A745E5702408F8E65401D329
:102A9D009400407C12BB01ECC0E0EDC0E0EEC0E064
:102AAD00EFC0E0E5702411F8E675F008A4FFE570BD
:102ABD002412F8EF2625E025E024D9F582E434131D
:102ACD00F583E0FCA3E0FDA3E0FEA3E0242CFBEEE8
:102ADD003401FAE43DF9E43CF8D0E0FFD0E0FED05B
:102AED00E0FDD0E0FCC31208D15025129FD2E57055
:102AFD00240DF8E4F6E570240DF8E6C39408500BA8
:102B0D0012853FE570240DF80680EA7F00023242FF
:102B1D00E5702408F8E65402D39400407C12BB0102
:102B2D00ECC0E0EDC0E0EEC0E0EFC0E0E5702411D8
:102B3D00F8E675F008A4FFE5702412F8EF2625E0FD
:102B4D0025E024B9F582E43415F583E0FCA3E0FD1E
:102B5D00A3E0FEA3E0242CFBEE3401FAE43DF9E4FE
:102B6D003CF8D0E0FFD0E0FED0E0FDD0E0FCC31299
:102B7D0008D15025129FD2E570240DF8E4F6E570CA
:102B8D00240DF8E6C39408500B12853FE570240D13
:102B9D00F80680EA7F00023242E5702408F8E6303C
:102BAD00E003022F95E5702412F8E6FFE57024117D
:102BBD00F8E675F008A42FF582E435F0F583E5828B
:102BCD002449F582E5833415F583E02408FFE433C9
:102BDD00FEE5702413F8E66F7001EE60057F0002CC
:102BED00324212BB01EFC0E0E5702411F8E6F97531
:102BFD00F008A4FFE5702412F8E6FB2F25E025E090
:102C0D0024D9F582E43413F583D0E0FF1209DCCF2B
:102C1D00E9CFCDEBCD7B5012A61AE5702411F8E665
:102C2D00FFE5702412128CD0128990E5702412F8F1
:102C3D00E6FFE5702411F8E6FE75F008A42FF58285
:102C4D00E435F0F583E5822449F582E5833415F505
:102C5D0083E0045407FD75F008EEA42FF582E435EA
:102C6D00F0F583E5822449F582E5833415F583ED8E
:102C7D00F0E5702412F8E6FFE5702411F8E675F022
:102C8D0008A42FF582E435F0F583E5822449F58219
:102C9D00E5833415F583E09040F293C454F0440776
:102CAD00FD7F02129127E5702411F8E6FFE57024EF
:102CBD0012F8E6FD7B4012A61AE570240FF8E6B473
:102CCD008529E5702409F812095FE41203BDE4FBC0
:102CDD00FA7980784B1202A77B0A7AD779A37840CC
:102CED0012019E7B0A7AD779238030E570240FF884
:102CFD00E6B48633E5702409F812095FE41203BDCA
:102D0D00E4FBFA7980784B1202A77B587A39790661
:102D1D00784112019E7B3F7A35798678C01200ADDD
:102D2D00A8701209D08009A8701209E800000000EF
:102D3D00A870E8C0E012095FE4FBFA79CA78421284
:102D4D00019ED0E0F81209D0E5702412F8E675F076
:102D5D0008A4FFE5702413F8E67C002FFFEC35F096
:102D6D00FEEF7802C333CE33CED8F92439F5827411
:102D7D00113EF583E0FCA3E0FDA3E0FEA3E0FFE53B
:102D8D00702404F81209D0E4FFFE7D807CBFE5704D
:102D9D002404F81209771203446048A870E8C0E0D3
:102DAD0012095FECC0E0EDC0E0EEC0E0EFC0E07FE7
:102DBD000A7ED77D237C3CE5702404F81209771236
:102DCD00019EC8ECC8C9EDC9CAEECACBEFCBD0E0A5
:102DDD00FFD0E0FED0E0FDD0E0FC1200A9D0E0F87D
:102DED001209D0E4FFFE7D7A7C44A8701209771297
:102DFD00019EE4FBFAF9783F1200AD1203FBEC12D1
:102E0D0003BDE4FBFA797A78441202A7A87012097F
:102E1D00D0A87012095FE5702414F8CBE6CB08E654
:102E2D00FA08E6F912094512BB01C8ECC8C9EDC98B
:102E3D00CAEECACBEFCBE5182432FFE43517FEE41A
:102E4D003516FDE43515FCD31208D15003022F9031
:102E5D00E5702413F8E624F8FFE434FFFEEF780262
:102E6D00C333CE33CED8F9FFE5702412F8E675F0F2
:102E7D0003A42459F582E43413F583E0FBA3E0FAAF
:102E8D00A3E0F98F828E831209A0E8C0E0A870122A
:102E9D00095FD0E0F81200A9E5702404F81209D0FA
:102EAD00E5702404F812095F12BB6B7B6F7A1279FF
:102EBD0083783A1203444003022F90E5702404F8FE
:102ECD0012095F12BB6BE4FBFA79207841120344BF
:102EDD0060025003022F90E4FFFEFD7C40E570245C
:102EED0004F8120977120344600E400CE5702404B7
:102EFD00F81209E840000000E4FFFEFD7CC0E5701B
:102F0D002404F8120977120344500CE5702404F8D8
:102F1D001209E8C0000000E5702412F8E675F0080B
:102F2D00A4FFE5702413F8E67C002FFFEC35F0FECE
:102F3D00EF7802C333CE33CED8F924D9F582741588
:102F4D003EF583E0FCA3E0FDA3E0FEA3E0FFE5700A
:102F5D002404F81209771200A98F4D8E4C8D4B8CDD
:102F6D004AE570240FF8E6FFE5702411F8E6FDE55B
:102F7D00702412F8E6FBE5702413F8E624F8F54901
:102F8D001285917F04023242E5702408F8E630E1A3
:102F9D000302323CE5702412F8E6FFE5702411F8C7
:102FAD00E675F008A42FF582E435F0F583E582246B
:102FBD0059F582E5833415F583E02410FFE433FEE3
:102FCD00E5702413F8E66F7001EE60057F000232A4
:102FDD004212BB01EFC0E0E5702411F8E6F975F07F
:102FED0008A4FFE5702412F8E6FB2F25E025E02468
:102FFD00B9F582E43415F583D0E0FF1209DCCFE991
:10300D00CFCDEBCD7B6012A61AE5702411F8E6FF4B
:10301D00E5702412128CD0128990E5702412F8E616
:10302D00FFE5702411F8E6FE75F008A42FF582E493
:10303D0035F0F583E5822459F582E5833415F58362
:10304D00E0045407FD75F008EEA42FF582E435F089
:10305D00F583E5822459F582E5833415F583EDF08A
:10306D00E5702412F8E6FFE5702411F8E675F00816
:10307D00A42FF582E435F0F583E5822459F582E538
:10308D00833415F583E09040FA93C454F04406FD63
:10309D007F02129127E5702411F8E6FFE5702412E6
:1030AD00F8E6FD7B4012A61AE5702413F8E624F02D
:1030BD00FFE434FFFEEF7802C333CE33CED8F9FFF1
:1030CD00E5702412F8E675F003A42459F582E43472
:1030DD0013F583E0FBA3E0FAA3E0F98F828E831250
:1030ED000915E4FBFA79707841120344600E400C27
:1030FD00A8701209E8BF8000000231D6E570240FD8
:10310D00F8E6B4852BE5702409F812095FE4120383
:10311D00BDE4FBFA7980784B1202A77B0A7AD77946
:10312D0023784012019E7B0A7AD779A378BF80322B
:10313D00E570240FF8E6B48633E5702409F812091A
:10314D005FE41203BDE4FBFA7980784B1202A77B92
:10315D00DD7A247986784012019E7BDD7A2479060A
:10316D0078C01200ADA8701209D08009A87012099C
:10317D00E8000000007B007A40791C7846E8C0E04A
:10318D00A87012095FD0E0F81202A77B007A2479AB
:10319D0074784912019EA8701209D0E4FFFE7D7A61
:1031AD007C44A87012097712019EE4FBFAF9783F6E
:1031BD001200AD1203FBEC1203BDE4FBFA797A7831
:1031CD00441202A7A8701209D0A87012095FECC0B2
:1031DD00E0EDC0E0EEC0E0EFC0E0E5702412F8E6EF
:1031ED0075F008A4FFE5702413F8E67C002FFFECC2
:1031FD0035F0FEEF7802C333CE33CED8F92419F56E
:10320D008274113EF583D0E0FFD0E0FED0E0FDD01A
:10321D00E0FC1209DCA87012095FE5702414F8CBEC
:10322D00E6CB08E6FA08E6F91209457F0480067F29
:05323D000080027F018A
:07324200E5702417F570226E
:10B7D80020202020557067726164696E6700202000
:10B7E80020204669726D776172652E2E2E003230E8
:10B7F80031352D30362D3132202D20326132313322
:03B80800613800A4
:08B699000184FF421839FFFF94
:1093D2007BFF7AB779F67D2D12B39FEA494B60196C
:1093E2007BFF7AB779F67D2D12B39FE92402F9E467
:1093F2003A8B44F54589468004E4FEFF22AB44AA39
:1094020045A94690000112072DFFC3648094B04025
:109412000ED3EF648094B95006EF24D0FF801E90E3
:10942200000112072DFFC3648094E1400ED3EF6464
:109432008094E65006EF24A9FF80027F00EF7D00B2
:10944200FC120714FFC3648094B0400ED3EF648013
:1094520094B95006EF24D0FF8021AB44AA45A94617
:10946200120714FFC3648094E1400ED3EF6480942A
:10947200E65006EF24A9FF80027F00EFC454F04CAF
:10948200FCAB44AA45A94690000212072DFFC36413
:109492008094B0400ED3EF648094B95006EF24D08C
:1094A200FF801E90000212072DFFC3648094E140EA
:1094B2000ED3EF648094E65006EF24A9FF80027F6A
:1094C20000EF75F010A4FFEC45F0FEED4FFF9000A9
:1094D2000312072DFDC3648094B0400ED3ED648067
:1094E20094B95006ED24D0FD8024AB44AA45A94688
:1094F20090000312072DFDC3648094E1400ED3ED6A
:10950200648094E65006ED24A9FD80027D00EF4DB3
:09951200FF901A26EEF0A3EFF021
:01951B00222D
:1072EB00E47880F612BB27C28575840F75E104E440
:1072FB00F5E275E344F58475B7B075840F758A8331
:10730B00F597438901758D01758F01758E04F542D3
:10731B00F5430543E54370020542640F454270F2A5
:10732B00438902E4F542F543AE42AF43E4FCFD7BF7
:10733B00507AC3F9F8D31208BB400FE58920E40A51
:10734B000543E54370E2054280DE75970212AF807C
:10735B0012B0578F41E4F584E541D39400400EE51C
:10736B00EF5402D394004005AF41128B3712B98B07
:10737B00E4FF12B9AA43EF04E4F542F5437D01AFF4
:10738B004312B86C0543E54370020542C39402E512
:10739B0042940040E8E4F520C22FC22DC233C23222
:1073AB00C2317880F6C23408F67886F618F6788BF8
:1073BB00F6F542F54374452543F58274183542F5CD
:1073CB0083E4F00543E54370020542B400E7E54270
:1073DB00B401E2E4F542F54374452543F582741993
:1073EB003542F583E4F00543E54370020542644002
:1073FB00454270E4E4F584E5EF20E10CE5EF540839
:10740B00D394004003D38001C392037D08E4FF12A1
:10741B00B4987D087F0112B498124102E4788AF681
:10742B007882F6AB1DAA1EA91F7882E6FF75F01DA8
:10743B00A4F58285F08312072DFE788A26F6EE607E
:10744B000578820680DDEFD394004032AB1DAA1E77
:10745B00A91F90000D120A6D120714F541745512F5
:10746B00075A12071464556002D23174AA12075AD4
:10747B0012071464AA6002D231E54112075AE4F5EF
:10748B0084E5EF5402D3940040047F018002E4FFB3
:10749B00129E068F40E54020E036C22E74FF788D99
:1074AB00F608F608F608F67E007F107D007B007A62
:1074BB00007993120B227548FF754982754AF17555
:1074CB004B00754C107B007A00799312B3F5800258
:1074DB00D22E1293D27891A60608A607E54030E18A
:1074EB0003027596E4F542F543AB1DAA1EA91F8551
:1074FB004382854283741D120A4C12072D700302BE
:10750B00758DAE42AF437C007D1D12078EE92FF9BE
:10751B00EA3EFA90000412072D20E25BE4F53FE50A
:10752B003FC3787D965050AB1DAA1EA91F85438281
:10753B00854283741D120A4C12072DFF7E00C00674
:10754B00C0077F00C007AE42AF437C007D1D120712
:10755B008EE92FF9EA3EFA90000D120A6D788AE651
:10756B00853FF0A429F9EA35F0FAD005D007D0060B
:10757B00120B22053F80A80543E54370020542022A
:10758B0074F47F0112700CC2308007E4FF12700C90
:10759B00D230E4F542F5437A007B967D03AF43127C
:1075AB00AAD80543E54370020542C39402E5429411
:0375BB000040E4A9
:0175BE0022AA
:05BB9000788BE6FF22A6
:030023000298D16F
:1098D100C0E0C0F0C083C082C0D075D000C000C05D
:1098E10001C002C003C004C005C006C00730993ED4
:1098F100C2997886067986E77881667015F678864A
:01990100F66F
:0D99020075270A75281300D528FCD527F617
:04990F00C285801C71
:0D99130075271475281300D528FCD527F6FC
:109920007886E62445F582E43419F583E0F599203C
:1099300098030299CC209A08202F05C2980299C852
:10994000C29A7885E6062445F582E43418F583E565
:1099500099F0C298E6FFB40112901845E0FE70033A
:10996000F68069EE54072402788CF6EFB4020D7885
:109970008CE6B40907901846E02403F67885E6FFE4
:10998000B40007E4B40103F68042EFC3788C96403C
:109990003B7885E624FFFDE434FFFC7B017A1879EF
:1099A0004512AC867885E62444F582E43418F583C4
:0899B000E06F600476008014F2
:0D99B80075271475281300D528FCD527F657
:1099C50012202F78857600D007D006D005D004D098
:1099D50003D002D001D000D0D0D082D083D0F0D037
:0299E500E0326E
:10002600901846E075F01DA4AB1D251FF9E51E3599
:10003600F0FA90000D120A6D788BE6FF18E68FF045
:10004600A4252BF582E435F0F58312072DFF7B00FE
:040056007A0079298A
:10005A008F398B3A8A3B893CE4F584EA494B601C28
:10006A00AB3AAA3BA93C120714FFE539FD7C001202
:0C007A00BB78AB3AAA3BA93CEF12075A36
:0D008600753D14753E1300D53EFCD53DF6CA
:0E0093008539997F0112B8993099FDC29922E2
:10B7A2009019457478F07885E62444F582E43418DB
:09B7B200F583E0901946F07F02D6
:09B7BB00E4F5847881EFF6D285F3
:0DB7C400753914753A1300D53AFCD539F6E5
:07B7D100901945E0F59922F3
:10B62200C9EFC9E964017028EDC39B4034787DE617
:10B63200FFEB2FFFE433FEEDC39FEE6480F87480CE
:10B6420098501ED22FC3ED9B788BF6788776012215
:10B65200B90214ED6B700AD22F788BF678877602D6
:08B6620022C22FE47887F622D2
:10B12A00C9EFC9BAFF15BBFF12ED6B7002EC6A706A
:10B13A0049D22F788BF67887E9F622E964017025DF
:10B14A00C3ED9BEC9A401C787DE62BFFE43AFEC3E4
:10B15A00ED9FEC9E500DD22FC3ED9B788BF678872E
:10B16A007601228015B90218ED6B7002EC6A700A3A
:10B17A00D22F788BF67887760222C22FE47887F668
:01B18A0022A2
:10202F00901845E0FF54F8F52AE4F584EF120AF60C
:10203F00207F09208C0A209F1020A81120B9122080
:10204F00D01920E61A210B2021142821B02922B201
:10205F003322ED37231D39233741234249234D4E78
:10206F0023805023C861227C7023C098000023F87E
:10207F00901846E0FD788EE6FB7F0180279018468A
:10208F00E0FCA3E0FD788DE6FA08E6FB7F01802BEC
:10209F00D22F788776030223F8901846E0FD7890C8
:1020AF00E6FB7F0212B6220223F8901846E0FCA34B
:1020BF00E0FD788FE6FA08E6FB7F0212B12A0223D1
:1020CF00F8901846E0FD788EE6FB7F0112B62220CD
:1020DF002F030223F8801A901846E0FCA3E0FD7846
:1020EF008DE6FA08E6FB7F0112B12A202F030223A7
:1020FF00F89019457478F07F010223F5E4F58475A3
:10210F00EF100223F8C2ACE4F529D285FB7A0079EF
:10211F00297F7F12005A7B007A0079297F1E1200D7
:10212F005A7B007A0079297F0512005A7882E612CD
:10213F000053788DE6120053788EE6120053788F95
:10214F00E61200537890E61200537891E61200538E
:10215F007892E6120053E4F52B7493252BF8E612D0
:10216F000053052BE52BC3941040EEE4F52B74338D
:10217F00252BF582E43418F583E0120053052BE587
:10218F002BC3940640E87B007A007900AF29120038
:01219F005AE5
:0D21A00075370A75381300D538FCD537F6B1
:1021AD00022267901846E0FFC37882964003022210
:1021BD006EEF75F01DA4251FF9E51E35F0851D3454
:1021CD00F5358936C2ACE4F529D285FB7A0079293B
:1021DD007F7F12005A7B007A0079297F0D12005AF9
:1021ED00AB34AA35A936120714120053AB34AA35F5
:1021FD00A936900001120050AB34AA35A9369000D3
:10220D0002120050AB34AA35A936900003120050CB
:10221D00AB34AA35A936900004120050E4F52BAB6F
:10222D0034E5362405F9E43535FA7E00E9252BF938
:10223D00EE3AFA120714120053052BE52BC394083E
:0D224D0040DD7B007A007900AF2912005AB5
:0D225A0075370A75381300D538FCD537F6F6
:10226700C285D2AC0223F89019457478F0E4A3F044
:102277007F020223F512BB1478A31209D0901945E7
:10228700747CF078A3E6A3F008E6A3F008E6A3F0D1
:1022970008E6A3F07C007D057B017A19794512AC2D
:1022A7008690194AEFF07F060223F5901846E0FF63
:1022B700B4010FA3E0FDA3E0788DCDF608EDF6029B
:1022C70023C0EFB4020A901847E0788DF60223C0C6
:1022D700901846E0B4030CA3E0FFA3E0788FCFF695
:1022E70008EFF60223C0E4F52B901846E0FFE52B34
:1022F700C39F501B7447252BF582E43418F583E000
:10230700FF7493252BF8EFF6052BE52BB410DAE4D1
:1023170078A2F60223C07A007B327D01788BE6FF34
:1023270012AAD8901846E0FDE4FF12B4980223F8E9
:10233700901846E024FF92020223F8901846E02402
:10234700FF92010223F87A007B327D017F0012AAF7
:10235700D8E4F52B7446252BF582E43418F583E091
:10236700FF743B252BF582E43418F583EFF0052B3A
:10237700E52BB406DFD2348078788BE66005752DBF
:1023870002800B203205752D038003752D019019EE
:10239700457479F0A3E52DF07C007D027B017A1965
:1023A700794512AC86901947EFF07F0312B7BBE56A
:1023B7002D6401703CD2338002D22D788076F18073
:1023C700307A007B327D017F0012AAD890194574BC
:1023D70079F0901846E0901946F07C007D027B0169
:1023E7007A19794512AC86901947EFF07F0312B737
:1023F700BBE52A64A06003022607901845E064A1A4
:1024070060030224F7A3E0C378829640030224EC1A
:10241700AB1DAA1EA91FE0FF75F01DA4F58285F06C
:102427008312072DF52DEF75F01DA429F9EA35F074
:10243700FA90000412072D30E237901846E012BBDD
:102447008B8F2D901945747FF0A3E52DF02402FDA5
:10245700E433FC7B017A19794512AC867447252D44
:10246700F582E43419F583EFF0E52D2403FF022606
:1024770004901846E0FF12BB8BC2ACE4F529D28565
:10248700E52DD39406402B7B007A0079297F7F12B4
:10249700005A7B007A007929AF2D12005AE4F52BF8
:1024A700E52BC3952D5007120026052B80F2052D2D
:1024B7008018E52D2478120053E4F52BE52BC395FE
:1024C7002D5007120026052B80F27B007A00790039
:0524D700AF2912005ABC
:0D24DC0075370A75381300D538FCD537F672
:1024E9000225F69019457478F07F010226049018A8
:1024F90045E064A260030226077882E6FFA3E0FEB6
:10250900C39F40030225FCA3E0FDC39F40030225AE
:10251900FCEE9D40030225FC901846E0F52BE4F5FE
:1025290032F533901847E0FFE52BD39F5026AF2BA8
:1025390012BB8BAB1DAA1EA91F75F01DE52BA4F5B7
:102549008285F08312072D2533F533E43532F532D0
:10255900052B80CFC2ACE4F529D285FB7A00792915
:102569007F7F12005AC3E5339480E532940050020C
:102579008007E5324480120053AF3312005490189B
:1025890046E0F52B901847E0FFE52BD39F5046E432
:10259900F52CAB1DAA1EA91F75F01DE52BA4F5820C
:1025A90085F08312072DFFE52CC39F5024E52B7579
:1025B900F01DA429F9EA35F0FA90000D120A6D7898
:1025C9008BE6FF18E68FF0A4252C120049052C8014
:1025D900C1052B80AF7B007A007900AF2912005A20
:0D25E90075370A75381300D538FCD537F664
:1025F600C285D2AC800B9019457478F07F0112B772
:10260600BBE52A6458704DFA7B327D01788BE6FF74
:1026160012AAD8753C01753D19753E467B017A189C
:10262600794612BAC68F2DE52D2478901945F0EF1C
:102636002401FDE433FC7B017A19794512AC8674DA
:1026460046252DF582E43419F583EFF0E52D2402B5
:10265600FF12B7BBE52A64806009E52A6488600337
:1026660002282C7887E6B4010F7A007B327D017848
:102676008BE6FF12AAD8801AE4F52BE52BC3787DEA
:1026860096500F7A007B327D01AF2B12AAD8052B0C
:1026960080E9901845E05407F52DB4070A752C011A
:1026A600A3E0F52DA38006E4F52C901846E0F52E60
:1026B600152DE52EC37882964003022819AB1DAA74
:1026C6001EA91F75F01DE52EA4F58285F08312075D
:1026D6002DFFE52DD39F40028F2D7887E6B40109A3
:1026E600788BE6F531F5308009E4F530787DE6142F
:1026F600F531788BA630788BE6D3953140030227E7
:10270600F0E4F52BE52BC3952D40030227E5E52ED6
:1027160075F01DA4AB1D251FF9E51E35F0FA9000D6
:102726000412072D30E2030227E090000112072D64
:1027360064387041E52DD394044011E52C252B24F3
:1027460047F582E43418F583E0FD80707885E6C3AA
:10275600952BFFE49400FE74432FF58274183EF522
:1027660083E0FDE52E75F01DA4AB1D251FF9E51EC2
:1027760035F0FA8047AB1DAA1EA91F75F01DE52E80
:10278600A4F58285F08312072DFF7885E6C39FFFA7
:10279600E49400FE7C00EF252BFFEC3EFEEF252C9B
:1027A600FFEC3EFE74442FF58274183EF583E0FD7F
:1027B600E52E75F01DA429F9EA35F0FA90000D1200
:1027C6000A6D788BE6FF18E68FF0A4FFE52B2FF550
:1027D60082E435F0F583ED12076C052B02270AAF6C
:1027E6002E12B83D788B060226FC788BA630E52E95
:1027F60075F01DA4AB1D251FF9E51E35F0FA9000F6
:102806000412072D30E5047884A62EE52A64887024
:10281600158010E52EB4FF0E901847E0F520E52A46
:10282600B4880312B7A2E52A64A860030229647873
:1028360087E6B4010F7A007B327D01788BE6FF12C2
:10284600AAD8801AE4F52BE52BC3787D96500F7A2B
:10285600007B327D01AF2B12AAD8052B80E9901898
:1028660046E030E711547FFEA3E0FDEEF532EDF5CC
:1028760033752C03800C901846E0753200F53375DD
:102886002C027445252CF582E43418F583E0FF7498
:1028960046252CF582E43418F583E0F52F8F2EE5D6
:1028A6002ED3952F4003022961E52EC378829640E8
:1028B6000302295CAB1DAA1EA91F75F01DE52EA4F7
:1028C600F58285F08312072DF52D7887E6B4010988
:1028D600788BE6F531F5308009E4F530787DE6143D
:1028E600F531788BA630788BE6D39531505EE4F5DA
:1028F6002BE52BC3952D504AE52E75F01DA4AB1D77
:10290600251FF9E51E35F0FA90000412072D20E286
:102916002DE52C252B2447F582E43418F583E0FDBC
:1029260090000D120A6D788BE6FF18E68FF0A4FF73
:10293600E52B2FF582E435F0F583ED12076C052BB8
:1029460080AFAF2E12B83D788B06809A788BA63072
:0E295600E52D252CF52C052E0228A512B7A282
:012964002250
:10B5D5008E6C8F6D901839E0656C7004A3E0656D15
:10B5E500603A901829740AF0E56CA3F0E56DA3F0B4
:10B5F5007C007D037B017A18792912AC8690182C82
:10B60500EFF07B017A187929750D017D047C001214
:0DB61500AA46901839E56CF0A3E56DF0220F
:03B44700CCEECC7C
:10B44A00901829741AF0A3ECF0EFA3F07C007D03A6
:10B45A007B017A18792912AC8690182CEFF07B01BF
:10B46A007A187929750D017D047C0012AA467B01A0
:10B47A007A1879297D0A7C0012A268EF7002FF22ED
:0DB48A00901829E0647860037F00227F01A4
:01B497002292
:10F000007880E664F1600302F668E478ADF608F60D
:05F010007881E6601E9E
:0DF01500753F0A75401300D540FCD53FF64D
:10F0220078AE06E61870010678ADB627E108B6108C
:10F03200DDC2AF7584015398FC75FFDE75FFADE448
:10F0420078A9F618F6E4F584209830E478ADF6084D
:10F05200F6209823C378AEE6948818E694135017E6
:0DF06200753F0A75401300D540FCD53FF600
:10F06F0078AE06E61870DD0680DAB28680CD78A815
:10F07F00A699C298E6FF641A6008EF640A6003025B
:10F08F00F168E478ADF608F6209823C378AEE694DD
:07F09F008818E694135017D6
:0DF0A600753F0A75401300D540FCD53FF6BC
:10F0B30078AE06E61870DD0680DA30988778A9A660
:10F0C30099C298E478ADF608F6209823C378AEE6A3
:08F0D300948818E6941350170D
:0DF0DB00753F0A75401300D540FCD53FF687
:10F0E80078AE06E61870DD0680DA20980302F0474D
:10F0F80078A9A699C298E478ADF608F6209823C3B3
:0BF1080078AEE6948818E694135017C8
:0DF11300753F0A75401300D540FCD53FF64E
:10F1200078AE06E61870DD0680DA20980302F04714
:10F1300078A9A699C29818E6641A600302F659D213
:03F1400085C299EC
:0DF14300753F1475401300D540FCD53FF614
:06F150007599783099FD6D
:0DF15600753F0A75401300D540FCD53FF60B
:10F16300C28502F65978A8E6FF6450600302F1FDF8
:10F1730078ADF608F6209823C378AEE6948818E6AF
:04F18300941350177A
:0DF18700753F0A75401300D540FCD53FF6DA
:10F1940078AE06E61870DD0680DA20980302F047A0
:0AF1A40078A9A699C298D285C299F5
:0DF1AE00753F1475401300D540FCD53FF6A9
:08F1BB007599793099FDC299A4
:0DF1C300753F1475401300D540FCD53FF694
:08F1D0007599013099FDC29907
:0DF1D800753F1475401300D540FCD53FF67F
:06F1E500E4F5993099FDEC
:0DF1EB00753F0A75401300D540FCD53FF676
:0EF1F800C28502F659EF6401703ED285C299BD
:0DF20600753F1475401300D540FCD53FF650
:08F213007599783099FDC2994C
:0DF21B00753F1475401300D540FCD53FF63B
:06F22800E4F5993099FDA8
:0DF22E00753F0A75401300D540FCD53FF632
:10F23B00C28502F65978A8E66402600302F30C78E3
:10F24B00ADF608F6209823C378AEE6948818E694BA
:03F25B0013501736
:0DF25E00753F0A75401300D540FCD53FF602
:10F26B0078AE06E61870DD0680DA20980302F047C8
:10F27B0078A9A699C298E408F618E6FF13B392860C
:10F28B00EF25E0FEC3E49400EE94F0502DE6FD7FF5
:10F29B000025E0FEC394E05021ED20E024E4F5844A
:10F2AB0043B701758F0378AFEEF608EFF6F5828E54
:10F2BB0083E4F053B7F0F58F800478AA76FFE4F57A
:05F2CB0084D285C29908
:0DF2D000753F1475401300D540FCD53FF686
:08F2DD007599783099FDC29982
:0DF2E500753F1475401300D540FCD53FF671
:08F2F20078AAE6F5993099FDB8
:0DF2FA00753F0A75401300D540FCD53FF666
:10F30700C28502F65978A8E66403600302F46778B9
:10F31700ADF608F6209823C378AEE6948818E694ED
:03F3270013501769
:0DF32A00753F0A75401300D540FCD53FF635
:10F3370078AE06E61870DD0680DA20980302F047FB
:10F3470078A9A699C298E478ADF608F6209823C361
:0BF3570078AEE6948818E69413501777
:0DF36200753F0A75401300D540FCD53FF6FD
:10F36F0078AE06E61870DD0680DA20980302F047C3
:10F37F0078ABA699C29878A9E6FF139286EF25E09D
:10F38F00FEC3E49400EE94F0400302F047E67D00E4
:10F39F0025E0FCC394E0400302F047E4F58443B753
:10F3AF0001758F0178ABE675F020A42DFFE5F03CD9
:10F3BF0078AFF608EFF6E4F58478ACF678ACE6C3F0
:10F3CF009420504CE408F608F6209823C378AEE654
:08F3DF00948818E694135017FE
:0DF3E700753F0A75401300D540FCD53FF678
:10F3F40078AE06E61870DD0680DA20980302F0473E
:10F4040078AF0806E618CEE6CE70010614F5828EB3
:10F4140083E599F0C29878AC0680ACE4F58453B7E0
:09F42400F0F58FF584D285C29940
:0DF42D00753F1475401300D540FCD53FF627
:08F43A007599783099FDC29923
:0DF44200753F1475401300D540FCD53FF612
:06F44F00E4F5993099FD7F
:0DF45500753F0A75401300D540FCD53FF609
:10F46200C28502F65978A8E6FD6404600302F52419
:10F4720078ADF608F6209823C378AEE6948818E6AD
:04F482009413501778
:0DF48600753F0A75401300D540FCD53FF6D8
:10F4930078AE06E61870DD0680DA20980302F0479E
:10F4A30078A9A699C298E625E078B1F608E4F6783B
:10F4B300AAF678ADF608F678B10806E618CEE6CED9
:10F4C30070010614F5828E83E49378AA26F678AE4B
:10F4D30006E61870010678AEE6700418E66402705A
:05F4E300D6D285C2999C
:0DF4E800753F1475401300D540FCD53FF66C
:08F4F5007599783099FDC29968
:0DF4FD00753F1475401300D540FCD53FF657
:08F50A0078AAE6F5993099FD9D
:0DF51200753F0A75401300D540FCD53FF64B
:10F51F00C28502F659ED6405600302F64D78ADF62B
:10F52F0008F6209823C378AEE6948818E694135013
:01F53F0017B4
:0DF54000753F0A75401300D540FCD53FF61D
:10F54D0078AE06E61870DD0680DA20980302F047E3
:10F55D0078A9A699C298E478ADF608F6209823C349
:0BF56D0078AEE6948818E6941350175F
:0DF57800753F0A75401300D540FCD53FF6E5
:10F5850078AE06E61870DD0680DA20980302F047AB
:0AF5950078ABA699C298D285C299FE
:0DF59F00753F1475401300D540FCD53FF6B4
:08F5AC0075997F3099FDC299A9
:0DF5B400753F1475401300D540FCD53FF69F
:10F5C1007599203099FD78A9E625E0FC78ABE675C0
:10F5D100F020A42400FFE5F03C78B1F608EFF6E452
:08F5E10078AAF678ACF6C29995
:0DF5E900753F1475401300D540FCD53FF66A
:10F5F60078B1E6FE08E6F5828E83E493F5993099B4
:10F60600FD78B10806E618CEE6CE70010614F5823E
:10F616008E83E49378AA26F678AC06E6B420C2C2B6
:01F62600994A
:0DF62700753F1475401300D540FCD53FF62B
:08F6340078AAE6F5993099FD72
:0DF63C00753F0A75401300D540FCD53FF620
:10F64900C285800C78A8E6B40606E4F58475EF1047
:0FF6590078A8E66407600302F0477880F6D2AF26
:01F66800227F
:109EEE007F0012B899202E0B7A007B327D017F0005
:109EFE0012AAD830310B7A007B1E7D017F0012AA88
:109F0E00D8302D173032147A007B327D01788BE6F3
:109F1E00FF12AAD8C22D12A6A2D22E20300C303299
:109F2E0009788076F112A6A2D23030332A30322749
:109F3E00C23312BB5EE4FDFF12BADA7BFF7AB77949
:109F4E00D812B8F07D01E4FF12BADA7BFF7AB77946
:109F5E00E612B8F012F00030340B7B017A18793B20
:109F6E0012AE28C23412BB01C8ECC8C9EDC9CAEE84
:109F7E00CACBEFCB90184112096BEF245AFFE43E87
:109F8E00FEE43DFDE43CFCD31208D1500F12BB01A0
:109F9E00901841120984D31208D1401212BB0190BD
:109FAE0018411209DC7B017A18793312A18D203207
:109FBE001212BB01E47B2C7A01F9F8C31208D150BE
:049FCE0002D2322267
:10000E00E4F58475EF027F64DFFE1272EB129EEE52
:05001E00125F0080F8F4
:109798004D656D6F727920746573742E2E2E004D91
:1097A800656D6F7279206572726F722062616E6B7F
:1097B8002025626400005EBCE2613FDD83C29C7EBE
:1097C80020A3FD1F419DC3217FFCA2401E5F01E332
:1097D800BD3E6082DC237D9FC1421CFEA0E1BF5DCF
:1097E8000380DE3C62BEE0025CDF81633D7C22C018
:1097F8009E1D43A1FF4618FAA427799BC584DA3831
:1098080066E5BB5907DB856739BAE406581947A5E9
:10981800FB7826C49A653BD987045AB8E6A7F91B92
:1098280045C6987A24F8A6441A99C7257B3A6486CF
:10983800D85B05E7B98CD2306EEDB3510F4E10F2FC
:10984800AC2F7193CD114FADF3702ECC92D38D6F99
:1098580031B2EC0E50AFF1134DCE90722C6D33D166
:109868008F0C52B0EE326C8ED0530DEFB1F0AE4C7F
:109878001291CF2D73CA947628ABF517490856B4C0
:10988800EA6937D58B5709EBB536688AD495CB2961
:1098980077F4AA4816E9B7550B88D6346A2B75971A
:1098A800C94A14F6A8742AC896154BA9F7B6E80A47
:1098B80054D7896B35000000002B6096CBDDEE0095
:0998C8002C96CBDDE5EEF7FAFD6C
:05B6A100C1B601770AAB
:10BAEE0074FFF51CF51BF51AF519AF1CAE1BAD1A3C
:02BAFE00AC1981
:01BB00002222
:10AC860015701570A870ECF608EDF61570157015B0
:10AC960070A870C6EBC608C6EAC608C6E9C6E5705F
:04ACA60024FCF57025
:10ACAA00F80808E4F6A870F608F6E5702407F9A88B
:10ACBA0070E6FE08E6FFC3099719E76480F8EE64B8
:10ACCA0080985037E5702404F8CBE6CB08E6FA08FA
:10ACDA00E6F98F828E8312072DA870080866FFE5B1
:10ACEA00702403F8EFF6E69097BD93A8700808F66B
:10ACFA00A8700806E61870B20680AFA8700808E6C1
:01AD0A00FF49
:07AD0B00E5702409F5702238
:0BBB7800ED6F78A7F6E69097BD93FFF5
:01BB8300229F
:0300A30002B3495C
:10B34900C0E0C083C082C0D0E8C0E0EEC0E0EFC07A
:10B35900E0E59830E1055398FDD236E59830E024D0
:10B369007876E62401FFE433FEEF64404E700280F4
:10B37900107876E606248EF582E43419F583E5998A
:10B38900F05398FED0E0FFD0E0FED0E0F8D0D0D066
:06B3990082D083D0E032F7
:0AAA46008B088A09890A8C0B8D0C1D
:10AA5000E47876F6758401D284E50D24FF929BE4B8
:10AA6000787EF6787EE6C3950CE50B6480F87480FA
:05AA7000985060C236A1
:0DAA7500750E14750F1300D50FFCD50EF6ED
:10AA8200E50C24FFFFE50B34FFFE787EE66F7001D4
:10AA9200EE701EC2ACAB08050AE50AAA09700205EF
:10AAA2000914F9120714F5993036FDC284D2AC802C
:10AAB20016AB08050AE50AAA097002050914F9127B
:10AAC2000714F5993036FD7F0112B899787E068019
:05AAD20090C284AF0CEE
:01AAD700225C
:0AA268008B108A1189128C138D14DB
:10A2720012BB0178721209D0E47871F612BB01ECBC
:10A28200C0E0EDC0E0EEC0E0EFC0E0787212095F1E
:10A29200CBEFCBCAEECAC9EDC9C8ECC8D0E0FFD03B
:10A2A200E0FED0E0FDD0E0FCC3EF9BFFEE9AFEEDB6
:10A2B20099FDEC98FCE47B01FAF9F8C31208D1503D
:10A2C200037F00227876E6FED39400405390198EE5
:10A2D200E0FDB478037F0122ED54F8647860037FD7
:10A2E200002290198EE0540724027871F66E7030C5
:10A2F2007876E6D39514E5136480F8748098400666
:10A30200AE13AF1480067876E6FF7E00A812AC1179
:10A31200AD107B017A19798E1206EE7871E6FF2272
:08A322007F0112B89902A27E2E
:07000300E47876F6D2362204
:10B49800EF7025F5847598D0F584759115F5847548
:10B4A800C90875CBFFED9098BC93F5CA75C804E43C
:10B4B800F584D2ACC2BC80267584017598D0E4F5B9
:10B4C80084E589540F4420F589758E02ED9098C65D
:10B4D80093F58DD28E43E74043F740120003D2AF75
:01B4E8002241
:10AFEC009019CE120A01000000009019D2120A0129
:10AFFC00000000009019857464F0E478A8F678A835
:10B00C00E6FFC394025043EF25E025E02486F58249
:10B01C00E43419F583E4F0EF25E025E02487F5828C
:10B02C00E43419F583E4F0EF25E025E02488F5827B
:10B03C00E43419F583E4F0EF25E025E02489F5826A
:0AB04C00E43419F583E4F00680B443
:01B0560022D7
:10B98B00D2AFD2A9C2BBE4F584E589540F4401F5CB
:0FB99B0089758E02758CAFE4F58AD28C02AFEC01
:029D14001570C8
:109D1600A870E4F6A870E6FFC394024003029E030F
:109D2600EF25E025E02489F582E43419F583E0FF88
:109D3600D394005003029DD8E625E025E02487F55C
:109D460082E43419F583E06003029DD8EF30E01910
:109D5600E6FF25E025E02489F582E43419F583E061
:109D6600D3940140047D0080067D01A870E6FF12B1
:109D7600AF12A870E6FF25E025E02489F582E434D9
:109D860019F583E0B401057D0112AF12A870E6FF54
:109D960025E025E02489F582E43419F583E014F002
:109DA600EF25E025E02489F582E43419F583E060A7
:109DB60021E6FF25E025E02488F582E43419F583C1
:109DC600E0FEEF25E025E02487F582E43419F583EB
:109DD600EEF0A870E6FF25E025E02487F582E4345E
:109DE60019F583E06011EF25E025E02487F582E48C
:0D9DF6003419F583E014F0A87006029D1AE0
:039E0300057022C5
:03000B0002A9192E
:10A91900C0E0C0F0C083C082C0D0E8C0E0E9C0E0B8
:10A92900EAC0E0EBC0E0ECC0E0EDC0E0EEC0E0EF73
:10A93900C0E0758CAF9019CEE0FCA3E0FDA3E0FE6A
:10A94900A3E02401FFE43EFEE43DFDE43CFC901954
:10A95900CE1209DC901985E014F0E070259019D227
:10A96900E0FCA3E0FDA3E0FEA3E02401FFE43EFE3A
:10A97900E43DFDE43CFC9019D21209DC9019857480
:10A9890064F0129D1412B969D0E0FFD0E0FED0E066
:10A99900FDD0E0FCD0E0FBD0E0FAD0E0F9D0E0F85F
:0BA9A900D0D0D082D083D0F0D0E032BC
:10B86C001570A870EDF61570A870EFF6A870E6FFCD
:10B87C00C39402501308E6FEEF25E025E02486F57C
:0DB88C0082E43419F583EEF005700570229A
:10AAD80015701570A870EAF608EBF61570A870EDF9
:10AAE800F61570A870EFF6A870E6FFC39402506AD6
:10AAF800EF25E025E02489F582E43419F583E07038
:10AB080059E6FB25E025E02487F582E43419F5832E
:10AB1800E0704708E625E004FFA870E6FA25E0257E
:10AB2800E02489F582E43419F583EFF00808E6FE9D
:10AB380008E6FF7C007D0A1207F5EA25E025E024F7
:10AB480088F582E43419F583EFF0EB25E025E0245D
:10AB580087F582E43419F583E4F0E5702404F57090
:01AB680022CA
:0EAF12001570A870EDF61570A870EFF61570AA
:10AF2000A87008E6FFC394025024EF25E025E02432
:10AF300086F582E43419F583E06013A8700808E60A
:10AF400070047F0180027F00A8700808EFF6A870E7
:10AF5000A68475840FA87008E6FF700BA870080817
:10AF6000E624FF9286800DEFB40109A8700808E678
:09AF700024FF9287A870E6F58425
:07AF79000570057005702250
:10BB0100C2AF9019CEE0FCA3E0FDA3E0FEA3E0FFED
:02BB1100D2AFB1
:01BB1300220F
:10BB1400C2AF9019D2E0FCA3E0FDA3E0FEA3E0FFD6
:02BB2400D2AF9E
:01BB260022FC
:10B899001570A870EFF6A870E670057878F608F6C6
:10B8A9003035167877E675F064A4FFC37879E69F9A
:0CB8B90018E695F0500375FFA5057022FD
:10B9AA00D235E47878F608F6EF78776003F6800205
:0FB9BA00760A75FF0775FFA5E4F58475EF042283
:10BB2700C235E47878F608F6787776FF75FFDE7524
:03BB3700FFAD223D
:10B96900787906E6187001063035167877E675F0AD
:10B9790064A4FFC37879E69F18E695F0500375FF34
:02B98900A522F5
:04B8C5008E448F45D9
:10B8C900E4F546F547C3E5479545E54695445016E1
:10B8D9007FE87E0312B2417F0112B8990547E54717
:06B8E90070E3054680DF5C
:01B8EF002236
:04B241008E658F6621
:10B24500D3E56694FAE56594005010AF66EFD394A4
:10B255000040407E1600DEFD1F80F285656785662D
:10B2650068D3E56894FAE567940040157FFA7E0097
:10B2750012B24174062568F56874FF3567F5678075
:10B28500E0D3E5669400E56594004007AF68AE67D6
:03B2950012B241B1
:01B298002293
:10B0C20075500075510075524A7B007A0079487DAF
:01B0D200027B
:08B0D3008B4C8A4D894E8D4F14
:10B0DB007F0112B899AB50AA51A95212082B240028
:10B0EB00FFE5F034E0FE854C53854D54854E55E419
:10B0FB00FDEDC3954F501BEF2DF582E43EF583E438
:10B10B0093AB53AA54A9558D8275830012076C0D0E
:0FB11B0080DFAB50AA51A952E4854FF0020856CD
:10A3EB00754112754234754900754A00754B437BB4
:07A3FB00007A0079417D02A8
:08A402008B458A4689478D480D
:10A40A007880E664F1600302A49F12BB27C2AFE41E
:10A41A00F58443B701758F01AB49AA4AA94B1208C3
:10A42A002B2400FFE5F034E078A8F608EFF6AA46F8
:10A43A00A94778ACA64508C6EAC608C6E9C6E478BC
:10A44A00AAF678AAE6C39548503278ACCBE6CB0890
:10A45A000806E618CAE6CA70010614F91207147843
:10A46A00ABF6E6FF78A80806E618CCE6CC7001063B
:10A47A0014F5828C83EFF078AA0680C6E4F58F5330
:10A48A00B7F0AB49AA4AA94B8548F0120856D2AF91
:05A49A00E4FF12B9AA65
:01A49F00229A
:10B539007880E664F17046C2AF12BB27E4F5844314
:10B54900B701758F0378A976E008F678A8F678A987
:10B55900E6FE08E6F5828E83E4F07F0112B8997859
:10B56900AAE426F618740236F61806E6C3940840CB
:0DB57900DDE4F58F53B7F0D2AFFF12B9AA91
:01B5860022A2
:10A6A20012B539E4F543F544F549754A00754B4353
:10A6B200FB7A00798D7D1612A40212A3EBE4F54019
:10A6C200E540C3787D965073E4F53FAB1DAA1EA901
:10A6D2001F75F01DE53FA4F58285F08312072D60FA
:10A6E20056E53F75F01DA429F9EA35F0FA90000D00
:10A6F200120A6D788AE68540F0A429F9EA35F0FA63
:10A70200EBC0E0EAC0E0E9C0E0AB1DAA1EA91F75DC
:10A71200F01DE53FA4F58285F08312072DFD7549F2
:10A7220000754A00754B43D0E0F9D0E0FAD0E0FB67
:10A7320012A402053F80940540808512A3EBE478C1
:02A7420080F69F
:01A7440022F2
:029E06008F4487
:109E0800E4F54AF54BF547F55075510075524AFB94
:109E18007A00798D7D1612B0D312B0C2E549643448
:109E28007004E54864127003434701E4F546E546CB
:109E3800C3787D964003029ED9E4F545AB1DAA1E62
:109E4800A91F75F01DE545A4F58285F08312072D3D
:109E5800607AE5446054E54575F01DA429F9EA35B2
:109E6800F0FA90000D120A6D788AE68546F0A4296A
:109E7800F9EA35F0FAEBC0E0EAC0E0E9C0E0AB1D72
:109E8800AA1EA91F75F01DE545A4F58285F0831269
:109E9800072DFD75500075510075524AD0E0F9D074
:109EA800E0FAD0E0FB12B0D3801DAB1DAA1EA91F9B
:109EB80075F01DE545A4F58285F08312072D254B25
:109EC800F54BE4354AF54A0545029E440546029E8F
:109ED8003612B0C2E54964347004E5486412700370
:059EE800434702AF47F3
:019EED002252
:10B9E700EF540778AAF6EF30E306E64420F6800422
:0CB9F70078AAE6F678AAE644C0F6F5C887
:01BA03002220
:028B37008F4469
:108B390012BB5E7D017F0212BADA7BFF7A977998C0
:108B49001256E9E478A9F612BB27C2AFE478A8F671
:108B590078A8E6FFC395444003028C9A12B9E778D6
:108B6900A8E6FF7D0312BADA7FDA12BA9B902000D9
:108B7900AF82AE83C3EF94FFEE94FF5005E4F0A3F8
:108B890080EE902000AF82AE83C3EF94FFEE94FF96
:108B9900500CE0600678A976018003A380E778A9E4
:108BA900E66003028C9A78A8E6FF7D0312BADA7FA1
:108BB900D912BA9B902000AF82AE83C3EF94FFEE27
:108BC90094FF50067455F0A380ED902000AF82AE5B
:108BD90083C3EF94FFEE94FF500EE064556006786E
:108BE900A976018003A380E578A9E66003028C9A3F
:108BF90078A8E6FF7D0312BADA7FD812BA9B9020D3
:108C090000AF82AE83C3EF94FFEE94FF500674AABF
:108C1900F0A380ED902000AF82AE83C3EF94FFEE06
:108C290094FF500EE064AA600678A976018003A338
:108C390080E578A9E6705A78A8E6FF7D0312BADACA
:108C49007FD712BA9B902000AF82AE83C3EF94FF07
:108C5900EE94FF500674FFF0A380ED902000AF82E0
:108C6900AE83C3EF94FFEE94FF500DE0F4600678F5
:108C7900A976018003A380E678A9E6701478A8E6AE
:108C8900FF7D0312BADA7FD612BA9B78A806028B47
:108C990059D2AFE4FF12B9AA12B9E778A9E6601B65
:108CA9007D02E412BADA7BFF7A9779A778A8E6F50C
:0B8CB900491256E97F0012B89980F9BB
:018CC400228D
:10B05700E4F58475A338F5A275A10475840F759C72
:10B06700FF759DFF759EFF759FFF75F8FF75E8FFDC
:10B0770075D8FF75C8FFFF12B9E7902000E078A8E0
:10B08700F67455F0E064556008E6F0E4F584F5A33E
:10B097002278A8E6F07F0812B9E7E078A8F674AA44
:10B0A700F0E0B4AA0AE6F0E4FF12B9E77F102278CD
:0AB0B700A8E6F0E4FF12B9E77F08F5
:01B0C100226C
:03BB95002020006D
:0AB76B00AB3FAA40A94112072DFFD1
:02B775008F48FB
:10B77700E478ACF6E5481392927F0A7E0012B24154
:10B78700D2937F0A7E0012B241C293E548C313F5F4
:0AB797004878AC06E6C3940840DAD7
:01B7A1002285
:02AE9E008F6EB5
:10AEA000C293E4F58475D2FF75D30F7F0AFE12B208
:10AEB0004175840F43A504AF6E12B77575840F53A7
:10AEC000A5FBD2927F0A7E0012B241E4787BF6188D
:10AED000F6787C7601309207787BE6797C47F6D26B
:10AEE000937F0A7E0012B241C2937F0A7E0012B2A3
:10AEF00041787CE625E0F6787A06E6C3940840D5EA
:10AF0000E4F584F5D2F5D37F0AFE12B241787BE6F0
:01AF1000FF41
:01AF1100221D
:06A18D008B3F8A4089416E
:10A19300C293E4F58475D2FF75D30F7F0AFE12B222
:10A1A3004175840F43A5047FBF12B77575840F53A0
:10A1B300A5FBD2927F0A7E0012B241E478A9F6E4AD
:10A1C30078AAF678A8F678AB760130920778AAE6F3
:10A1D30079AB47F6D2937F0A7E0012B241C2937FD6
:10A1E3000A7E0012B24178ABE625E0F678A806E6CF
:10A1F300C3940840D578A9E6FFC39403501908E631
:10A20300FEEFFDC374059DFDE49400AB3FAA40A996
:10A21300418D82F583801E78A9E6FFC3940550180B
:10A2230008E6FEEF7C0024FDF582EC34FFF583ABFA
:10A233003FAA40A941EE801178A9E6B4060E08E6CC
:10A24300AB3FAA40A94190000212076C78A906E629
:10A25300C39407500302A1C2E4F584F5D2F5D37F7A
:05A263000AFE02B241F9
:10B80B008F468D47C293E4F58475D2FF75D30F7FB6
:10B81B000AFE12B24175840F43A504AF4612B775E9
:10B82B00AF4712B775E4F584F5D2F5D37F0AFE0264
:02B83B00B24118
:10AE28008B3F8A408941C293E4F58475D2FF75D37C
:10AE38000F7F0AFE12B24175840F43A5047FBE122C
:10AE4800B77590000512B76B90000412B76BAB3F53
:10AE5800AA40A94190000312B771AB3FAA40A9418B
:10AE6800120714FF12B775AB3FAA40A94190000121
:10AE780012B7717F0112B775AB3FAA40A941900084
:10AE88000212B771E4FF12B775E4F584F5D2F5D371
:06AE98007F0AFE02B24138
:10B6F8008D6FEF14601614601914601C14601F1409
:10B70800602224057025AD6F7F86801CAD6F7F8811
:10B718008016AD6F7F8C8010AD6F7F84800AAD6F0F
:0CB728007F828004AD6F7F8012B80B227E
:109C0C008B3F8A408941120714FFF47049AB42AA7A
:109C1C0043A944900007743F12076C900006743FF0
:109C2C0012076C900004743F12076C900003743F91
:109C3C0012076C900001743F12076C743F12075AA4
:109C4C00AB42AA43A944900005742D12076C9000F6
:109C5C0002742D029D09EFC4540F2430AB42AA4369
:109C6C00A94412075AAB3FAA40A941120714540F3A
:109C7C002430AB42AA43A94490000112076C900017
:109C8C0002742D12076CAB3FAA40A941900001123F
:109C9C00072DC4540F2430AB42AA43A944900003AF
:109CAC0012076CAB3FAA40A94190000112072D543A
:109CBC000F2430AB42AA43A94490000412076C90C5
:109CCC000005742D12076CAB3FAA40A9419000020D
:109CDC0012072DC4540F2430AB42AA43A944900060
:109CEC000612076CAB3FAA40A94190000212072D47
:109CFC00540F2430AB42AA43A94490000712076CBE
:089D0C00900008E412076C222C
:1099E7008B3F8A408941120714F47049AB42AA435E
:1099F700A944900007743F12076C900006743F1249
:109A0700076C900004743F12076C900003743F12B8
:109A1700076C900001743F12076C743F12075AAB32
:109A270042AA43A944900005743A12076C900002B9
:109A3700743A029AF1AB3FAA40A94190000312077A
:109A47002DC4540F2430AB42AA43A94412075AAB82
:109A57003FAA40A94190000312072D540F2430ABB1
:109A670042AA43A94490000112076C900002743A7D
:109A770012076CAB3FAA40A94190000412072DC4FE
:109A8700540F2430AB42AA43A94490000312076C39
:109A9700AB3FAA40A94190000412072D540F243070
:109AA700AB42AA43A94490000412076C90000574C6
:109AB7003A12076CAB3FAA40A94190000512072D47
:109AC700C4540F2430AB42AA43A94490000612079E
:109AD7006CAB3FAA40A94190000512072D540F24F3
:109AE70030AB42AA43A94490000712076C900008C4
:059AF700E412076C22DF
:10B4E9007B017A1A794012A18D901A40E0F4603FED
:10B4F90075420175431A7544467B017A1A794012DF
:10B509009C0C7B017A1A794612B8F07BFF7ABB79D9
:10B519009512B8F075420175431A7544467B017A54
:0FB529001A79401299E77B017A1A794612B8F025
:01B5380022F0
:10BB3A00E4FF12AE9E787FEFF6F460047F01800284
:02BB4A007F007A
:01BB4C0022D6
:07BB8400E4FD7F8E02B80B07
:106A1700202020202020202020200025622A6264B8
:106A27000025622A62750025622A640025622A759C
:106A37000025622A2E622A660025622A6C640025D8
:106A4700622A6C7500253262753A25730020202072
:106A57002020202020004E6F207661726961626CD1
:106A6700657320646566696E6564002020202020B8
:106A7700202020202020202020202020202000450A
:106A8700534320454E5445522020202D20202020BE
:106A97002B20200045534320454E544552202020AB
:106AA7002D20202020202B200045534320454E54E5
:106AB700455220202000455343202020202020201D
:106AC7002020002020202020002000506172616DCE
:106AD7006574657273207772697474656E00746F7C
:106AE70020666C617368206D656D6F72792E00F496
:106AF70070000000F76E000000FA8F000000FD6DC7
:106B07000000000000000000036B000000064D00BD
:106B1700000009470000000C54000000630000005B
:106B270000016D0000000267000000037300000011
:106B3700046D000000056800000006410000000722
:106B47004B000000088043000009804600001448FD
:106B57007A000015506100001662610000175700A7
:106B67000000185600000019B50000001A54000074
:106B7700001B6C2F73001C52504D001D4600000077
:106B87001E4A0000005A250000005B52504D005C71
:106B9700636E74005D78000000000000000002359D
:106BA7000000004E6F64652041647200008D010093
:106BB700000000000000003F8000000235000000D8
:106BC700477270204164720000008F0100000000CE
:106BD700000000003F8000000A3800000054696D83
:106BE7006500000000011A1C010000000000000001
:106BF700003F8000000A380000004461746500000F
:106C07000000011A0C0100000000000000003F8096
:106C17000000040800000154656D700000000001C9
:106C270019E40200000000000000003F800000049B
:106C370018000001312E3856000000000119FC022F
:106C470000000000000000004000000004180000E1
:106C570001332E3356000000000119E8020000003E
:106C67000000000000400000000418000001355635
:106C77006578740000000119F002000000000000B0
:106C870000004000000004180000013234560000E4
:106C97000000000119F40200000000000000003F9E
:106CA7008000000418000001323456657874000033
:106CB7000119F80200000000000000003F800000FA
:106CC700040600000149203234560000000119EC87
:106CD7000200000000000000004000000000320039
:106CE7000004466C617368000000000000000000AB
:106CF7000000000000000000000000320000045205
:106D070065626F6F74000000000000000000000063
:076D17000000000000000075
:0AB6A600C1A4C12CC12BC125C1268F
:0675BF008B3F8A40894168
:1075C50090000112072D643870598542488543495A
:1075D50085444AF54B754C0A7B017A1A790012B33A
:1075E500F57B017A1A790012BAB1C3EF940AEE94C9
:1075F50000502DE4901A3CF07B017A1A790012BAFA
:10760500B1C3740A9FFFE49EFE901A3CE0C39FE459
:107615009E500D7F2012BA9B901A3CE004F080D852
:1076250002787FE4901A00F0AB3FAA40A941900090
:107635000212072D6068E4901A3CF0901A3CE07540
:10764500F005A424F6F582E4346AF583E493FF6437
:10765500636019AB3FAA40A94190000212072DFEB5
:10766500EF6E6008901A3CE004F080CF901A3CE081
:10767500FF75F005A424F6F582E4346AF583E493F6
:10768500601CEF75F005A424F7F9746A35F07548A8
:10769500FFF549894A7B017A1A790012B2F1AB3FAD
:1076A500AA40A94190000112072D6066E4901A3C9A
:1076B500F0901A3CE075F005A42428F582E4346BBB
:1076C500F583E493FF6019AB3FAA40A941900001FF
:1076D50012072DFEEF6E6008901A3CE004F080D191
:1076E500901A3CE0FF75F005A42428F582E4346B7C
:1076F500F583E493601CEF75F005A42429F9746BF8
:1077050035F07548FFF549894A7B017A1A790012E7
:10771500B2F17B017A1A790012BAB1901A3DEFF0F5
:10772500AB3FAA40A94112071414601D14606424DC
:10773500FE70030277E82404600302787F7BFF7AFA
:107745006A791712B8F002787FAB3FAA40A9419039
:10775500000412072D901A3D30E11CE0FFC3740AA6
:107765009FF549AB42AA43A944120714F54A7BFF8A
:107775007A6A792202787CE0FFC3740A9FF549ABE7
:1077850042AA43A944120714F54A7BFF7A6A79286D
:1077950002787CAB3FAA40A94190000412072D90C6
:1077A5001A3D30E11FE0FFC3740A9FF549AB42AAB9
:1077B50043A94412082BF54B85F04A7BFF7A6A7979
:1077C5002E02787CE0FFC3740A9FF549AB42AA43B9
:1077D500A94412082BF54B85F04A7BFF7A6A793369
:1077E50002787CAB3FAA40A94190000412072D30D6
:1077F500E033901A3DE0FFC3740A9FF549900010ED
:1078050012072DFF600280027F038F4AAB42AA4315
:10781500A9441208F58F4E8E4D8D4C8C4B7BFF7A0B
:107825006A79388052AB3FAA40A9419000041207FB
:107835002D901A3D30E121E0FFC3740A9FF549AB55
:1078450042AA43A9441208F58F4D8E4C8D4B8C4AA4
:107855007BFF7A6A7940801FE0FFC3740A9FF54970
:10786500AB42AA43A9441208F58F4D8E4C8D4B8C23
:107875004A7BFF7A6A79461256E97B017A1A7900C2
:0378850012B8F046
:0178880022DD
:0D324900901A2FE0FBA3E0FAA3E0F97DFF4F
:103256008D428B3F8A40894190000112072D6438C8
:103266007003023A5AAB3FAA40A94112071424FE42
:1032760070030234BB24FE70030237142403600378
:10328600023A5A90000412072D20E103023375AB6F
:103296003FAA40A9419000191209A0C000C001C070
:1032A60002C003AC42EC1203C7D003D002D001D057
:1032B6000012019EC004C005C006C0079019D6E0E2
:1032C600FC1203C7D003D002D001D0001200AD1209
:1032D60003FB9019D6EFF0AB3FAA40A94190001529
:1032E6001209159000111209A01203447003023A44
:1032F6005AAB3FAA40A941900011120915C004C05B
:1033060005C006C0079019D6E0FC1203C7A804A999
:1033160005AA06AB07D007D006D005D00412034491
:103326005014AB3FAA40A94190001112091512038F
:10333600FB9019D6EFF0AB3FAA40A94190001512B9
:103346000915C004C005C006C0079019D6E0FC12D6
:1033560003C7A804A905AA06AB07D007D006D0055F
:10336600D00412034460025003023A5A0234A6E51E
:1033760042F4704CAB3FAA40A941900011120915C6
:10338600C004C005C006C0079019D6E0FCE41203CD
:10339600C7A804A905AA06AB07D007D006D005D052
:1033A60004120344701AAB3FAA40A94190001512BB
:1033B60009159000111209A01203446003023A5A3B
:1033C600AB3FAA40A9419000191209A0C000C00154
:1033D600C002C003AC42EC1203C7D003D002D00136
:1033E600D00012019EC004C005C006C0079019D6C1
:1033F600E0FCE41203C7D003D002D001D0001200D3
:10340600AD1203FB9019D6EFF0AB3FAA40A941904D
:1034160000151209159000111209A0120344700339
:10342600023A5AAB3FAA40A941900011120915C0B1
:1034360004C005C006C0079019D6E0FCE41203C715
:10344600A804A905AA06AB07D007D006D005D00464
:103456001203445014AB3FAA40A94190001112092F
:10346600151203FB9019D6EFF0AB3FAA40A9419085
:103476000015120915C004C005C006C0079019D66C
:10348600E0FCE41203C7A804A905AA06AB07D00707
:10349600D006D005D00412034460025003023A5A03
:1034A600AB3FAA40A9419000151209151203FB90E3
:1034B60019D6EFF022AB3FAA40A9419000041207AB
:1034C6002D20E1030235B99000191209A0C000C0F1
:1034D60001C002C003AC42EC1203C7D003D002D035
:1034E60001D00012019EC004C005C006C007901995
:1034F600D6E0FCA3E0FDEC1203C2D003D002D0015B
:10350600D0001200AD1203FB9019D6EEF0A3EFF037
:10351600AB3FAA40A941900015120915900011125F
:1035260009A01203447003023A5AAB3FAA40A941CC
:10353600900011120915C004C005C006C0079019F5
:10354600D6E0FCA3E0FDEC1203C2A804A905AA0676
:10355600AB07D007D006D005D0041203445017ABF2
:103566003FAA40A9419000111209151203FB9019B8
:10357600D6EEF0A3EFF0AB3FAA40A941900015129A
:103586000915C004C005C006C0079019D6E0FCA303
:10359600E0FDEC1203C2A804A905AA06AB07D007F2
:1035A600D006D005D00412034460025003023A5AF2
:1035B6000236FCE542F4704FAB3FAA40A9419000A9
:1035C60011120915C004C005C006C0079019D6E03F
:1035D600FCA3E0FDE41203C2A804A905AA06AB07F2
:1035E600D007D006D005D004120344701AAB3FAA08
:1035F60040A9419000151209159000111209A01258
:1036060003446003023A5AAB3FAA40A9419000190D
:103616001209A0C000C001C002C003AC42EC1203F4
:10362600C7D003D002D001D00012019EC004C0054D
:10363600C006C0079019D6E0FCA3E0FDE41203C261
:10364600D003D002D001D0001200AD1203FB9019B6
:10365600D6EEF0A3EFF0AB3FAA40A94190001512B9
:1036660009159000111209A01203447003023A5A78
:10367600AB3FAA40A941900011120915C004C0052C
:10368600C006C0079019D6E0FCA3E0FDE41203C211
:10369600A804A905AA06AB07D007D006D005D00412
:1036A6001203445017AB3FAA40A9419000111209DA
:1036B600151203FB9019D6EEF0A3EFF0AB3FAA402C
:1036C600A941900015120915C004C005C006C0071F
:1036D6009019D6E0FCA3E0FDE41203C2A804A905F4
:1036E600AA06AB07D007D006D005D0041203446063
:1036F600025003023A5AAB3FAA40A9419000151264
:1037060009151203FB9019D6EEF0A3EFF022AB3F9A
:10371600AA40A94190000412072D20E0030237D6E3
:103726009019D6E0F8A3E0F9A3E0FAA3E0FBC00005
:10373600C001C002C003AB3FAA40A94190001912C4
:1037460009A0C000C001C002C003AC42EC1203C70E
:10375600D003D002D001D00012019ED003D002D0F7
:1037660001D0001200AD9019D61209DCAB3FAA4079
:10377600A9419000111209159019D6E0F8A3E0F9B5
:10378600A3E0FAA3E0FB1203445012AB3FAA40A900
:10379600419000111209159019D61209DCAB3FAA07
:1037A60040A9419000151209159019D6E0F8A3E03A
:1037B600F9A3E0FAA3E0FB12034460025003023AC5
:1037C6005AAB3FAA40A941900015120915023A5476
:1037D600AB3FAA40A94190000412072D20E1030245
:1037E60038F19000191209A0C000C001C002C00340
:1037F600AC42EC1203C7D003D002D001D0001201B4
:103806009EC004C005C006C0079019D6E0FCA3E020
:10381600FDA3E0FEA3E0FFEC1203BDD003D002D06F
:1038260001D0001200AD1203FB9019D61209DCABD1
:103836003FAA40A9419000151209159000111209DE
:10384600A01203447003023A5AAB3FAA40A9419022
:103856000011120915C004C005C006C0079019D68C
:10386600E0FCA3E0FDA3E0FEA3E0FFEC1203BDA88D
:1038760004A905AA06AB07D007D006D005D00412C6
:1038860003445015AB3FAA40A941900011120915F7
:103896001203FB9019D61209DCAB3FAA40A941904E
:1038A6000015120915C004C005C006C0079019D638
:1038B600E0FCA3E0FDA3E0FEA3E0FFEC1203BDA83D
:1038C60004A905AA06AB07D007D006D005D0041276
:1038D600034460025003023A5AAB3FAA40A9419002
:1038E60000151209151203FB023A54E542F470550D
:1038F600AB3FAA40A941900011120915C004C005AA
:10390600C006C0079019D6E0FCA3E0FDA3E0FEA325
:10391600E0FFE41203BDA804A905AA06AB07D00779
:10392600D006D005D004120344701AAB3FAA40A9B2
:10393600419000151209159000111209A0120344B6
:103946006003023A5AAB3FAA40A9419000191209F6
:10395600A0C000C001C002C003AC42EC1203C7D035
:1039660003D002D001D00012019EC004C005C006DB
:10397600C0079019D6E0FCA3E0FDA3E0FEA3E0FF9C
:10398600E41203BDD003D002D001D0001200AD1264
:1039960003FB9019D61209DCAB3FAA40A94190005F
:1039A600151209159000111209A0120344700302A2
:1039B6003A5AAB3FAA40A941900011120915C0041A
:1039C600C005C006C0079019D6E0FCA3E0FDA3E041
:1039D600FEA3E0FFE41203BDA804A905AA06AB07EF
:1039E600D007D006D005D0041203445015AB3FAA29
:1039F60040A9419000111209151203FB9019D61225
:103A060009DCAB3FAA40A941900015120915C00474
:103A1600C005C006C0079019D6E0FCA3E0FDA3E0F0
:103A2600FEA3E0FFE41203BDA804A905AA06AB079E
:103A3600D007D006D005D00412034460174015AB5A
:103A46003FAA40A9419000151209151203FB9019CF
:053A5600D61209DC227C
:10B6B1008F3FE92405F9E43AFA78007C1A7D017E8E
:10B6C100007F081206EEE4901A08F0901A06E0FFD7
:10B6D1006007901A05F0E4A3F0853F49754A0175AA
:10B6E1004B1A754C007BFF7A6A794C1256E97BFF45
:07B6F1007A6A795402B8F0F7
:100BF400127889EF6003D22422302440E49019E370
:100C0400F09019DB120A01000000009019DF120AAB
:100C14000100000000C227C228C229C22AE4901A97
:100C240035F012BB01E47B2C7A01F9F8C31208D128
:100C340040030216BEC224D219125AF6202C1EC238
:100C440019125AF6901A35EFF070030216AED22C30
:100C5400E0640260030216AED22B0216AE202B0310
:100C640002102B901A0C742DF0E4A3F0901A1C744B
:100C74002DF0E4A3F075420175431A7544367545A9
:100C840002FB7D02FF12965D901A36E0C4F854F020
:100C9400C868FCA3E0C4540F48FDE41203C2E4FB9B
:100CA400FAF978411202A7901A381209DCE4FFFE1F
:100CB4007D207C41901A38E0F8A3E0F9A3E0FAA380
:100CC400E0FB12019EE4FBFAF9783F1200AD120337
:100CD400FBEC1203BDE4FBFA792078411202A790E1
:100CE40019E41209DC75420175431A7544367545D9
:100CF400027B017D02E4FF12965D901A36E0C4F88F
:100D040054F0C868FCA3E0C4540F48FDE41203C2C5
:100D1400E4FBFA79A0784012019EE4FBFA7980782A
:100D2400451202A7901A381209DCE4FFFE7DC87C44
:100D340042901A38E0F8A3E0F9A3E0FAA3E0FB122A
:100D4400019EE4FBFAF9783F1200AD1203FBEC12AA
:100D540003BDE4FBFA79C878421202A79019E8129D
:100D640009DC75420175431A7544367545027B02E8
:100D74007D02E4FF12965D901A36E0C4F854F0C880
:100D840068FCA3E0C4540F48FDE41203C2E4FBFA78
:100D94007920784012019EE4FBFA798078451202AA
:100DA400A7901A381209DC901A38E0FCA3E0FDA3DE
:100DB400E0FEA3E0FF7B007AC0792878451202A701
:100DC400901A381209DC901A38E0FCA3E0FDA3E085
:100DD400FEA3E0FF7B007AC0795A784612019E9008
:100DE4001A381209DCE4FFFE7DC87C42901A38E010
:100DF400F8A3E0F9A3E0FAA3E0FB12019EE4FBFAF6
:100E0400F9783F1200AD1203FBEC1203BDE4FBFAC8
:100E140079C878421202A79019EC1209DC754201D4
:100E240075431A7544367545027B037D02E4FF124F
:100E3400965D901A36E0C4F854F0C868FCA3E0C488
:100E4400540F48FDE41203C2E4FBFA79C878401257
:100E5400019EE4FBFA798078451202A7901A3812B1
:100E640009DCE4FFFE7DC87C42901A38E0F8A3E078
:100E7400F9A3E0FAA3E0FB12019EE4FBFAF9783F40
:100E84001200AD1203FBEC1203BDE4FBFA79C8783F
:100E9400421202A79019F01209DC75420175431A37
:100EA4007544367545027B047D02E4FF12965D901D
:100EB4001A36E0C4F854F0C868FEA3E0C4540F48DE
:100EC400FF7C007D0B12078EAC06AD07E41203C253
:100ED400E4FBFA7920784012019EE4FBFA798078E9
:100EE400451202A7901A381209DCE4FFFE7DC87C83
:100EF40042901A38E0F8A3E0F9A3E0FAA3E0FB1269
:100F0400019EE4FBFAF9783F1200AD1203FBEC12E8
:100F140003BDE4FBFA79C878421202A79019F412CF
:100F240009DC75420175431A7544367545027B0523
:100F34007D02E4FF12965D901A36E0C4F854F0C8BE
:100F440068FEA3E0C4540F48FF7C007D0B12078E9B
:100F5400AC06AD07E41203C2E4FBFA792078401230
:100F6400019EE4FBFA798078451202A7901A3812A0
:100F740009DCE4FFFE7DC87C42901A38E0F8A3E067
:100F8400F9A3E0FAA3E0FB12019EE4FBFAF9783F2F
:100F94001200AD1203FBEC1203BDE4FBFA79C8782E
:100FA400421202A79019F81209DC75420175431A1E
:100FB4007544367545027B067D02E4FF12965D900A
:100FC4001A36E0C4F854F0C868FCA3E0C4540F48CF
:100FD400FDE41203C2E4FBFA7920784012019EE496
:100FE400FBFA798078451202A7901A381209DCE4DA
:100FF400FFFE7DC87C42901A38E0F8A3E0F9A3E034
:10100400FAA3E0FB12019EE4FBFAF9783F1200AD6B
:101014001203FBEC1203BDE4FBFA79C87842120216
:10102400A79019FC1209DC901A2F302B1374FFF0CF
:10103400A3746BF0A374A5F0901A33740CF08013AE
:10104400E51DF0A3E51EF0A3E51FF07882E61490F9
:101054001A33F0901A33E0FFC394035005E4A3F06D
:10106400801B9019E3E0FE7002800EEE9019E3B548
:101074000705E024FE8002E014901A34F07882E63A
:101084007014202B11FDFF12BADA7BFF7A6A795DA6
:101094001256E90211D4E4901A32F0901A32E0FDAB
:1010A400C3940340030211D4E4FF12BADA901A3253
:1010B400E0FF901A34E02FFFE433FE9019E3E07C64
:1010C40000B50708ECB506047F1580027F2012BA2C
:1010D4009B901A32E0FD7F0112BADA901A32E0FFD7
:1010E400901A34E02FFFE433FE901A33E0FDD3EF7F
:1010F4009D7480F86E98400C7BFF7A6A7972125660
:10110400E90211CB901A32E0FF901A34E02FFFE489
:1011140033FE7C007D1D12078E901A2FE0FBA3E0A6
:10112400FAA3E02FF9EA3EFAA3E0FF901A34E02F85
:10113400FF12B6B1901A32E0FD7F0A12BADA3025F6
:101144003A901A32E0FF901A34E02FFFE433FE9015
:1011540019E3E07C00B50723ECB5061F7D1D1207DB
:101164008E901A2FE0FBA3E0FAA3E02FF9EA3EFAEF
:101174007542017543197544D68049901A32E0FFCF
:10118400901A34E02FFFE433FE7C007D1D12078E9D
:10119400901A2FE0FBA3E0FAA3E02FF9EA3EFAC08D
:1011A40003C002C001901A2FA3E0FAA3E02FF9EACA
:1011B4003EFA90000D120A6D8B428A438944D00195
:1011C400D002D0031275BF901A32E004F002109FCF
:1011D4009019E3E075F01DA4302B0F24A5F9746B6E
:1011E40035F0FA901A2F74FF800D251FF9E51E358E
:1011F400F0FA901A2FE51DF0A3EAF0A3E9F03026E7
:101204005A7D03E4FF12BADA7BFF7A6A798612B850
:10121400F09019DAE075F003A4240DFF901A34E07D
:10122400FE9019E3E0C39EFD12BADA200A0A3027C1
:1012340007C226E4FF12BB4D200B030216AE302872
:10124400030216AE9019DAE004F0E06403600302CE
:1012540016AEC226FF12BB4D0216AE2025030214A1
:10126400237D03E4FF12BADA7BFF7A6A799B12B812
:10127400F0901A34E0FF9019E3E0C39FFD7F13124E
:10128400BADA200A0A302707C225E4FF12BB4D3020
:101294000B53202850C225E4FF12BB4D901A2FE0B7
:1012A400FBA3E0FAA3E0F9120714FF7E00901A2FC3
:1012B400A3A3E090000D120A6DA801AC02AD037B5C
:1012C400017A1979D61206EE302B129019E3E0FF59
:1012D4006003B40110D22D788076F180089019E370
:1012E400E0FF12B83D300C0F20290C12324912BB1A
:1012F400019019DB1209DC300C2D12BB01A804A9E2
:1013040005AA06AB079019DBE0FCA3E0FDA3E0FE11
:10131400A3E02446FFE43EFEE43DFDE43CFCD3129E
:1013240008D14003123249300C3B12BB01A804A976
:1013340005AA06AB079019DBE0FCA3E0FDA3E0FEE1
:10134400A3E024F4FFEE3401FEE43DFDE43CFCD3D1
:101354001208D14010901A2FE0FBA3E0FAA3E0F9A1
:101364007DF7123256200C0A9019DB120A01000094
:101374000000300D1C202A19901A2FE0FBA3E0FA7C
:10138400A3E0F97D0112325612BB019019DF120954
:10139400DC300D3A12BB01A804A905AA06AB0790DC
:1013A40019DFE0FCA3E0FDA3E0FEA3E02446FFE494
:1013B4003EFEE43DFDE43CFCD31208D14010901AFB
:1013C4002FE0FBA3E0FAA3E0F97D01123256300DC1
:1013D4003B12BB01A804A905AA06AB079019DFE0DC
:1013E400FCA3E0FDA3E0FEA3E024F4FFEE3401FE41
:1013F400E43DFDE43CFCD31208D14010901A2FE0E8
:10140400FBA3E0FAA3E0F97D09123256300D030282
:1014140016AE9019DF120A01000000000216AE7D1C
:1014240003E4FF12BADA7882E6D394005003302B37
:1014340037901A2FE0FBA3E0FAA3E0F99000191209
:101444000915E4FBFAF9F81203444014901A2FE04A
:10145400FBA3E0FAA3E0F990000412072D30E208A0
:101464007BFF7A6A79B080067BFF7A6A79BD12B80D
:10147400F07F1212BA9B7BFF7A6A79CA12B8F07FA6
:101484001312BA9B7BFF7A6A79D012B8F0200A0C47
:10149400302709C22CC22BD219125AF6200B030290
:1014A400158C30280302158C7882E6D394004061B1
:1014B400901A2FE0FBA3E0FAA3E0F9120714FFD37C
:1014C4009404504DEF94004048900019120915E41B
:1014D400FBFAF9F81203445038D225901A2FE0FB96
:1014E400A3E0FAA3E0F9120714FF7E0090000D12A6
:1014F4000A6D78D67C197D011206EE901A34E0FF4D
:101504009019E3E0C39FFD7F1312BADA7F0112BB87
:101514004D302B2A9019E3E0FF64026004EFB4031A
:101524001DD226E49019DAF0901A34E0FF9019E302
:10153400E0C39FFD7F0D12BADA7F0112BB4D302B41
:10154400379019E3E0640B702FD22D788076F11276
:10155400BB5EE4FDFF12BADA7BFF7A6A79D212B875
:10156400F07D01E4FF12BADA7BFF7A6A79E512B8FA
:10157400F07FB87E0B12B8C5302B0D9019E3E0B4A0
:101584000C06E4F58475EF10300C2A2029279019F5
:10159400E3E07012202B077882E614F0800E901995
:1015A400E3740CF080069019E3E014F012BB019090
:1015B40019DB1209DC300C4812BB01A804A905AAE6
:1015C40006AB079019DBE0FCA3E0FDA3E0FEA3E07B
:1015D4002446FFE43EFEE43DFDE43CFCD31208D186
:1015E400401E9019E3E07012202B077882E614F075
:1015F400800E9019E3740CF080069019E3E014F067
:10160400200C0A9019DB120A0100000000302B089C
:10161400901A32740DF080077882E6901A32F03016
:101624000D25202A229019E3E02401FFE433FE90E3
:101634001A32E0FD7C001207A09019E3EDF012BB12
:10164400019019DF1209DC300D4312BB01A804A973
:1016540005AA06AB079019DFE0FCA3E0FDA3E0FEBA
:10166400A3E02446FFE43EFEE43DFDE43CFCD3124B
:1016740008D140199019E3E02401FFE433FE901AE5
:1016840032E0FD7C001207A09019E3EDF0200D0A72
:101694009019DF120A0100000000300C0D300D0A11
:1016A400202B07E49019E3F0D22BA20A9227A20B75
:0A16B4009228A20C9229A20D922A9E
:0116BE002209
:04965D008D408B4170
:109661007B08E4FD12BA95E4901A44F0E5405408F1
:10967100D394004003D38001C392B30000000000E3
:10968100000000000000000000000000000000D207
:10969100B000000000000000000000000000000019
:1096A1000000000000C2B0E54025E0F540901A44FA
:1096B100E004F0E0B404B5E4901A44F0E541540844
:1096C100D394004003D38001C392B3000000000093
:1096D100000000000000000000000000000000D2B7
:1096E100B0000000000000000000000000000000C9
:1096F1000000000000C2B0E54125E0F541901A44A8
:10970100E004F0E0B404B5E4901A44F0E54575F0E6
:1097110008A4FF901A44E0FDC39FE5F06480F8744B
:109721008098505CED9400400FE05407700A0425C6
:1097310044F544E43543F543C2B0000000000000A5
:109741000000000000000000000000000000AB422B
:10975100AA43A94412071425E0FFA2B4E4334F122F
:10976100075AD2B000000000000000000000000015
:109771000000000000000000901A44E004F0808C1A
:10978100D2B2000000000000000000000000000054
:06979100000000000000D2
:0197970022AF
:04A0B1007D0AAF4530
:04A0B5008D468B4702
:10A0B900D2B2000000000000000000000000000013
:10A0C900000000000000C2B2000000000000000013
:10A0D9000000000000000000000000007B08E4FD13
:10A0E90012BA95E4901A44F0E5465408D394004016
:10A0F90003D38001C392B3000000000000000000F8
:10A109000000000000000000000000D2B0000000C4
:10A119000000000000000000000000000000000036
:10A1290000C2B0E54625E0F546901A44E004F0E0A7
:10A13900B404B5E4901A44F0E5475408D3940040B8
:10A1490003D38001C392B3000000000000000000A7
:10A159000000000000000000000000D2B000000074
:10A1690000000000000000000000000000000000E6
:10A1790000C2B0E54725E0F547901A44E004F0E055
:03A18900B404B566
:01A18C0022B0
:10B58700E4901A2DF0EF5480D394004003D3800148
:10B59700C392B3000000000000000000000000009C
:10B5A70000000000000000D2B00000000000000012
:10B5B70000000000000000000000000000C2B0EF23
:0DB5C70025E0FF901A2DE004F0E0B408B874
:01B5D4002254
:02A32A008F455D
:10A32C00E4FB7D0712A0B5E4FB12A0B1E4FF12B56B
:10A33C0087E4FF12B5877B0212A0B1E4FF12B58748
:10A34C00E4FF12B587E4901A2AF0901A2AE0FBC3B6
:10A35C00940750697D0CAF4512A0B5901A2AE0FF06
:10A36C00700AA37403F0A37420F08017EF901A2BDB
:10A37C00B402097401F0A374D9F08007740FF0A330
:10A38C0074FFF0901A2BE0C4F854F0C8A3E0C45446
:10A39C000F48FF12B587901A2CE0540FC4F8540FD5
:10A3AC00C868FF12B587E4FF12B587E4FF12B587C2
:10A3BC007F3A12B587901A2AE004F0808DE4FB7D79
:10A3CC000DAF4512A0B57FFF12B5877FFF12B58781
:0FA3DC00E4FF12B587E4FF12B5877F1402B5873F
:10B9C900E4FB7D0912A0B5D2B2000000000000001E
:0EB9D90000000000000000000000000000223E
:04B91A008F468D4780
:10B91E007B017A1A792F12A9B4E547901A2F600687
:10B92E00E04401F08004E054FEF0901A2FE0FDAFE9
:04B93E004602AD9E72
:10BA6D007B017A1A792AE4FF12A9B4901A2AE030E0
:07BA7D00E7037F00227F01B7
:01BA8400229F
:10BA54007B017A1A792FE4FF12A9B4901A2FE030EF
:08BA6400E704540FFF227F00EC
:01BA6C0022B7
:10BA20007B017A1A792F12A9B4901A2FE0FFF460E3
:0ABA300007EF60047F0180027F0031
:01BA3A0022E9
:02B299008F63C1
:10B29B0075840FE4F5A6C290C294D295D2967F0125
:10B2AB00FE12B241C296E4F5647F0A7E0012B241EF
:10B2BB0030A7090564E564C394C840ED75840F7528
:10B2CB00A6FFD290C295A22392948563A07F017EA4
:10B2DB000012B241D2967F017E0012B241C2967F1C
:06B2EB00017E0002B241E9
:10AF8000D23775840F43A580C2977F017E0012B827
:10AF9000C5D2977F327E0012B8C5C296C295C294C0
:10AFA00075840F75A6FF43A503D290D291C2237F6B
:10AFB0003412B299C2237F0B12B299C2237F30128E
:10AFC000B299C2237F0212B299C2237F0C12B299A6
:10AFD000C2237F0112B299C2237F3412B299C223D5
:0CAFE0007F0612B299C2237F3002B299A2
:0DBB5E00C2237F0112B299E4FDFF02BADAA2
:10BB4D00EF6006C2237F0F8004C2237F0C12B299CF
:01BB5D0022C5
:10BADA00ED5403C43354E0FEEF541F44804EFFC2BA
:04BAEA002302B299E8
:10BA9B008F62E562640D600BE562640A6005D22378
:06BAAB0012B299AF622205
:10B942008B698A6A896BAB69AA6AA96B1207146050
:10B9520015056BE56B7002056A14F9120714FFD224
:07B962002312B29980E022DC
:1000A600020467E86480F8E933E83360110460F01D
:1000B600ED33EC337009E8FCE9FDEAFEEBFF2204C0
:1000C60060DED3EB9FEA9EE99DE8C2E78CF0C2F7BB
:1000D60095F0400CE8CCF8E9CDF9EACEFAEBCFFB87
:1000E60012043285D0F05804700320D5B3E80470AA
:1000F600075002B2D502047192D5EC0460F7E4CC45
:10010600C0E0C398F8603B94186008400DD0E0FB4F
:10011600020449E4FBFAC9FC8028E830E406E4C995
:10012600FBE4CAFCE830E305E4C9CACBFCE85407A3
:100136006010F8C3E913F9EA13FAEB13FBEC13FCAE
:10014600D8F130F52FC3E49CFCEF9BFFEE9AFEED51
:1001560099FDD0E0FBEF4E4D4C701222DB030204FA
:100166006EEC2CFCEF33FFEE33FEED33FDED30E7A6
:10017600EB020449EF2BFFEE3AFEED39FDD0E0FB32
:1001860050130BBB0003020471ED13FDEE13FEEFDB
:0801960013FFEC13FC02044905
:10019E00EC4D6011E8497017ED33EC3304600DE45B
:1001AE00FCFFFEFD22E933E8330470F80204671207
:1001BE00043258046009E4CC248150062850090208
:1001CE00047128400302046EC0E0EB4A7044B9800B
:1001DE0006D0E0FB02045DEF4E701CBD8008EBFF05
:1001EE00EAFEE9FD80EBE98DF0A4FEE5F002028760
:1001FE00E9CDF9EAFEEBFFEF89F0A4FCE5F0CE893C
:10020E00F0A42EFFE435F0CD89F0A42DFEE435F0F8
:10021E008067EF4E7005BD80D780C3EF8BF0A4AC26
:10022E00F0EE8BF0A42CFCE435F0F8EF8AF0A42C61
:10023E00E5F038FCE433CB8DF0A42CFCE5F03BF874
:10024E00EE8AF0A42CFCE5F038F8E433CF89F0A464
:10025E002CFCE5F038CF3400CE89F0A42FFFE5F06A
:10026E003EFEE433C98DF0A42EFEE5F039CD8AF0C2
:10027E00A42FFFE5F03EFEE43DFD33D0E0FB50073A
:10028E000BBB000F020471EC2CFCEF33FFEE33FEC0
:06029E00ED33FD020449EE
:1002A400020471EC5D046005E859047003020467FC
:1002B400120432580460F6EC4860F2EC7004FDFE5F
:1002C400FF22C860DB2481C85009C398600250062D
:1002D40002046E9850CAF582E9294B4A7005AB8234
:1002E40002045D75F0007C1A7880C3EF9BEE9AEDF2
:1002F40099400DC3EF9BFFEE9AFEED99FDE842F0A5
:10030400DC23ACF0D0E0FFD0E0FED0E0FDAB8220F7
:10031400E7101BEB60BAEC2CFCEF33FFEE33FEED81
:1003240033FD020449E803F830E705C0F075F00036
:10033400EF2FFFEE33FEED33FD40B830E7C280AA65
:1003440074F8CC6480CCC86480C8F58204604FC360
:10035400EB9FF5F0EA9E42F0E99D42F0E89C45F0FF
:10036400603C501DE5825FFFE582D313CB5BCBF489
:100374002B5582FB50280ABA002409B900200880B2
:100384001DE5825BFBE582D313CF5FCFF4C3132F4C
:100394005582FF50090EBE00050DBD00010CC3EBD4
:1003A4009FF5F0EA9E42F0E99D42F0E89C45F0603A
:0903B40007CC4820E701B3EC225C
:1003BD0075F020800E75F010800575F0087D007EBB
:1003CD00007F003392D530D5031208ADEC334010C9
:1003DD00EF33FFEE33FEED33FDEC33FCD5F0ED22C4
:0E03ED00E5F0247EA2D513CC92E7CDCEFF2200
:1003FB00EDD2E7CD33EC3392D524814006E4FFFEFA
:10040B00FDFC22FCE4CFCECDCC24E0501174FF8058
:10041B00EDC3CC13CCCD13CDCE13CECF13CF0470F5
:07042B00F030D5DE0208AD40
:10568700E55D2449F8E6055D227846302102784930
:10569700E475F001120A5D020714201AEB7F2ED27F
:1056A7001A8018EF540F2490D43440D4FF301E0BC7
:1056B700EF24BFB41A0050032461FFE55E600215B2
:1056C7005E0561E5617002056030210D7846E4757D
:1056D700F001120A5DEF02075A02BA9B7403D22146
:1056E7008003E4C221F55D8B468A478948E4F55E6D
:1056F700F560F561E55E60077F201256C280F5759B
:105707005FFFC21BC21AC21CC21DC21FC220C22217
:10571700125690FF700D3021057F001256D3AF61EE
:10572700AE6022B4255FC2D5C21E125690FF24D0A8
:10573700B40A00501A75F00A785E30D50508B6FF2E
:105747000106C6A426F620D5047002D21D80D924EE
:10575700CFB41A00EF5004C2E5D21E0259C0D21BC3
:1057670080C6D21A80C0D21C80BCD2D580BAD21FC4
:1057770080B47F201256C2201C077401B55E00401A
:10578700F1125687FF1256C20256FBD222D2208050
:1057970095125687FB125687FA125687F94A4B70AD
:1057A7000679B77A5A7BFF201C2EE55E602A7E00B9
:1057B7008E8275830012072D60060EEE655F70F00E
:1057C700C2D5EBC0E0EAC0E0E9C0E0EE125A20D053
:1057D700E0F9D0E0FAD0E0FB120714FF60AAEBC0B3
:1057E700E0EAC0E0E9C0E01256C2D0E02401F9D0F7
:1057F700E03400FAD0E0FBE55F0460DCD55FD980D8
:1058070087D21C80A2125A0360F7E55F7001041269
:10581700047CA95F600DE55F600914F55F125AAA61
:10582700EF60F3EA30E702F404C3995077EAF4250E
:105837005F0430E701E404F55F800D125A0360C18D
:10584700EA055F255F12047CEA785CF630E701E43D
:10585700255F04D55F04201F0114125A20E4C0E01D
:10586700125AAA785CE6601320E70714F61256AAC4
:10587700802204F6D0E014C0E07F001256AAE55F4C
:1058870060071256A1155F800B301F031256A1D077
:10589700E00256FBD0E00480C5125A0360A0E55F22
:1058A7000412047C785CEAF6E55F201F02600104BD
:0558B7002404125A2038
:1058BC0074FF04C0E0125AAA1256AAE55F201F0218
:1058CC0060031256A1D0E0B55FE87F451256B4785C
:1058DC005CE67F2B30E7047F2DF404C0E01256C247
:1058EC00D0E075F00A84C0F01256ABD0E01256AB83
:1058FC000256FB791080027908C220C2228008D29D
:10590C00D5790A8004790AC2D5E55F047002F55F87
:10591C00E4FAFDFEFF125687FC7B08201B1312567F
:10592C0087FD7B10301A0A125687FE125687FF7BB2
:10593C0020EC3382D592D55013C3E4301A069FFF66
:10594C00E49EFEE4201B039DFDE49CFCE4CBF8C22A
:10595C001BEC700CCFCECDCCE824F8F870F380178C
:10596C00C3EF33FFEE33FEED33FDEC33FCEB33FBD7
:10597C00994002FB0FD8E9EB301B05F8D0E0C44886
:10598C00B21BC0E00AEC4D4E4F78207B0070C2EA8F
:10599C00B55F0040BCC0E0125A22D0F0D0E0201B12
:1059AC0004C4C0E0C4B21BC0F01256ABD0F0D5F0AA
:1059BC00EB0256FB120AF657985358FF5857694C8E
:1059CC0057654259034F590B44590B49577E43595C
:1059DC00115558424658A045580C475AD750576D48
:1059EC002D57712E57942B5775235792205AC02A36
:1059FC00572D480000578CE55FB4FF03755F061206
:105A0C005687FC125687FD125687FE125687FF7872
:105A1C00550204AB790AA2D5201D14301F09B91008
:105A2C00020404B9080104A2D5202002500104206C
:105A3C001C68921CB55E005034C0E07F20301D19EC
:105A4C007F30A21C7220721F500F125A79C21CC2D6
:105A5C0020C21FC2227F30800F301F03E9C0E0122A
:105A6C0056C2301F03D0E0F9D0E0B55ECC301F1722
:105A7C007F30B9100C1256C27F58301E077F7880C9
:105A8C0003B908031256C2301C057F2D0256C27F83
:105A9C00202022F87F2B2020F322921C80CF7F0025
:105AAC00B4070050052455F8E6FF22286E756C6C7F
:105ABC002900D21B125687301BF8C21B785E30D5DA
:105ACC000108F602572D2D504349581256872403CE
:105ADC00B405004001E4905AD2931256B3743A12B2
:0A5AEC0056B3D21D755E040258FF88
:0DBB6B00ED33EC3360065004EC6480FC22E6
:10A4A0008F498E488D478C4674FFFFFEFDFCAB49FB
:10A4B000AA48A947A846C31208D1602C7F807E967F
:10A4C0007D187C4BAB49AA48A947A84612034460B3
:10A4D0000250157F807E967D187CCBAB49AA48A997
:10A4E00047A8461203445009AF49AE48AD47AC46B1
:10A4F00022AF49AE48AD47AC461203FB8F4D8E4CA0
:10A500008D4B8C4AEC1203BDC8ECC8C9EDC9CAEE2C
:10A51000CACBEFCBAF49AE48AD47AC461200A9E479
:10A52000FBFAF9F8120344601A401874FF254DF540
:10A530004DE54C34FFF54CE54B34FFF54BE54A3423
:10A54000FFF54AAF4DAE4CAD4BAC4AEC1203BD2209
:10043200E9D2E7C933E833F892D5EDD2E7CD33EC10
:0704420033FC5002B2D52289
:10044900EC30E7100FBF000C0EBE00080DBD000414
:100459000BEB6014A2D5EB13FCED92E7FD2274FFC0
:10046900FCFDFEFF22E480F8A2D574FF13FC7D8019
:03047900E480EF2D
:10047C00F920E72824F950037907E4F42402FB1847
:10048C00DBFDE624FB5014E9600DE4F618E604F6F7
:0F049C00B40A08E4F6D9F57401F60A22C2D52293
:1004AB00ED33EC3392D5FA602AB4FF33EDC2E77B20
:1004BB00FF60067A0479D0E4227A0479D920D50436
:1004CB007A0479D4224E614E002B494E46002D49B9
:1004DB004E4600E47A08F608DAFC7B00740722E843
:1004EB00C0E0ECC0E0EDC0E0EEC0E0EFC0E0EA75CC
:1004FB00F010A4CAABF075F04DA42BFBE435F0FC67
:10050B00EA2410FAEB34C5FBEC34D9FCEDC2E7FF5F
:10051B0075F056A4F42411C5F0F434C58FF0A42A59
:10052B00E5F03BE43CF620E7141205DED0E0FFD00B
:10053B00E0FED0E0FDD0E0FC1202A78014F4041220
:10054B0005DED0E0FFD0E0FED0E0FDD0E0FC1201F4
:10055B009ED0E0F8E6FAEDD2E7CD33EC332482FB04
:10056B00E4C3CF33CFCE33CECD33CD33DBF37B07E9
:10057B0075F00A846004F6081B0AE5F0F6088FF0A4
:10058B00740AA4FFACF08EF0740AA42CFEACF050ED
:10059B00010C8DF0740AA42CFDE435F0F608DBDEBB
:0305AB00740722B0
:1005AE003F8000004120000042C80000447A000055
:1005BE00461C400047C35000497424004B189680D7
:1005CE004CBEBC205A0E1BCA6753C21C749DC5AECE
:1005DE00FB60065407601C232312060CEB54386094
:1005EE00091205F812060712019EECF8EDF9EEFA63
:1005FE00EFCB22EB12060780F1543803241C900532
:10060E00AEFE93FC0EEE93FD0EEE930ECE93FF22F6
:0300000002AD123C
:0CAD1200787FE4F6D8FD7581B202AD59DF
:10061E00E709F608DFFA8046E709F208DFFA803EBE
:10062E0088828C83E709F0A3DFFA8032E309F608AB
:10063E00DFFA8078E309F208DFFA807088828C8313
:10064E00E309F0A3DFFA806489828A83E0A3F608C7
:10065E00DFFA805889828A83E0A3F208DFFA804CA1
:10066E0080D280FA80C680D4806980F28033801078
:10067E0080A680EA809A80A880DA80E280CA8033E1
:10068E0089828A83ECFAE493A3C8C582C8CCC58359
:10069E00CCF0A3C8C582C8CCC583CCDFE9DEE78029
:1006AE000D89828A83E493A3F608DFF9ECFAA9F0A8
:1006BE00EDFB2289828A83ECFAE0A3C8C582C8CCFE
:1006CE00C583CCF0A3C8C582C8CCC583CCDFEADE17
:1006DE00E880DB89828A83E493A3F208DFF980CC79
:1006EE0088F0EF60010E4E60C388F0ED2402B40472
:1006FE000050B9F582EB2402B4040050AF23234519
:06070E00822390066E73C9
:10071400BB010689828A83E0225002E722BBFE02E3
:09072400E32289828A83E4932216
:10072D00BB010CE58229F582E5833AF583E0225081
:10073D0006E92582F8E622BBFE06E92582F8E222CB
:0D074D00E58229F582E5833AF583E49322E5
:10075A00BB010689828A83F0225002F722BBFE017E
:02076A00F32278
:10076C00F8BB010DE58229F582E5833AF583E8F0C3
:10077C00225006E92582C8F622BBFE05E92582C86F
:02078C00F22257
:10078E00EF8DF0A4A8F0CF8CF0A428CE8DF0A42E7F
:02079E00FE2239
:1007A000BC000BBE0029EF8DF084FFADF022E4CC3D
:1007B000F875F008EF2FFFEE33FEEC33FCEE9DEC06
:1007C000984005FCEE9DFE0FD5F0E9E4CEFD22ED4C
:1007D000F8F5F0EE8420D21CFEADF075F008EF2F96
:1007E000FFED33FD4007985006D5F0F222C398FD87
:0507F0000FD5F0EA2224
:1007F500C2D5EC30E709B2D5E4C39DFDE49CFCEE1F
:1008050030E715B2D5E4C39FFFE49EFE1207A0C3EF
:10081500E49DFDE49CFC80031207A030D507C3E4EA
:060825009FFFE49EFE228D
:10082B00BB010A89828A83E0F5F0A3E02250068798
:10083B00F009E71922BBFE07E3F5F009E31922895A
:0B084B00828A83E493F5F0740193228D
:10085600BB010789828A83020B4E500B09C5F0271C
:10086600F7C5F01937F722BBFE0D09F8E325F0F3BB
:10087600C5F019E338F322F889828A837401932537
:08088600F0C5F0F8E4933822FC
:10088E00BB010A89828A83F0E5F0A3F0225006F7B5
:0F089E0009A7F01922BBFE06F3E5F009F31922B2
:0E08AD00C3E49FFFE49EFEE49DFDE49CFC225C
:1008BB00EB9FF5F0EA9E42F0E99D42F0EC6480C8B4
:0608CB0064809845F02254
:1008D100EB9FF5F0EA9E42F0E99D42F0E89C45F07D
:0108E10022F4
:1008E200E8600FEFC333FFEE33FEED33FDEC33FC74
:0308F200D8F12218
:1008F500BB010789828A8302096B5005E9F8020961
:100905005FBBFE05E9F8020B6489828A83020B70DE
:10091500BB010DE58229F582E5833AF58302096B72
:100925005007E92582F802095FBBFE07E92582F831
:10093500020B64E58229F582E5833AF583020B70A3
:10094500BB010789828A830209DC5005E9F802099F
:0A095500D0BBFE05E9F8020B8D226D
:0C095F00E6FC08E6FD08E6FE08E6FF22C4
:0C096B00E0FCA3E0FDA3E0FEA3E0FF22FF
:0D097700E6FB08E6F908E6FA08E6CBF822F0
:0C098400E0F8A3E0F9A3E0FAA3E0FB22F6
:10099000E493F8740193F9740293FA740393FB22BD
:1009A000BB010DE58229F582E5833AF583020984CE
:1009B0005007E92582F8020977BBFE07E92582F88E
:1009C000020B80E58229F582E5833AF583020990DE
:0C09D000ECF608EDF608EEF608EFF62253
:0C09DC00ECF0A3EDF0A3EEF0A3EFF0228E
:1009E800D083D082E493F608740193F608740293D6
:0909F800F608740393F67404730D
:100A0100A8828583F0D083D082120A18120A1812A4
:100A11000A18120A18E473E493A3C583C5F0C583C9
:100A2100C8C582C8F0A3C583C5F0C583C8C582C83F
:010A310022A2
:100A3200BB010789828A83020A015005E9F802098B
:0A0A4200E8BBFE05E9F8020B99225B
:100A4C00F5F0C582A4C582C5F0C583A42583F583C2
:010A5C002277
:100A5D00FAE6FB0808E6F925F0F618E6CA3AF6229A
:100A6D00BB010DE58229F582E5833AF583020BC4BE
:100A7D005007E92582F8020BB2BBFE07E92582F883
:100A8D00020BD6E58229F582E5833AF583020BE860
:100A9D00BB0120E58229F582E5833AF583D0F0D0BC
:100AAD00E0F8D0E0F9D0E0FAD0E0FBE8C0E0C0F02B
:100ABD00020BCD5018E92582F8D083D082D0E0F911
:100ACD00D0E0FAD0E0FBC082C083020BBBBBFE18A6
:100ADD00E92582F8D083D082D0E0F9D0E0FAD0E0D9
:090AED00FBC082C083020BDF2272
:100AF600D083D082F8E4937012740193700DA3A38F
:100B060093F8740193F5828883E4737402936860A2
:060B1600EFA3A3A380DFA2
:060B1C008A838982E47364
:10B8F000120714601CFF09E970010AC0E0EAC0E009
:10B90000EBC0E012BA9BD0E0FBD0E0FAD0E0F980C7
:0AB91000DF7F0A12BA9BE4FEFF225B
:10B2F1008B458A4689478B4B8A4C894DAB4505471F
:10B30100E547AA467002054614F912071470ED7458
:10B31100FF2547F54774FF3546F546AB48054AE535
:10B321004AAA497002054914F9120714FFAB4505F1
:10B3310047E547AA467002054614F9EF12075A700D
:08B34100DAAB4BAA4CA94D2226
:10B3F5008B458A468947E4F54DF54EE54C154CAE2F
:10B405004B7002154B4E6033AB48AA49A94A120747
:10B4150014FFAB45AA46A947054EE54EAC4D700253
:10B42500054D14F5828C83EF12076CEF60CD740126
:10B43500254AF54AE43549F54980C0AB45AA46A9F0
:02B4450047229C
:10BAB100E4FFFE120714600C0FEF70010E09E9702C
:05BAC100F20A80EF22F3
:10BA0400E94A4B700122120714FF6D700122EF7096
:0CBA140004FBFAF92209E970ED0A80EA4F
:10B39F008B478A4889498B4A8A4B894CAB4AAA4BBF
:10B3AF00A94C120714600D7401254CF54CE4354B74
:10B3BF00F54B80E8AB4AAA4BA94C1207146D7001EC
:10B3CF0022E54C154CAA4B7002154BF9E547854801
:10B3DF0083854982654A7008E965827003EA65834F
:06B3EF0070D2FBFAF92206
:100B2200EF4E6012EF60010EEDBB010B89828A83EA
:100B3200F0A3DFFCDEFA2289F05007F709DFFCA9F7
:0C0B4200F022BBFEFCF309DFFCA9F0224E
:10AD1E0002000EE493A3F8E493A34003F68001F23D
:10AD2E0008DFF48029E493A3F85407240CC8C33336
:10AD3E00C4540F4420C8834004F456800146F6DF05
:10AD4E00E4800B010204081020408090B66AE47E75
:10AD5E00019360BCA3FF543F30E509541FFEE493FA
:10AD6E00A360010ECF54C025E060A840B8E493A3C1
:10AD7E00FAE493A3F8E493A3C8C582C8CAC583CAEC
:10AD8E00F0A3C8C582C8CAC583CADFE9DEE780BEA4
:01B6B0000099
:100B4E00C5F0F8A3E028F0C5F0F8E5821582700232
:060B5E001583E038F022CF
:0C0B6400E2FC08E2FD08E2FE08E2FF22CD
:100B7000E493FC740193FD740293FE740393FF22CB
:0D0B8000E2FB08E2F908E2FA08E2CBF822F5
:0C0B8D00ECF208EDF208EEF208EFF222A4
:100B9900D083D082E493F208740193F2087402932B
:090BA900F208740393F274047362
:090BB200E6FB08E6FA08E6F92268
:090BBB00EBF608EAF608E9F6225F
:090BC400E0FBA3E0FAA3E0F92232
:090BCD00EBF0A3EAF0A3E9F02229
:090BD600E2FB08E2FA08E2F92250
:090BDF00EBF208EAF208E9F22247
:0C0BE800E493FB740193FA740293F92269
:00000001FF
